:1000000000800020BD010000A1DA000059DA0000E4
:1000100059DA000059DA000059DA000059DA000014
:1000200059DA000059DA000059DA0000A1DA0000BC
:10003000A1DA000059DA000021D1000025D2000029
:10004000A1DA0000A1DA0000A1DA0000A1DA0000C4
:10005000A1DA0000A1DA0000A1DA0000A1DA0000B4
:10006000A1DA0000A1DA0000A1DA0000A1DA0000A4
:10007000A1DA0000A1DA0000A1DA0000A1DA000094
:10008000A1DA0000A1DA0000A1DA0000A1DA000084
:10009000A1DA0000A1DA0000A1DA0000A1DA000074
:1000A0005DB6000069B60000A1DA0000A1DA000028
:1000B000A1DA0000A1DA0000A1DA0000A1DA000054
:1000C000A1DA0000A1DA0000A1DA0000A1DA000044
:1000D000A1DA0000A1DA0000A1DA0000A1DA000034
:1000E000A1DA0000A1DA0000A1DA0000A1DA000024
:1000F000A1DA00000DFB0000A1DA000039FC0000CD
:10010000A1DA000079E40000A1DA0000A1DA000021
:10011000A1DA0000A1DA0000A1DA0000A1DA0000F3
:10012000A1DA0000A1DA0000A1DA0000A1DA0000E3
:10013000A1DA0000A1DA0000A1DA0000A1DA0000D3
:10014000A1DA0000A1DA0000A1DA0000A1DA0000C3
:1001500011D3000025D3000039D300004DD3000097
:10016000A1DA000095E70000A1DA0000A1DA0000A2
:10017000A1DA0000A1DA0000A1DA0000A1DA000093
:10018000A1DA0000A1DA0000A1DA0000A1DA000083
:10019000A1DA0000A1DA0000A1DA0000A1DA000073
:1001A000A1DA0000A1DA0000A1DA0000A1DA000063
:1001B000A1DA0000A1DA0000A1DA0000564B4CF2EF
:1001C000205210B51A804DF628121A8000BF00BFC9
:1001D0000DF06AFC514B4FF010621A60504A9A6061
:1001E000504ADA60504A136813F4807304D14F49BF
:1001F0000B604FF4A85313604D4B1A78110703D5C9
:100200001A7842F008021A704A4B4B492A221A7097
:100210004A4A4B4B8B4204D252F8040F43F8040B6A
:10022000F8E7484B484900228B4202D243F8042B9E
:10023000FAE74649464A002352F8230041F82300D2
:1002400001336F2BF8D1434B434A802103F8011B44
:100250009342FBD1414B3D4A1A60414B8A221A70AE
:10026000A3F5805324225A70A0221A709A7992071B
:10027000FCD59A79D406FCD43A4A937903F00C035E
:10028000082B384BF9D103221A7140225A719A79FE
:100290009006FCD5334A9179324B4906FBD5324A58
:1002A000324911600221516020221A709A7902F0BD
:1002B0000C020C2AFAD12E4B2E4A1A602E4B2F4AD2
:1002C0001A6000225A60072243F8042C2C4AC3F813
:1002D0000C2D62B60DF098FF144B1B68DA0705D59C
:1002E00028480DF065FD284B284A1A60284B1B78DA
:1002F0005B0609D5244C254B22689A4204D121483B
:100300000DF056FD0023236010F04EFF0DF0D2FBE0
:100310000DF000FBFEE700BF0E20054030800440DA
:10032000823F04000100002B10D0034014D0034092
:1003300002D0074000E007406C9CFF1FA44B010067
:100340004088FF1F6C9CFF1FA4A4FF1F0082FF1F9B
:100350000000000000E400E05FE400E008ED00E0E1
:100360000050064000400640448004400000030165
:1003700004800440C010050014E000E0FF76010096
:1003800000002020D801825F1CE00340A5C3945ADE
:1003900000F00740FFFFFFFFFFFFFFFFFFFFFFFF32
:1003A000FFFFFFFFFFFFFFFFFFFFFFFFFFFFFFFF5D
:1003B000FFFFFFFFFFFFFFFFFFFFFFFFFFFFFFFF4D
:1003C000FFFFFFFFFFFFFFFFFFFFFFFFFFFFFFFF3D
:1003D000FFFFFFFFFFFFFFFFFFFFFFFFFFFFFFFF2D
:1003E000FFFFFFFFFFFFFFFFFFFFFFFFFFFFFFFF1D
:1003F000FFFFFFFFFFFFFFFFFFFFFFFFFFFFFFFF0D
:10040000FFFFFFFFFFFFFFFFFFFFFFFFDEF9FFFF23
:1004100010B5054C237833B9044B13B10448AFF33E
:1004200000800123237010BD6C9CFF1F00000000A2
:10043000A84B0100084B10B51BB108490848AFF3A1
:1004400000800848036803B910BD074B002BFBD0A0
:10045000BDE81040184700BF00000000709CFF1F5F
:10046000A84B01006C9CFF1F0000000038B504463B
:10047000104621700A491D4610F078FC01464FF0E5
:100480007E5010F027FD074910F070FCE5606060B9
:10049000256165610DF048FEE061204638BD00BF72
:1004A000DB0FC9400024744938B50446104621705A
:1004B00009491D4610F05AFC01464FF07E5010F0DD
:1004C00009FD064910F052FCE56060602561656138
:1004D0000DF02AFEE06138BDDB0FC94000247449ED
:1004E00038B503780446032B20D8DFE803F01A1848
:1004F0001002C168406910F02FFB0D490546606885
:1005000010F0E8FC0146284610F0E4FC38BD08492C
:10051000406810F0DFFCE16810F028FC38BDC068CE
:1005200038BDC168406910F017FB38BD002038BDE8
:100530000024744970B504460E460DF0F5FD0546DD
:10054000E069281A10F0BEFBE3682361E56166618B
:10055000A0610146606810F0BDFC0146A060104833
:1005600010F0B8FC0FF08EFF0FF02EFC10F0A0FA88
:10057000054601464FF07E5010F0EEFA616910F02A
:10058000F5FB21690646284610F0F0FB014630468F
:1005900010F0E4FAE0602046BDE87040FFF7A0BF2D
:1005A000000080BF38B50E201C4C0DF08DF821885E
:1005B0001B4B884205461A881DDA0023511AB1F5F3
:1005C000805FAABF1B03C3EB03330131142093FBED
:1005D000F1F10DF0FFFB134B1988F1B923889D420F
:1005E00010DAC3F57F630F33282091FBF3F1BDE8E8
:1005F00038400DF0EFBB9042D4BFC1EB0003C1EB1C
:100600000203DBE740F6FF718D42D4BFC3EB050167
:10061000C3EB0101C1EB0131E3E738BD689DFF1F6A
:10062000349FFF1FD49EFF1F10B504460CF04EFEF2
:10063000204610BD70B44C88A04220D9012301335C
:10064000DBB21CB2660031F8144084421D46F6D37A
:10065000A04211D005F10045013D965B31F815101F
:1006600032F81530401AF21A00FB02F0641A90FBBF
:10067000F4F4E01870BC7047905B70BC70470226C1
:100680000125E5E700280CDA064A434282FB0320F5
:10069000DA17C2EB600000EB4000A3EB8000C0F172
:1006A0000C007047ABAAAA2A38B5234B1B78002B45
:1006B0002CD015200DF008F8204B1860204B1B881B
:1006C000984203DA1F4C237863BB38BD1E4A148856
:1006D000A042A4EB0302A8BF20467F2A1CDDC01A5B
:1006E000C001541C90FBF4F4002CEBD0154B1A788D
:1006F0000AB901221A70154D2B689C4204D0144B84
:10070000E1B2187809F090F82C6038BD11200DF096
:100710001FFF0A4B1860D1E7C01AC0EBC01090FB56
:10072000F2F4E1E70A4B0021187809F07DF8002384
:10073000064A2370136038BD889EFF1F989CFF1FD8
:100740000E9DFF1F609FFF1F009FFF1F589FFF1FF1
:10075000E89CFF1F38B50F200DF0FAFE1B4A1C4B1A
:1007600012881860C0F53B600830904220DB194BBE
:100770001B889842A3EB0204A8BF1846801A7F2C5E
:10078000C6BFC0010134C0EBC01090FBF4F47CB1D3
:10079000114B1A780AB901221A70104D2B689C422D
:1007A00004D00F4BE1B2187809F03EF82C6038BD48
:1007B000094C237803B938BD094B0021187809F09A
:1007C00033F80023054A2370136038BD6C9DFF1F6A
:1007D000809EFF1FEC9EFF1F109FFF1F1C9DFF1F91
:1007E000069DFF1FF0B40E8886420DD203F1004330
:1007F000013B31F81350854202D9F0BCFFF71ABF14
:1008000032F81300F0BC70471088F0BC704700BF8E
:10081000094B1B880C2B09D8084A80B252F82320B8
:1008200028B143F6FE73984203D9108C70471088A4
:1008300070470349FFF7FEBEBE9CFF1F0426010060
:10084000A02701004B4B4C4A2DE9F0471E88146845
:100850004A4BB442B3F80080494B33DB4445A8BF50
:100860004446A6421C60C8BF00202DDDC6EB080729
:10087000B7F5804F33DB80037B1C90FBF3F0FFF771
:10088000C7FF404A404B15881B88C0F3C61909FBB7
:1008900005F57F2D8246A8BF7F252BB3A64253DCEA
:1008A0004445D4BFC6EB0404C6EB08049F42CCBF4A
:1008B00003FB04445C43354BC8BF013794FBF7F797
:1008C0001F6013E034461E60C6EB0807A045D4BF86
:1008D000C6EB0800C6EB0400B7F5804FCBDAC0EBDF
:1008E000803090FBF7F0CAE7284A1360284C236851
:1008F000994508D0274B1B88002B34D1264B1B88E9
:100900006BBBC4F80090254C23689A4506D0214B58
:100910001B885A1F032A19D9C4F800A0204C236849
:100920009D420FD01F4B188848B11A4B1E4A1B8896
:10093000D35C834203D0C0B2E9B208F075FF2560F2
:10094000BDE8F087BDE8F0870024AFE7164AD05C29
:100950002030C0B20AF07F0108F066FFDCE74846AD
:1009600008F0D6FFCDE7104A4946D05C08F05CFF9E
:10097000C4E700BF689DFF1FD09EFF1F349FFF1F6D
:10098000909CFF1FA09CFF1FA29CFF1F389FFF1F72
:10099000009DFF1FB89EFF1F5A9DFF1FB89CFF1FA1
:1009A0005C9DFF1FC69EFF1F0C8AFF1F2DE9F04FA5
:1009B00001208BB00DF0CCFDDFF870B3DFF870A331
:1009C000CBF8000000200DF0C3FDBA4BCAF80000C0
:1009D0001B880C2B00F05E82B74EB84A3188B84BAA
:1009E00052F8214000221A70B64BB74A1B88B7490B
:1009F0001288013B012A31F91330059300F0AE81D2
:100A0000B34B0193B34B0293B34FDFF8288300231A
:100A10000093B24B1B88012B00F0F481DFF8189390
:100A2000AF4B0393D9F80050AE4B04930023AE4A6A
:100A30001288013A032A00F24982DFE812F0A50089
:100A4000ED000400C9002846059310F03BF9A749C2
:100A500010F08CF9059B0546184610F033F9A449AF
:100A600010F084F90146284610F078F810F044FBA5
:100A70000546C9F80050386810F024F99B4910F079
:100A800075F98146009810F01DF9994910F06EF93A
:100A90000146484610F062F810F02EFB3860954A87
:100AA000954B17881988954BDBF800201B88DFF8D9
:100AB0008CE2C7EB050C3D44039FC7F800C0471A02
:100AC000084404990D6001990F600299BEF8007006
:100AD00008609A4280F2E7800025C3EB070E744558
:100AE000DAF8000080F2D380611C984205FB01F522
:100AF0000EF1010E95FBFEF5C0F25F838742A8BFA1
:100B00000746FF1A01FB07F494FBFEF49A4200F338
:100B1000A780984200F3A480794C206810F0D2F8A6
:100B2000784910F023F9784910F018F810F0E4FA39
:100B3000A0F5FF531C3B082B98BF4FF40050D8F88A
:100B40000030184400282060C0F29F80B0F5804F2C
:100B500080F2F6806D4B1B781BB1B0F5005F40F062
:100B6000F7806B4D2B78002B40F0AB81694D2068EE
:100B70002B68634C984204D080B208F033FF23689E
:100B80002B600BB0BDE8F08F2846059310F09AF863
:100B9000614910F0EBF8059B0546184610F092F8F5
:100BA0005E4910F0E3F8014628460FF0D7FF10F039
:100BB000A3FA0546C9F80050386810F083F8564982
:100BC00010F0D4F88146009810F07CF853495DE7A6
:100BD0002846059310F076F84A4910F0C7F8059BAF
:100BE0000546184610F06EF84D4910F0BFF8014662
:100BF00028460FF0B3FF10F07FFA0546C9F8005001
:100C0000386810F05FF83F4910F0B0F8814600985E
:100C100010F058F8424939E72846059310F052F889
:100C2000404910F0A3F8059B0546184610F04AF815
:100C30003D4910F09BF8014628460FF08FFF10F059
:100C40005BFA0546C9F80050386810F03BF83549A2
:100C500010F08CF88146009810F034F8324915E70E
:100C60003388002B3FF458AF2B1B002BB8BF5B42DF
:100C7000092B00F32D81D8F80030214C4FF400509F
:100C8000184400282060BFF661AF00225AE0984265
:100C900005FB04F5B8BF002195FBFEF580F28482C8
:100CA00091FBFEF432E7BA42D4BFC3EB0205C3EBBB
:100CB000070512E7029FFF1FF69CFF1F8889FF1F91
:100CC000969CFF1F2089FF1FD69EFF1FE02A010070
:100CD0005C9FFF1F2C9DFF1F889CFF1F649EFF1FB2
:100CE000F49EFF1F689EFF1F5E89FF1FCDCC4C3F07
:100CF000CDCC4C3E188AFF1F5C89FF1FCC9EFF1F86
:100D0000C089FF1F9A99193FCDCC4C4512A0FF1FF7
:100D1000589DFF1F2489FF1F3333733FCDCC4C3DBB
:100D2000CDCCCC3E6666663FCDCCCC3DF09CFF1F63
:100D3000B49CFF1F0C9FFF1FF09EFF1FD49CFF1F42
:100D400043F6FF72C04B22601B78002B3FF409AFC3
:100D500005F03EFFBD4B01221A7007E7BC4BBD4AB0
:100D60001B88BD491278013B31F91350002A40F02D
:100D7000C78011200DF0ECFB0090B84B0193D3F825
:100D80000080009B984540F3C080B54BB54F1B8851
:100D9000B54A012B3B68B2F80090B44A0292204653
:100DA000A3EB050500F0E2800FF08CFF029A52F8E9
:100DB00029100FF0DBFF014600200FF0CDFE10F0F0
:100DC0009BF9009BC8EB05029D42B8BF1D469042AF
:100DD000C8EB050580F2DE8000FB0555013295FB6E
:100DE000F2F5A34BDFF8B4820293D8F800302B441D
:100DF00003EBD3735B10C8F800309E4B1B88012BAC
:100E00007FF40CAE9C4B03931D460F200DF0A0FB0E
:100E10002A6804929042034680F2CC80904A12885D
:100E2000012A00F03F81904A079012888F4D069268
:100E300020460FF047FF069ADFF8649255F822101B
:100E4000D9F800500FF092FF014600200FF084FE09
:100E5000059BEA1A059210F04FF9059A079B049931
:100E60009A42C1EB020EB8BF1A46704580F2448127
:100E7000521A00FB02220EF1010192FBF1F2D8F8A6
:100E800000107E4804900A4402EBD2725210C8F857
:100E90000020CCE57A4B1B78002B3FF49DAD794EBA
:100EA000794A3188794B52F8210001221A700FF0EB
:100EB00009FF4FF07C510FF059FF10F01DF9044667
:100EC00092E505F081FE00232B704FE63868E6E5D9
:100ED00005F500500130001B0FF0F4FE6C496D4C1D
:100EE0000FF044FF054620680FF0ECFE6A490FF052
:100EF0003DFF014628460FF031FE10F0FDF81EE6DA
:100F000015200CF0E1FB009037E7594B0293D3F822
:100F10000080009B984542DA514B524F1B88524A41
:100F2000012B3B68B2F80090504A039220461D44C2
:100F300000F0E9800FF0C6FE039A52F829100FF076
:100F400015FF10F0D9F8009B9D42C8EB0502A8BF21
:100F50001D46C8EB05059042BABF00FB055501329E
:100F6000454395FBF2F5DFF834813EE70FF0AAFE2A
:100F7000029A52F829100FF0F9FE10F0BDF8009B0C
:100F8000C8EB05029D42B8BF1D468242C8EB05056D
:100F90003FF722AF00FB05F595FBF2F521E7DFF8FF
:100FA000FC80304FD8F8003003EBD3735B10C8F8E7
:100FB00000302EE5314A049212680692904237DDE5
:100FC000274A1288012A00F0BC80274A099011881C
:100FD000264A0891204607920FF074FE079A089956
:100FE000DFF8BC9052F82110D9F800500FF0BEFE87
:100FF000059B2B44059310F07FF80599099B069AF1
:101000009942C2EB010EA8BF1946704580F2BE801E
:10101000891A00FB01110EF1010291FBF2F2D8F8DE
:1010200000100A4402EBD2725210C8F80020FEE40D
:10103000D8F80020DFF8689002EBD2725210D9F88D
:101040000050C8F80020F2E412A0FF1F589DFF1FB7
:10105000648AFF1F889EFF1F582701005C9FFF1FA7
:101060003E9DFF1F889CFF1FDC9CFF1FF82A01008C
:101070002C9DFF1F649EFF1FF49EFF1F689EFF1F95
:10108000AC9CFF1FF69CFF1F8889FF1F969CFF1FCB
:10109000CDCCCC3EC089FF1F9A99193F0C9FFF1FF2
:1010A000F09EFF1F464A08901188464A0791204645
:1010B00006920FF007FE069A0799DFF80C9152F896
:1010C0002110D9F800500FF051FE059BE91A059147
:1010D00010F012F80599089B049A9942C2EB010E90
:1010E000B8BF1946704558DA891A00FB01110EF194
:1010F000010291FBF2F2C2E60499521A00FB02F2DD
:1011000092FBFEF2BBE60FF0DDFD039A52F82910C8
:101110000FF02CFE014600200FF01EFD0FF0ECFF3B
:10112000009A9542C8EB0503A8BF1546C8EB050514
:101130009842BABF00FB05550133454395FBF3F5D3
:1011400011E71F491F4A089020460D8807920FF0AB
:10115000B9FD079ADFF8709052F82510D9F80050C1
:101160000FF004FE014600200FF0F6FC059B2B4417
:1011700005930FF0C1FF0599089B069A9942C2EBAF
:10118000010EA8BF19467045FFF642AF069A891AAC
:1011900000FB01F191FBFEF241E7049A891A00FB82
:1011A00001F191FBFEF26AE6B842D4BFC3EB000145
:1011B000C3EB070104FB01F172E51F46A1E400BF88
:1011C000DC9CFF1FF82A0100F09EFF1F08B5244B8E
:1011D0001B88FBB1234B1B78FBB1234B1B78E3B17E
:1011E000224B1B78CBB1224B1B78B3B1214B224849
:1011F0001A78C2B9214A2249008812880968024433
:10120000B1EB620F09DD01221A706420BDE80840CD
:1012100005F0F2BC174A117801B908BD1370BDE89A
:10122000084008F0A9BB154A1649008812880968C9
:101230000244B1EB620FF0DD00221A7008F09CFB53
:10124000642005F0D9FC642005F0D6FC642005F08C
:10125000D3FC4FF41670BDE808400CF087BF00BF08
:10126000769EFF1F309FFF1F319FFF1F329FFF1F82
:10127000339FFF1FBC9CFF1FD49CFF1FCC9EFF1FF2
:10128000F09CFF1FB49CFF1F38B5114C232025781C
:101290000CF01AFA0F4A42F82500131F02F1C4009D
:1012A000002253F8041F83420A44FAD123780A49E2
:1012B00007480A4C0133DBB2322B81FB025108BFD5
:1012C0000023D217C2EB21120370226038BD00BF89
:1012D000A49CFF1F789DFF1F1F85EB51C89EFF1F19
:1012E0002DE9F04FB84CB94D2068B94F83B00FF0DD
:1012F000E9FCB8490FF03AFD064610200DF028F938
:101300000FF0E0FCB4490FF031FD31460FF026FC40
:101310000FF0F2FE2988206088423B8843DA9E461F
:101320005B1A7F2B4FF0000247DDD2015E1C92FB5F
:10133000F6F2AA4EDFF8C882B6F800C0C8F800205E
:10134000BCF1190F00F0DF80BCF11A0F00F017811B
:10135000BCF11E0F00F020810126B146A04A128880
:10136000002A00F09D808842C0F207817045D4BFFA
:10137000C1EB0000C1EB0E009A42BABF02FB0000B5
:101380000133504390FBF3F3964A1360964B188851
:10139000C0B9964A1288AAB9954B197801B11A704A
:1013A00003B0BDE8F08F9842D4BFC1EB0002C1EB9F
:1013B00003029E465B1A7F2BB7DCC2EBC21292FB84
:1013C000F3F2B6E72988D4F800E0DFF80082DFF80E
:1013D000F8A171456CDCDFF818C29CF80020002AE7
:1013E0002ED14FF0010B04288CF800B028D1002E2C
:1013F00040F094817D4B18880028D1D0B9F1000FBE
:10140000CED023682C883A88A34280F265810023DD
:10141000141B7E2C774DD5BFC3EB8313C3EBC313D3
:101420005B00013493FBF4F42B680134A34203D036
:10143000C0B2E1B208F0F8F92C6003B0BDE8F08F5B
:10144000012800F0F680022800F0EB800328D1D1BB
:10145000694B1B88092BCDD0002ECBD023682E885A
:101460003A88B34280F27B810023961B7E2EDFF800
:101470008CA1D5BFC3EB8313C3EBC3135B00013651
:1014800093FBF6F6DAF800300136B34203D0F1B23E
:101490004A2008F0C9F9CAF80060ABE71646914641
:1014A000BCF11E0F7FF472AF0022DFF858817EE09E
:1014B0004F4B1A78002A3FF473AF002401281C70A8
:1014C00000F0A480022840F00E81002E00F0A380DE
:1014D0004A4D2B68002B00F09E800420214608F026
:1014E000A3F9424B2C60188800283FF459AFB9F19A
:1014F000000F3FF455AFC0B2002108F095F93D4B05
:1015000000221A604CE7DFF8FC8098F80020C2B196
:10151000DFF8D890B9F800A0BAF1000F11D0DFF8C9
:10152000E89099F800B0934578D05FFA8AF07F216F
:1015300008F07AF998F80030B6F800C089F8003061
:1015400010E0DFF8C49099F800A0924566D0274BD0
:101550000021187808F068F998F80030B6F800C053
:1015600089F800301E4B1A88002A97D0BCF11E0F54
:1015700040F006810026B14619E00020FCE6DFF8C5
:10158000848098F80020002A0BBF012600264FF027
:1015900000094FF00109E1E6DFF86880104B98F888
:1015A00000601A88B6FA86F676094FF0000998F8B6
:1015B0000030002B3FF4E8AE2988B7F800E020683F
:1015C000C1EB0E03CFE600BFE49CFF1F7C9EFF1F14
:1015D000789EFF1F9A99193FCDCCCC3E029FFF1FEA
:1015E0003C9FFF1F709DFF1FEC9CFF1F149FFF1F60
:1015F000089FFF1FC89CFF1FB89EFF1F749DFF1F01
:10160000E89EFF1FAC9CFF1FA89CFF1F1EB1614DF1
:101610002B68002B7BD1604B188865E70026B1460C
:101620009CE6002E3FF4E6AEDFF868A1DAF8002071
:101630002EE0002E3FF4DEAEB7F80080F045D4BFB8
:10164000C1EB0802C1EB0E02C1EB0808B8F17E0F36
:10165000DFF840A1D5BFC2EB8212C2EBC21252002A
:1016600008F1010892FBF8F8DAF8002008F1010807
:10167000424506D05FFA88F10120009308F0D4F8C3
:10168000009B1888CAF8008002287FF4DFAE42462B
:101690002168B5F800803888414559DA0021C8EB47
:1016A0000008B8F17E0FD3BFC1EB8111C1EBC111AE
:1016B00008F10108490091FBF8F808F1010890458C
:1016C00006D05FFA88F10420009308F0ADF8009B83
:1016D0001888CAF80080B9E69342D4BFC4EB03036C
:1016E000C4EB020394E6032827D12C4B1B88092B5B
:1016F00091D0002E8FD0274D2B68002B8BD04A2005
:10170000214608F091F8244B2C601888ECE621461D
:1017100008F08AF8204B2C601888E5E640207F21ED
:101720008DE80C0008F080F8019B009A1888584555
:101730001CD002287FF48AAE76E704287FF46BAFD2
:10174000002E3FF468AF2146402008F06DF862E7B4
:101750008142D4BFC8EB0101C8EB00019FE793426F
:10176000D4BFC6EB0303C6EB02037EE6B8F8001055
:10177000DAF800E0B7F800808E45FFF665AF5DE768
:101780002988B7F800E020680026C1EB0E03B146B7
:10179000E9E500BF749DFF1F149FFF1FB89EFF1F48
:1017A00008B5114B1B88022B09D0052B07D0032B42
:1017B00015D0042B0BD00D4B01221A7008BD7F21D0
:1017C000412008F031F8094B01221A7008BD7F2131
:1017D000092008F029F8054B01221A7008BD4021A4
:1017E000092008F021F8E6E76E9DFF1F129DFF1FFC
:1017F00038B5074B074D1B88052B044606D02B68D0
:10180000834203D0C1B2052008F00EF82C6038BD29
:101810006E9DFF1F1C9FFF1F38B5124D124C2B8869
:10182000052B12D022684AB9022B0ED0033B012BA4
:1018300013D90E4A00231370236038BD0021052000
:1018400007F0F2FF2B88022B04D10021412007F082
:10185000EBFFEEE7052BE9D1F7E70021092007F0C0
:10186000E3FFE6E76E9DFF1F1C9FFF1F129DFF1FFA
:10187000464B1B881D2B70B541D0454D0024454B70
:101880001B88022B16D0444B1B88022B54D028886F
:10189000424B002C1B780ADB8442A8BF044634B1BB
:1018A000002B3AD02046BDE87040FFF7A1BF002BC7
:1018B0002FD170BD3A4B1B78002B37D015200BF081
:1018C00003FF384B1860384A1288002ADBD0374AA9
:1018D000186811888142D6DC354B2A881B888342E0
:1018E000A3EB0106A8BF03465B1AB242BABF02FBD4
:1018F00003330136534393FBF6F31C44C3E72A4BEF
:101900001C888CB12B4B224D1C78002CB7D02C8816
:10191000B5E7BDE87040FFF77FBFFFF741FF204606
:10192000BDE87040FFF764BF194DA8E711200CF027
:101930000FFE1C4B1860C6E70F200CF009FE1A4B77
:101940001D4A1B881060002BA1D01C4AC0F53B63C8
:10195000118808338B429ADB194A288812889342EF
:10196000A2EB0105A8BF1346A842A3EB010306DAC8
:1019700000FB0333013593FBF5F31C4488E700FBC0
:1019800003F292FBF5F31C4482E700BF029FFF1FA6
:101990000A9FFF1FD69EFF1F649EFF1F129DFF1F01
:1019A000889EFF1F989CFF1F6E9DFF1F0E9DFF1FAF
:1019B000009FFF1FAC9CFF1F809EFF1F6C9DFF1FA1
:1019C000EC9EFF1FF8B510200CF0C2FDC830B0F53A
:1019D000FA7FC0F29680B0F57A6F0146A8BF4FF447
:1019E0007A6101F51673B3F57A6FA8BF4FF47A6385
:1019F0009BB289B2914A924C11802220238008F038
:101A000097F821888F4D904C242008F091F80E20F3
:101A10000BF05AFE40F6FF71C8308842A8BF084656
:101A200020EAE07000F5FA6283B28A42A8BF0A4653
:101A30000220194622802B8008F07AF821880420A1
:101A400008F076F801200CF083FD044600200CF02D
:101A50007FFDA042B8BF204600F1C801B1F5FA7F72
:101A6000C0F2D180B1F57A6FA8BF4FF47A6101F569
:101A70004873B3F57A6FA8BF4FF47A639BB289B20B
:101A8000724A734C11800A20238008F051F8218893
:101A90000C2008F04DF80F200CF05AFDC0F53F6106
:101AA0000431B1F5AF6FC0F2AB80B1F5FA6FA8BFEA
:101AB0004FF4FA6189B2674BC0F54360B0F5AF6F80
:101AC0001980C0F29A80B0F5FA6FA8BF4FF4FA609F
:101AD00083B2614CA420238008F02AF82188A62034
:101AE00008F026F815200BF0EFFD00F59671B1F522
:101AF0002F7F0BDB41F25C23994240F3898019462A
:101B000008E040F24C434FF4FA7173E740F214538B
:101B10004FF42F71514A1180514C524D23800620B1
:101B200008F006F82188504E082008F001F8002738
:101B30004FF4AF74F9B24D4809F004FE55F8043B78
:101B4000C3F5967300FB03F086FB0023C017C0EBC0
:101B50006310844207F10107A8BF0446062FE9D1AC
:101B6000434F414E0025E9B2424809F0EBFD57F8DA
:101B7000043BC3F5967300FB03F086FB0023C017FC
:101B8000C0EB6310844205F10105A8BF04460C2D8B
:101B9000E9D1394F344E0025E9B2384809F0D2FD79
:101BA00057F8043B304AC3F5967300FB03F086FBFD
:101BB0000013C017C0EB6310844205F10105A8BFF4
:101BC00004460C2DE8D1A4F11401312931DD40F295
:101BD0003A73A4F5B97403FB04F482FB0432E417EE
:101BE000A4EB621289B232322548264B01801A607A
:101BF0002A20BDE8F84007F09BBF4FF4AF6368E7C9
:101C00004FF4AF6157E740F214534FF4FA7137E7DE
:101C1000124A00F5617089B2B0F52F7F1180B8BF0C
:101C20004FF42F73FFF678AF8342A8BF03469BB2F1
:101C300072E740F26C723221D6E700BF7C9EFF1F34
:101C4000789EFF1F689DFF1F349FFF1FCC9EFF1FC4
:101C5000D49CFF1F6C9DFF1FEC9EFF1F0E9DFF1F5E
:101C6000009FFF1F4C8AFF1FB5814E1BC09CFF1FAA
:101C70001C8AFF1FF49CFF1F2C89FF1F609DFF1F04
:101C80002E9FFF1F088AFF1F2DE9F84F0C200BF035
:101C9000E7FC0C200CF09CF9C44914200CF0A8F9C6
:101CA000C349C44809F0E0F9022103200CF036FAD8
:101CB000022104200CF032FA022105200CF02EFA49
:101CC000022106200CF02AFA01210A200CF026FA43
:101CD000012109200CF022FA01210D200CF01EFA3E
:101CE000012128200CF01AFA012114200CF016FA18
:101CF000012116200CF012FA172001210CF00EFA27
:101D000004200CF0FDF9002844D005200CF0F8F96F
:101D1000002849D00023A84D06202B700CF0F0F9C4
:101D2000B0FA80F35B090024A44A137006F0F8FAB5
:101D30002E785EBB204607F025FFA14BA1491B88EA
:101D40000F88A14ADFF8E4E2A04DA3F5AF7140F29D
:101D50003A7303FB01F382FB0312DB17A3EB62135D
:101D6000323301210D20CEF800302F700CF0C2F973
:101D700064200CF0FBF94FF416710A200CF02AF8DD
:101D80005D21934809F01AFDA8B9FEE7BDE8F84FB8
:101D900009F07AB806200CF0B3F90028B5D1864DC9
:101DA000034628700124BFE703200CF0A9F9B0FA1C
:101DB00080F35B09AFE764200CF0D8F931460A20C4
:101DC0000CF008F84FF4967109200CF003F85C2130
:101DD000804809F0F3FC00B9FEE764200CF0C6F976
:101DE000314609200BF0F6FF4FF4967116200BF0E8
:101DF000F1FF5B21784809F0E1FC00B9FEE76420BF
:101E00000CF0B4F9314616200BF0E4FF4FF4967154
:101E100017200BF0DFFF64200CF0A8F931461720E3
:101E20000BF0D8FF64200CF0A1F931460D200CF026
:101E300061F96A4A6A481268DFF8F4B1DFF8A8A1CC
:101E4000684FDFF8F091DFF8F08100230121FEF701
:101E50002BFB0123CAF800603E60C9F800608BF8D4
:101E6000003004260F200CF073FBD9F80030034437
:101E70000E20C9F800300BF027FCDAF800309BF890
:101E800000200344CAF800301520002A7DD00BF052
:101E90001BFC3B681844386006F0010080F001002C
:101EA00004F09AFEB8F80030002B14BF4B20DC2061
:101EB0000CF05CF9013ED5D1D9F80030DAF80020F9
:101EC00049493868DFF874E1484E002BB8BF033346
:101ED000002AB8BF033292100A604549454A098872
:101EE00012880028B8BF03309B10801038605F1A3A
:101EF00019443160CEF800703F4E404F4049C9F858
:101F00000030C2EB000E0244C7F800E032600B6004
:101F10000CB1FFF757FDB8F800305BB94FF4FA7019
:101F200004F06AFE04F054FE06F022FD4FF4AF60A8
:101F30000CF01CF9334B012404201C600CF0E0F879
:101F400010B9314B28701C70304B1B881C2B23D0D0
:101F50002F4C04F1C80523200BF0B6FB44F8040F06
:101F600001200CF003F9A542F5D12A4A2A4B10783A
:101F7000187007F011FD04F027FE45F6BF522749FF
:101F80002748BDE8F84F0BF057B911200CF0E0FAE4
:101F90003B68184438607FE7224B18880028D7D068
:101FA000214BC0B2197807F03FFCD1E7001B374640
:101FB00040420F007491FF1FC49CFF1F6C9EFF1FC7
:101FC0002E9FFF1F049FFF1FB5814E1B289DFF1FE3
:101FD000C09CFF1F609DFF1FF49CFF1F2889FF1FEF
:101FE000949EFF1F889CFF1F9C9CFF1F689EFF1FE5
:101FF000188AFF1F5C89FF1F2C9DFF1F5C9FFF1F1E
:10200000449FFF1FFC9EFF1FAD9CFF1F029FFF1FF1
:10201000749DFF1F849EFF1F639EFF1FA505000088
:10202000249FFF1F309DFF1FE09CFF1F088AFF1F9A
:10203000889EFF1FF09EFF1FC29EFF1FF49EFF1F82
:102040002DE9F04FAD4C2678012E95B000F0558269
:10205000C0F00B82022E00F0D880A949A94A91F85D
:1020600000801178A84ADFF83CE3A84DA84FA948A2
:10207000A94B0292A94A0092A94A9EF800B0019287
:102080002D78A84A3F7890F800E01B78DFF818A375
:10209000DFF818C3DFF818930392012E84BF0022E3
:1020A0002270A14AA1481370A14A80F800B01570AF
:1020B000A048A14A077082F80080A048A04A037097
:1020C0009CBF013626701170BEF1000F40F0748184
:1020D0009C4A10880D2800F0B9819B4C002020708C
:1020E000024604462DB197480088002840F0BA8186
:1020F0000546964806882544002E40F0678194489E
:10210000944C019E0078367824780130A0EB46008C
:10211000002C40F05682039C94F800E0CEEB0004C3
:10212000BEF1000F40F076820026DFF874E20298DC
:102130009EF800E00078A41BA4EB4E043C44CBEBDB
:10214000040410B1B7FA87F040099CF80060271822
:10215000BC1B1EB11EF1000618BF0126009F99F896
:10216000000097F800909AF800C07B4FC6EB040E71
:10217000C0EB0E00A0EB49008044C3EB0803A3EBC7
:1021800041010C2313FB0C113960744B744F754CD7
:1021900075481B880088D7F800C0744E2788744C97
:1021A0003688D4F800E0033BC0EBC00403EB4303E4
:1021B000C7EBC70001EB830364446E4F33447044A4
:1021C0006D4E57F8244056F820000C3B1D44254422
:1021D00005440AB1694B1960694A13689D4200F0D1
:1021E0003181684B684819680791079901601B683D
:1021F00008936648089B008815605B1A834284BF79
:10220000634B1D6015B0BDE8F08FDFF8A881614E0B
:1022100008AF0025E9B2604809F094FA58F8043B89
:10222000C3F5967300FB03F086FB00230135C0174E
:10223000C0EB63100C2D47F8040BEBD1574B384D16
:102240000195384DB3F800C00395109D09980F997A
:10225000404EDFF8C0A0DFF8B490DFF8BC806545E1
:1022600011AA8CCAAE46ACBF4FF0000E4FF0010E63
:102270008445D4BF0020012030708C4528480B9D38
:102280001F4E8AF800E0D4BF00210121017094455F
:102290002449DFF814A1D4BF002201220A709C4512
:1022A0003F4AD4BF00230123BC45AB46D4BF00271F
:1022B00001271370AC45164B0C9D1F70D4BF4FF017
:1022C000000B4FF0010B374B0F4A0292AC45DFF881
:1022D00034C0124A83F800B0D4BF0025012589F824
:1022E000005098F800309CF8001096F80080DFF855
:1022F000BCC02678DFF8B8900092CEE6629EFF1F41
:10230000B49EFF1FB69EFF1F409DFF1FBB9EFF1F79
:10231000109DFF1F689FFF1FB59EFF1F069FFF1F99
:10232000199FFF1F1A9FFF1F629FFF1F639FFF1FC1
:10233000649FFF1F659FFF1F669FFF1F679FFF1F13
:10234000079FFF1F6A9FFF1FAC9CFF1F949CFF1FEE
:102350001A8AFF1F509FFF1FBC9EFF1FDA9EFF1FA0
:10236000709DFF1F149DFF1FF89EFF1FA69CFF1F5F
:10237000389FFF1FF4280100A0220100489FFF1F83
:10238000089DFF1F50A0FF1FF89CFF1F129FFF1FFB
:10239000549FFF1FB5814E1B609DFF1F2E9FFF1F87
:1023A0001B9FFF1F119DFF1F6D9EFF1F619FFF1F42
:1023B0002C9FFF1F2C89FF1FAF4AB04814880122B1
:1023C000182C027040F2058100248BE6012E00F0EB
:1023D0008F81022E00F0EE81032EA94B00F01F81A9
:1023E0001E78009B9CF800E01C78019B99F800C0C7
:1023F0001878029B93F80080039B1F78A6EB4E038E
:10240000A4EB8404CCEB030CC0EB80760CEB040350
:10241000C0EB8600034403EB480303EB810327B1C1
:1024200098490978002940F0608201269AF8001046
:102430009548C1F1060101EB4101334403EB8101F1
:102440000160A2E69149924B0968D0E6002D3FF465
:1024500044AE894A894E14880122182C327040F209
:10246000B8807446A0F10D0543E6DFF87092894FFD
:102470000DF120080025E9B2874809F063F959F801
:10248000043BC3F5967300FB03F087FB0023013583
:10249000C017C0EB6310062D48F8040BEBD17F4B3F
:1024A000DFF83CA219880D9B00228B428AF800209D
:1024B00080F2A2807A4B8AF800507A497A4A7B48A7
:1024C00091F8008011787A4A1D7002920378794A57
:1024D000DFF810C2DFF810920092774A774E784DFD
:1024E000784892F800E0784A0192784A96F800B06D
:1024F0002D78077826780392CFE5DFF8F081654ED6
:1025000008AF0025E9B2724809F01CF958F8043BFD
:10251000C3F5967300FB03F086FB00230135C0175B
:10252000C0EB63100C2D47F8040BEBD15B4B0C9DFB
:102530001F885F4B02935F4B00930B9B0A98099A8D
:10254000DFF8A0C1089EDFF8A0910F99BB429E461C
:10255000ACBF4FF0000E4FF0010EAF42D4BF0025CC
:1025600001258742109B8CF80050D4BF0020012029
:10257000504D89F800009742D4BF00220122B74293
:10258000D4BF4FF000084FF001082A709F42474A1D
:102590004448474E80F80080D4BF002301231370C5
:1025A000129A414886F800E08F42D4BF00210121F1
:1025B000974201701ADC00224648DFF824A102701D
:1025C0008BE7039C46B12678002E40F06081441EC4
:1025D000ABE50C3C012285E594F800E00138CEEB38
:1025E0000004BEF1000F7FF4A0AD9DE5119A974263
:1025F000D4BF00220122DFE70C9A374B9142CCBFB7
:10260000012200221A7040F3458105258AF8005006
:10261000234B52E7002E3FF487AD012685E51C7859
:10262000009B029893F80080019B9CF800601B7847
:1026300090F800C099F800700398A4EB4604E71BDB
:1026400090F800E0C3EB8374A8EB88003844C3EB38
:102650008403034403EB4C0303EB8103BEF1000F3F
:1026600040F0488101269AF80010074833440C24B2
:1026700014FB0131016088E5029FFF1FAC9CFF1F26
:102680001A8AFF1F1B9FFF1FBC9EFF1FF89CFF1F86
:1026900050A0FF1FB5814E1BC09CFF1F2E9FFF1F28
:1026A0007A9EFF1FB49EFF1FB69EFF1FB59EFF1FA1
:1026B000409DFF1F069FFF1F689FFF1F119DFF1F6B
:1026C000BB9EFF1F109DFF1F199FFF1F1A9FFF1F1B
:1026D000F49CFF1FDA9CFF1F339FFF1F4C8AFF1FD4
:1026E0006D9EFF1F619FFF1F2C9FFF1F1C8AFF1FF6
:1026F000A34CDFF89CE2207805909EF800400198FA
:102700000494059C007801900134A4EB40040498E3
:10271000002840F0AF80039890F800E00498261A53
:10272000CEEB06000390BEF1000F40F09E80744691
:102730000298944E00780290039836780496041B11
:10274000A4EB460402983C44CBEB0404002800F0C0
:102750008780B7FA87F040099CF800602044871B07
:102760001EB10498061C18BF0126009C99F80000B1
:102770002478BE1B301AA0EB440080440198C3EBC0
:102780000803A3EB4103002867D1BEF1000F40F01E
:10279000BB807344002C5ED100290CBF00206FF079
:1027A00009009AF80010784C03440C2010FB01310A
:1027B0002160EAE4039E019C36780396009E24780B
:1027C000019434786F4E714899F800E0009496F8BF
:1027D00000906F4C9DF80C6086709DF80460067048
:1027E00080F806E09DF8006080F803909CF800C037
:1027F0002478DFF8B491DDF804E080F808800771F0
:1028000080F805C0C671417244704FF00008012085
:10281000009500215D4C0D465FFA88FC4F467646D8
:1028200007E0022809D00A290BD014F8016F17F825
:10283000010F864201F10101F3D101350A29EDB200
:10284000F3D1092D72D808F10108B8F1100F36D074
:1028500019F80A0FDDE70020A3E74FF0000E98E714
:10286000029879E7CEEB040003900198041C18BF8E
:1028700001245DE7019800284ED0039890F800E00D
:10288000BEF1000FEED1601E0390744650E7841B2A
:1028900001264AE40B9A3F4B9142CCBF0122002211
:1028A0001A703EDC0A9A3C4B9142CCBF01220022B6
:1028B0001A7052DD03258AF80050384BFDE5304888
:1028C00037490478C86B0299009D09780134204487
:1028D000CBEB0000084400219AF800402A4B401A34
:1028E0000C2111FB040119604FE41BF1000618BF15
:1028F00001269BE52349097800293FF4B3AE1BF17B
:10290000000618BF0126AEE6049800280CBF4FF061
:10291000000E4FF0090E3CE7039890F800E03046B7
:10292000FDE604258AF800501C4BC6E514481C49F6
:10293000047851F828000299009D09780134204458
:10294000CBEB000066460844002BC4D0002EC2D159
:10295000BBF1000FBFD00121BEE7099A114B914294
:10296000CCBF012200221A7004DD02258AF8005033
:102970000A4BA2E5089B994218DD01259AE500BFA4
:102980001A8AFF1F1B9FFF1FBC9EFF1F349DFF1F46
:10299000509FFF1F329FFF1F319FFF1F7A9EFF1F17
:1029A000C889FF1F309FFF1FC4270100154B1D78EA
:1029B000012D25D9144A8AF800501288D2B1134A41
:1029C0001288013A92B2062A14D8114A12788AB1B2
:1029D000104A1268012A7FF470AD0F4A0F4E10683A
:1029E0000C2290FBF2F102FB110232800C4A03210F
:1029F000117062E5074A1268012A7FF45EADF5E7BF
:102A000035465AE57A9EFF1FE49EFF1F869EFF1FF4
:102A10006A9DFF1FFC9EFF1F549FFF1FC09EFF1F4C
:102A2000BC89FF1F2DE9F04F3A4B1B788BB0002B70
:102A30006BD10E200AF048FE0EF044F901463648EC
:102A4000364E374DFDF776FD3348FDF749FD0EF064
:102A500053FB80F30C003060FFF7F2FA2C68012C76
:102A60007AD0022C00F0AB82032C00F0BD832D4EF7
:102A70002D4C33682D4A2E4E0993099B31681288DC
:102A80002360591A013A9142274F00F29382294E4E
:102A900032689A1A0D2A00F27C82274E32689A1AFE
:102AA000132A00F27182254E32689A1A252A1AD901
:102AB000234B1B88002B40F05781224B1B78002BA7
:102AC00040F05281FEF7E0FB1F4B1B881B3B9BB283
:102AD000022B04D81D4B1B78002B40F0488104F0DA
:102AE0009DF8236833601A4D2A689B1A502B00F218
:102AF0000782184B1B88012B00F01F8206F028FF6D
:102B000006F056FD0BB0BDE8F08F08F045F80BB0AD
:102B1000BDE8F08FC49CFF1F949EFF1FD09EFF1F37
:102B2000FC9EFF1F50A0FF1F909EFF1FC489FF1F28
:102B3000649DFF1F4C9DFF1F209DFF1F249DFF1FB5
:102B4000769EFF1FBC9CFF1F029FFF1FAC9CFF1FB8
:102B5000709EFF1FD49EFF1FDFF814939D4AB9F8A3
:102B600000001378834204D0C3B21846137006F0F5
:102B70002BFEDFF8F882984AB8F8003011789942B5
:102B800004D0964F3978002940F0EC86944A336897
:102B90001288944E9A42C0F2F480934A1278002A26
:102BA00040F0EF80DFF8CCA2BAF8003023B98F4BA9
:102BB0001B88002B00F0FF848D4A8E4B11881B88E8
:102BC0008D4A0B4412685B1093428C4A126880F263
:102BD000A18400219342B4BF01230B4604910093CA
:102BE000ACBF4FF0010B8B4605910E200AF06CFD37
:102BF000834B844A1B68176803930133A7F2523250
:102C0000002B8446029240F3D486802BA8BF8023F9
:102C10007D4A7E4912780191002A00F0BC80097833
:102C2000914200F0B880B8F80010DFF840E2994215
:102C300001F0F1806949AEF80030754B4FF0010E9C
:102C400081F800E01978DFF830E2019B8EF800107F
:102C50001A70009B002B00F01181BAF80030002B95
:102C600000F00C816B4B1B685A1C002A40F3A586B0
:102C7000802A00F3A186684C68496948248809883D
:102C800000682144B0EB610FC1F23A83A3F148021E
:102C90000F2A02D8473BA9F800300E200AF014FD95
:102CA0006FF454731F44874202DC5E4B00221A709B
:102CB0005D4B1B88002B00F025845C4B5C4A1B7825
:102CC0001178994243D0002B41D05A490C78002CFE
:102CD00000F03787584991F800C0BCF1000F40F070
:102CE0002E87564F0097564F56480297534F0078FD
:102CF00087F800C0524F4FF0010E87F800C081F8EE
:102D000000E0002841F0DE804F490978002900F0FA
:102D1000FA874E4903910C460978002940F0F08764
:102D20004B48474F0078397001210297217070B1EC
:102D30004248414900904748032707700020087027
:102D40000099029F0870039901243C700870137069
:102D5000414B1B88A3F11B02012A40F2C7851D2BA2
:102D600000F011863D4C84E6FEF730FAAAE63C4BB3
:102D70001B78002B3FF4B3AE2B68012B7FF4AFAE72
:102D8000AFE63168374A069106983749106002224B
:102D90000B602A6006E71E49DFF8DCE009780029AD
:102DA0003FF453AF9EF8000081423FF44EAF0398CA
:102DB0004B2840F3F7871833802BB8F80000A8BFE2
:102DC000802398423FF441AF284803800348012301
:102DD00003703AE7639EFF1F289DFF1FAD9CFF1FF6
:102DE000689DFF1F50A0FF1FBC9CFF1F529DFF1F2F
:102DF000D49CFF1FCC9EFF1FF09CFF1FB49CFF1FA5
:102E0000489FFF1F9C9CFF1F3E9FFF1F049DFF1FAD
:102E10003F9FFF1FBC9EFF1F7C9EFF1F789EFF1FD2
:102E2000E49CFF1FCC9CFF1F869EFF1FDA9CFF1FA8
:102E30008C9CFF1F659FFF1FC49EFF1F189FFF1FD5
:102E40006A9DFF1F669FFF1F629FFF1F8D9CFF1FD4
:102E5000AC9CFF1FBC89FF1F029FFF1F909EFF1F9E
:102E6000079FFF1F189DFF1F8C9EFF1F049FFF1FC2
:102E7000849EFF1F0C9DFF1F059DFF1F029B9C450D
:102E8000BFF60BAF8B4B1B88002B3FF406AFBBF19B
:102E9000000F7FF4E7AE884B1B881BB1059B002B0E
:102EA0007FF4E0AE049B002B3FF4F7AE834B1A781F
:102EB000002A7FF4F2AEDFF8809299F800400122F8
:102EC0001A70002C40F044837D4B1B78002B02F0DD
:102ED000D8807C4B1B78002B02F09B837A4B1B78AD
:102EE000002B7FF4DAAE794B1B78002B3FF4D5AE84
:102EF000B8F8003076490A3BA8F800300A70CCE6F2
:102F000005F056FA734B1B7873B9734B1B785BB99A
:102F1000724B1B7843B9724B1B782BB9714B1B78E2
:102F200013B903F051FE01E003F05AFE23682B6051
:102F30006D4B1B88012B7FF4E1AD6C4A6C4B116823
:102F40006C481A78A1F118032A2101FB03F10160F2
:102F5000002A00F0C182684C2368994200F36A831A
:102F600010DA66480278002A40F09287644A1068B6
:102F7000D0F17F0048BF0330801001301B1A994206
:102F800042F3D0862160A9E2FEF772FC2368336029
:102F900089E5FDF70BFDFEF7A3F95A4B1B88032BC0
:102FA00000F02B85584B1B88032B00F022852368EB
:102FB000336072E5FDF746FC3B68336067E5534AD2
:102FC00034681188A14204DB464B1B78002B00F0CB
:102FD00061834F4E4F48336807934F4B079A006801
:102FE0001B88121A9A4200F2AD80002B00F0AA80D2
:102FF0004A4B1A88002A3FF4B5AE494B49481B6832
:103000000088A342B8BF2346994241F37281464BE0
:103010001960DFF8288188F80020344FFDF712FC92
:1030200038687F2840F37D85404B7F3883FB003232
:10303000C317C3EB620303EB4303A0EB83007330BE
:103040003B4B01931B883860002B40F0D686234B06
:1030500000931B78002B00F0CA83364C2378002B9A
:1030600000F0C583DFF8D890DFF8C0A04FF0000B68
:103070000CE003F17300C0B298F8001006F0FCFBFE
:1030800023780BF1010B5B4540F3B1833B6859F8A2
:10309000040F1844A0F17F038AFB0321DA17C2EB67
:1030A000610202EB42027F28A3EB8203E1DCFDF721
:1030B000E9FAE0E7529DFF1F8A9EFF1FCC9CFF1F8D
:1030C000629FFF1F639FFF1F649FFF1F659FFF1F7E
:1030D000AD9CFF1F6A9DFF1FC49EFF1F189FFF1F0F
:1030E0008D9CFF1FBC9CFF1FD49EFF1F549FFF1F82
:1030F000129DFF1F449DFF1F549DFF1F209FFF1F18
:103100001C9FFF1FD69EFF1F649EFF1F689DFF1F11
:1031100050A0FF1F189DFF1F509DFF1FAA9CFF1F5F
:103120008C9EFF1F349FFF1F909CFF1FABAAAA2AF3
:10313000EA9CFF1F8489FF1F6D9EFF1F419DFF1F9B
:103140005C89FF1F554B564A1B681088554AA3429D
:10315000B8BF2346994200F38482534C12888342BD
:10316000A8BF03462360002A7FF453AF9942C8BF2B
:10317000134640F37D82401AB0F5804FAABF9B03EF
:10318000C3EB8333013093FBF0F0FDF741FBC0F359
:10319000C6100DF097FD454B044618880DF092FDC2
:1031A0004349074620460DF0E1FD014638460DF043
:1031B000DDFD21460DF0D2FC4FF07E5104460DF0AE
:1031C00073FF002841F079803A4920460DF08AFFCC
:1031D000002840F0718620460DF0B4FFC0B2DFF841
:1031E000F48088F8000018E7334B34681988A1424E
:1031F00074DD324B1B78002B70D1DFF8DC9099F82E
:1032000000007F2840F34086A3F155337F3803F157
:10321000004383FB0032C317C3EB620303EB43039A
:10322000A0EB83007330264B01931B88C0B289F852
:103230000000002B41F03380224B00931B78002BC1
:1032400000F0AC84204C2378002B00F0A7841F4FA3
:10325000DFF87C804FF0000A0AE003F17300C0B28F
:1032600006F032FB23780AF1010A534540F39684B5
:1032700057F8043F99F800001844A0F17F0388FB39
:103280000321DA17C2EB610202EB42027F28A3EBB3
:103290008203E2DCFDF7F6F9E1E700BF8C9EFF1F39
:1032A000349FFF1FAA9CFF1F909CFF1F409FFF1F82
:1032B000CDCCCC3D0000FE42689DFF1FBC9CFF1F93
:1032C000EA9CFF1F189FFF1F8489FF1F5C89FF1F57
:1032D000ABAAAA2A419DFF1FBA9EFF1FB84F3868AC
:1032E0007F2840F3CC81B74B7F3883FB0032C31774
:1032F000C3EB620303EB4303A0EB83007330DFF8FF
:10330000249399F800A0824500F01782AE4B1B88E9
:10331000002B43D1AD4AAE4812680088914205DCCB
:103320008242D4BFC1EB0203C1EB0003411AB1F5E5
:10333000804FA6BF9B030131C3EB833393FBF1F0B6
:10334000FDF766FAC0F3C6100DF0BCFCA14B0446B5
:1033500018880DF0B7FCA049804620460DF006FD08
:10336000014640460DF002FD21460DF0F7FB4FF0FF
:103370007E5104460DF098FE002840F00A879749D8
:1033800020460DF0AFFE002840F0938520460DF05A
:10339000D9FEC0B2DFF8908288F80000BAF17F0F42
:1033A00040F3B8838748AAF17F0A80FB0A304FEACE
:1033B000EA73C3EB600000EB4000AAEB80007330BF
:1033C000874B00931B78C0B289F80000002B40F0B7
:1033D0001883844B03931B78002B40F04985824B64
:1033E00002931B78002B40F07C87804B0193029B5B
:1033F0001B78FBB17E4B1B88012B00F0C185022B93
:1034000001F04D80032B01F08C81042B01F0978398
:10341000052B01F03884062B01F0FF85072B01F006
:10342000BB87082B02F0BA80092B02F0BF810A2B60
:1034300002F09283009B1B78002B00F07484019BA8
:103440006A4C1988002900F0FB8438687F2840F313
:1034500065835C4B7F3883FB0032C317C3EB620389
:1034600003EB4303A0EB830073303860002940F086
:10347000AA84009B1B78002B00F06B815D4C2378A5
:10348000002B00F06681DFF8A4A1DFF89C814FF0EB
:10349000000B0CE003F17300C0B298F8001006F0C6
:1034A000EBF923780BF1010B5B4540F352813B684C
:1034B0005AF8040F434A1844A0F17F0382FB03210A
:1034C000DA17C2EB610202EB42027F28A3EB820310
:1034D000E0DCFDF7D7F8DFE7474B1960474B1B6887
:1034E000A92202FB03F3002BBCBF03F57F533F333C
:1034F0009B13543B194481F30C0128200AF06AFC09
:10350000FFF7FCBA384C3E483549364A2370037001
:103510000B701CE493424FF0000B80F2B380012348
:10352000CDF800B0CDF814B00493FFF75EBB354B77
:103530001B78002B7FF4B1AB039B334A243B83F30E
:103540004703D9B25B20136006F06EF999F800408A
:10355000032C30D1DFF8D88098F80030002B42F0EF
:103560005E822A4F3B78002B42F04C82254C237818
:10357000002B42F03A82264B1B78002B42F0288227
:10358000244A1380244B1B78002B42F014820E4BEC
:103590007F221A8098F800306BB93B785BB92378AA
:1035A0004BB91E4A7F210720138006F03DF97F2189
:1035B0000B2006F039F91A4B1F68FFF76EBB00BFEE
:1035C000549FFF1FABAAAA2AAA9CFF1F909CFF1F13
:1035D000349FFF1F409FFF1FCDCCCC3D0000FE421B
:1035E000189FFF1F8D9CFF1F6A9DFF1FEA9CFF1FF6
:1035F000869EFF1F8489FF1F549DFF1FC089FF1FE8
:10360000C49EFF1F659FFF1FD09CFF1F649FFF1F6D
:10361000639FFF1F5A9DFF1F669FFF1FB89EFF1FDE
:103620009C9CFF1FBA9EFF1F419DFF1F5C89FF1FCF
:10363000629FFF1FB64A1078002840F05783B54AB2
:103640001268D2F17F0248BF033203EBA202531C7F
:10365000B14A23609942B8BF1160FFF63FAF1946E7
:103660003CE7AE4B12881960002A7FF4D2AC0B46BF
:103670009842D4BFC1EB0003C1EB03037BE5FDF728
:1036800001F83CE60123CDF810B0CDF800B0059369
:10369000FFF7ABBA01232B60A14EA24CFFF7E9B9AB
:1036A000029B1B78FBB1A04B1B88012B00F0EA8426
:1036B000022B00F07386032B01F0A980042B01F08C
:1036C0006382052B01F05683062B01F0AF84072B94
:1036D00001F0AF85082B01F01987092B02F02F802C
:1036E0000A2B02F0C381019B1B88002B00F074831E
:1036F000009B1B783BB9039B1B7823B9029B1B786B
:10370000002B01F00480894B1B78002B00F0FE8019
:1037100087490B78082B00F2F98086483A680068E0
:10372000854C0133DBB25F1E101A44F827000B7082
:10373000824B3468198889F800208C42784E7FF7D4
:1037400011AB32687E4B0892089A764C1A60FFF7EC
:1037500090B9039B1B78002BA2D03B68A3F10C000F
:103760007F2840F3828377488B3B80FB0320DA1766
:10377000C2EB600000EB4000A3EB800303F1730099
:10378000DFF8D481C0B298F8001006F075F8009BFD
:103790001B78002B84D0664C2378002B80D0DFF878
:1037A000BCA14FF0000B0CE003F17300C0B298F81D
:1037B000001006F061F823780BF1010B5B457FF7F1
:1037C0006FAF3B685AF8040F5E4A1844A0F18B03B0
:1037D00082FB0321DA17C2EB61020C3802EB4202D2
:1037E0007F28A3EB8203DFDCFCF74CFFDEE74F4BC7
:1037F0001B78002B40F0F6823B68534A1278002A6F
:1038000045D0A3F10C007F2840F33B834D4A8B3B0E
:1038100082FB0321DA17C2EB610202EB4202A3EB47
:10382000820303F17300C0B298F8001006F024F888
:10383000009B1B7853B33E4C23783BB3DFF81C91BD
:10384000DFF800A14FF0000B0BE003F17300C0B2F2
:1038500098F8001006F010F823780BF1010B5B4587
:1038600014DD3B6859F8040F1844A0F18B038AFB60
:103870000321DA17C2EB61020C3802EB42027F2807
:10388000A3EB8203E1DCFCF7FDFEE0E73B682F4A97
:103890001278FAB1244A1288012A00F07D84022AA3
:1038A00000F07B86032A01F02F80042A01F0938127
:1038B000052A01F0CC82062A01F0D083072A01F004
:1038C0001384082A01F0D386092A01F090870A2A76
:1038D00002F00A81019A1288002A00F095821C4A9F
:1038E000104C137003232B60FFF7C3B8DFF8708010
:1038F00098F80030002B40F01881164F3B78002BD1
:1039000040F01485074C3B70FFF7B3B83A680FE7F7
:10391000209FFF1F1C9FFF1F549DFF1F909CFF1F98
:1039200050A0FF1F909EFF1F869EFF1FC49EFF1F7B
:103930008489FF1FB09CFF1F6089FF1F689DFF1FC8
:10394000FC9FFF1FABAAAA2A8D9CFF1F6A9DFF1F29
:10395000BA9EFF1FA89CFF1F419DFF1F5C89FF1F90
:10396000AC9CFF1FDBB21846137005F03BFFB04B59
:10397000B0491A46B04B184600230B703B701370C9
:103980000370FFF703B9DFF8CC8298F80030002B02
:1039900040F0D781A94F3B78002BB3D0A84BA94C5E
:1039A0001988A22006F0C4F898F800303B70FFF7A1
:1039B00060B80123FFF72CB98024A349A34BA44A84
:1039C00009881B8812680B44B2EB630FBFF665A928
:1039D000A04B1B78002B40F02482B8F800309E4AA0
:1039E000A3423FF45AA99D4B148001221A70FFF79D
:1039F00054B9FCF7AFFEFFF7DABAFCF755FEFFF754
:103A0000D1BA974B01931B88002B42F085818A4BDA
:103A10000393944B0293944C23786BB3DFF85C824E
:103A2000DFF848A24FF0000B09E003F17300C0B2C9
:103A300005F04AFF23780BF1010B5B451CDD58F8BC
:103A4000043F99F800001844A0F17F038AFB03218A
:103A5000DA17C2EB610202EB42027F28A3EB82037A
:103A6000E3DCFCF70FFEE2E77E4B029305F02CFF50
:103A7000009B1B78002BCED1039B1B78002B3FF4BF
:103A8000B6AC99F80030A3F10C007F2840F3EA812E
:103A900076488B3B80FB0320DA17C2EB600000EB1B
:103AA0004000A3EB800303F17300C0B205F00CFFEC
:103AB000009B1B78002B00F0CA816B4C2378002BF5
:103AC00001F0C582DFF8B481DFF8A0A14FF0000B50
:103AD0000AE003F17300C0B205F0F6FE23780BF1A3
:103AE000010B5B457FF783AC58F8043F99F8000061
:103AF0001844A0F18B038AFB0321DA17C2EB6102A1
:103B00000C3802EB42027F28A3EB8203E1DCFCF7D6
:103B1000B9FDE0E75046FCF7B5FD51E4FCF7B2FD16
:103B2000A3E4FCF7AFFDFFF78BBA514A1278002AE5
:103B300040F0D581414F434C3B70FEF79ABF0020C7
:103B400008704C49087840B139490091097800293A
:103B500000F0B581009F002139704749097800299C
:103B60007FF4D7A8002C40F0CE80002840F0CB8016
:103B7000384C2F4F94F800E02F4C0394394C0294AA
:103B80002D4C2C492070374C0097087038702070ED
:103B9000BEF1000F7FF4CFA8FFF7D9B8264B1B78F2
:103BA000002B6DD099F80030A3F10C007F2840F372
:103BB000C8832E4A8B3B82FB0321DA17C2EB6102DA
:103BC00002EB4202A3EB820303F17300C0B205F0E3
:103BD0007BFE009B1B78002B52D0234C2378002BBC
:103BE0004ED0264FDFF884804FF0000A09E003F141
:103BF0007300C0B205F068FE23780AF1010A53454C
:103C00003EDD57F8043F99F800001844A0F18B03FB
:103C100088FB0321DA17C2EB61020C3802EB420287
:103C20007F28A3EB8203E2DCFCF72CFDE1E700BF79
:103C3000189FFF1FC49EFF1F8D9CFF1FA89CFF1F86
:103C40000A9FFF1F909EFF1F7C9EFF1F789EFF1FF5
:103C5000E49CFF1FAC9CFF1F049FFF1FAD9CFF1F38
:103C6000EA9CFF1F6A9DFF1F8489FF1FABAAAA2A37
:103C7000079FFF1F669FFF1F629FFF1F5C89FF1F3B
:103C8000A84B1B78FBB1A84B1B88012B00F0D086FA
:103C9000022B00F0CB87032B01F04281042B01F0B3
:103CA000CD81052B01F01784062B01F0D884072B5A
:103CB00001F0E785082B01F07087092B01F0D5870B
:103CC0000A2B01F0A287019B1B88002B00F0F082D9
:103CD000964B1B78002B40F0E682954B954A19884D
:103CE00034680020012310602B6026E50130C0B24B
:103CF000022886BF0021117010701946FFF7EEBB35
:103D00000398002101708C49097800293FF41FA80D
:103D1000844902910978002900F0AE8702980021B9
:103D20000170FFF714B8039B1B78002B7FF487AB5F
:103D3000029B1B78002B7FF482AB019B1988FFF755
:103D400084BB7E4A1278002A3FF4F4AE7C4F387868
:103D500002F0CEFF7B4B1B78002B00F0B784398834
:103D60007E2900F2B384784CDFF80C922368D9F8EE
:103D700000209B1A0F2B40F29680744B01311B8858
:103D800089B239802BB1052B03D0C9B2052005F0CB
:103D90004BFD6F4F226898F80030C9F800203B7047
:103DA000FEF767BE243B002BB8F8000040F3748494
:103DB00098423EF44AAF9BB26648A8F8003001230F
:103DC0000370FEF742BFDFF89081C0B298F8001090
:103DD00005F052FDFFF74DBB5F4B3878197805F0C1
:103DE0004BFD85E47F21402005F01EFD5B495C4AC8
:103DF0003B680B6000211170FFE4C0B298F800101E
:103E000005F03AFDFFF723B9D8B298F8001005F095
:103E100033FD3B6863E5534BDFF860E11978FEF74B
:103E200014BF4B2C40F34C821834802CB8F800306F
:103E30004D4AA8BF8024A3427FF4D5ADFEF72DBF25
:103E400099F8000005F040FD2188FFF7FEBA029BBB
:103E50001B78002B7FF4CEAA039B1B78002B7FF4EA
:103E6000EEAA6AE7FCF70EFC1FE6FCF70BFC87E402
:103E70003E4B01931B88002B7FF4F6AD294B029338
:103E8000FFE5FCF7FFFBCEE4FCF7FCFBFFF7CBB94B
:103E90000132D2B2022A40F25A820022027019463E
:103EA000FFF71CBB284C2A4F98F800303B70FEF7F8
:103EB000E0BD7F20FFF76EBA7F20FFF790B9194F62
:103EC0001A4902974FF0000C81F800C0009F029938
:103ED0004FF0010E87F800E081F800C03DE6244F66
:103EE000387802F005FF174B1B78002B00F0368264
:103EF00039887E2900F23282134CDFF87C902368E7
:103F0000D9F800209B1A0F2BCDD91A4B01311888F4
:103F100089B23980002800F03D82C9B2C0B205F0F4
:103F200083FC36E76A9DFF1F869EFF1FC49EFF1F0E
:103F3000689DFF1F909CFF1FAC9CFF1F079FFF1FEA
:103F40000A9FFF1F679FFF1F909EFF1F6E9DFF1F11
:103F5000A89CFF1FAD9CFF1F419DFF1FB09CFF1F32
:103F60008489FF1F3F9FFF1F049FFF1FEA9CFF1FC5
:103F7000E09CFF1F309DFF1F4C9FFF1F059DFF1FF3
:103F8000DFF89CA399F80000BAF80030DF4AE04C53
:103F9000C31A82FB031ED917C1EB6E0101EB41016D
:103FA000A3EB810303EB430354F8233018447F2829
:103FB00040F3A6847F3882FB0032C317C3EB620351
:103FC00003EB4303A0EB83007330DFF858B3C0B2B8
:103FD00005F07AFCBBF80030022B7FF62BAA99F88B
:103FE0000010BAF80030C94ACB1A82FB030ED8176A
:103FF000C0EB6E0000EB4000A3EB800303EB430338
:1040000004EB8303586808447F2840F318877F38FF
:1040100082FB0032C317C3EB620202EB4202A0EB49
:1040200082007330C0B205F04FFCBBF80030032BA8
:104030007FF600AA99F80010BAF80030B34ACB1AFC
:1040400082FB030ED817C0EB6E0000EB4000A3EB21
:10405000800303EB430304EB8304A06808447F2838
:1040600040F351817F3882FB0032C317C3EB6202F9
:1040700002EB4202A0EB82007330C0B205F024FCD8
:10408000FFF7D8B9DFF898A23868BAF800309F4A2D
:104090009F4CC31A82FB031ED917C1EB6E0101EBC3
:1040A0004101A3EB810303EB430354F8233018448D
:1040B0007F2840F3A0847F3882FB0032C317C3EB14
:1040C000620303EB4303A0EB83007330DFF85882F5
:1040D000DFF850B298F80010C0B205F0CDFBBBF885
:1040E0000030022B7FF6FFAA3968BAF80030874A01
:1040F000CB1A82FB030ED817C0EB6E0000EB40001A
:10410000A3EB800303EB430304EB830358680844E9
:104110007F2840F398867F3882FB0032C317C3EBB9
:10412000620202EB4202A0EB82007330C0B298F848
:10413000001005F0A1FBBBF80030032B7FF6D3AADB
:104140003968BAF80030714ACB1A82FB030ED817CF
:10415000C0EB6E0000EB4000A3EB800303EB4303D6
:1041600004EB8304A06808447F2840F3F4807F3880
:1041700082FB0032C317C3EB620202EB4202A0EBE8
:104180008200733098F80010C0B205F075FBFFF79D
:10419000AABA0120FFF7FEB8DFF884A15B49BAF89C
:1041A00000205B4C9A1A81FB020ED017C0EB6E0008
:1041B00000EB4000A2EB800202EB420254F8220026
:1041C00018447F2840F31B84A0F17F0381FB032167
:1041D000DA17C2EB610000EB4000A3EB8000733004
:1041E000DFF840B198F80010C0B205F045FBBBF80D
:1041F0000030022B50D93968BAF80030434ACB1A44
:1042000082FB030ED817C0EB6E0000EB4000A3EB5F
:10421000800303EB430304EB8303586808447F28BF
:1042200040F3E1867F3882FB0032C317C3EB6202A2
:1042300002EB4202A0EB82007330C0B298F800108B
:1042400005F01AFBBBF80030032B25D93868BAF803
:1042500000302E4AC31A82FB031ED917C1EB6E0130
:1042600001EB4101A3EB810303EB430304EB830464
:10427000A36818447F2867DD7F3882FB0032C317AC
:10428000C3EB620202EB4202A0EB82007330C0B2C9
:1042900098F8001005F0F0FA3B68FFF71BBB05F03B
:1042A00013FBFEF7C9BF0021402005F0BDFA14E55D
:1042B00099F8000005F008FB0AE50120FEF78FBF22
:1042C000243C002CB8F8003040F32486A3423EF48E
:1042D000E4ACA4B20F4BA8F8004001221A70FEF71C
:1042E000DCBC0D4B01931B88002B7FF4BFABFFF7A9
:1042F0007EB80A498342A8BF03460B60FEF789BE19
:104300001446FFF765BBFCF7BDF9B6E6ABAAAA2ACF
:10431000C8260100AD9CFF1FEA9CFF1F909CFF1F59
:10432000C09EFF1FC29CFF1F419DFF1FDD4BDE4C47
:1043300019886A2005F0FCFB98F800303B70FEF706
:1043400098BBFCF79FF941E4FCF79CF99FE70270EA
:104350001946FFF7C3B8FCF795F913E7D34B1B7861
:10436000002B3FF49FAD3B88CE4F002B3FF49AAD1E
:10437000CD4CDFF848932268D9F80010521A0F2A62
:104380007FF691ADCA4A013B108899B23980002866
:104390007FF4C3ADC8B205F0BBFAFAE4DFF820A39E
:1043A0003868BAF80030C34AC34CC31A82FB031EF4
:1043B000D917C1EB6E0101EB4101A3EB810303EBC4
:1043C000430354F8233018447F2840F328847F386F
:1043D00082FB0032C317C3EB620303EB4303A0EB82
:1043E00083007330DFF8DC82DFF8DCB298F800106D
:1043F000C0B205F041FABBF80030022B7FF673A97A
:104400003968BAF80030AB4ACB1A82FB030ED817D2
:10441000C0EB6E0000EB4000A3EB800303EB430313
:1044200004EB8303586808447F2840F326867F38CE
:1044300082FB0032C317C3EB620303EB4303A0EB21
:1044400083007330C0B298F8001005F015FABBF87D
:104450000030032B7FF647A93868BAF80030954A38
:10446000C31A82FB031ED917C1EB6E0101EB410198
:10447000A3EB810303EB430304EB8304A368184419
:104480007F287FF768AF7F3882FB0032C317C3EB0A
:10449000620303EB4303A0EB8300733072E6DFF8A3
:1044A00020A299F80000BAF80030824A824CC31A60
:1044B00082FB031ED917C1EB6E0101EB4101A3EB97
:1044C000810303EB430354F8233018447F2840F35F
:1044D0007F837F3882FB0032C317C3EB620303EB99
:1044E0004303A0EB83007330DFF8DCB1C0B205F00A
:1044F000EBF9BBF80030022B7EF69CAF99F8001068
:10450000BAF800306B4ACB1A82FB030ED817C0EB07
:104510006E0000EB4000A3EB800303EB430304EBCE
:104520008303586808447F2840F39F857F3882FBC7
:104530000032C317C3EB620303EB4303A0EB83001A
:104540007330C0B205F0C0F9BBF80030032B7EF623
:1045500071AF99F80010BAF80030564ACB1A82FBB6
:10456000030ED817C0EB6E0000EB4000A3EB8003F6
:1045700003EB430304EB8304A06808447F287FF720
:10458000C2AE7F3882FB0032C317C3EB620303EB7A
:104590004303A0EB830073306FE5DFF824A14549A6
:1045A000BAF80020444C9A1A81FB020ED017C0EBD7
:1045B0006E0000EB4000A2EB800202EB420254F8D6
:1045C000220018447F2840F32E83A0F17F0381FB53
:1045D0000321DA17C2EB610000EB4000A3EB80007F
:1045E0007330DFF8E4B098F80010C0B205F044F979
:1045F000BBF80030022B7FF64FAE3968BAF80030B6
:104600002C4ACB1A82FB030ED817C0EB6E0000EBCE
:104610004000A3EB800303EB430304EB83035868E0
:1046200008447F2840F325857F3882FB0032C3177A
:10463000C3EB620303EB4303A0EB83007330C0B210
:1046400098F8001005F018F9BBF80030032B7FF63E
:1046500023AE3868BAF80030164AC31A82FB031E2C
:10466000D917C1EB6E0101EB4101A3EB810303EB11
:10467000430304EB8304A36818447F287FF764AEE8
:104680007F3882FB0032C317C3EB620303EB4303A3
:10469000A0EB83007330FAE501283EF4D6AA01238B
:1046A000FFF78ABBE09CFF1F909EFF1F669FFF1FC6
:1046B000309DFF1FABAAAA2A9C2901004C9FFF1F17
:1046C000C09EFF1F419DFF1FC29CFF1FCE4B1B784A
:1046D000002B3FF4E7AB3B88CC48012B7FF6E2ABE5
:1046E000CB4CDFF83C932268D9F80010521A0F2AFD
:1046F0007FF6D9ABC74A013B128899B20180002AE4
:104700003FF447AB052A7FF440ABFFF742BB4FF4C1
:104710007A43013BFDD199F8000005F0D5F8FEF78A
:10472000F2BFDFF800A399F80000BAF80030BA4AE7
:10473000BA4CC31A82FB031ED917C1EB6E0101EB01
:104740004101A3EB810303EB430354F823301844E6
:104750007F2840F3E8817F3882FB0032C317C3EB28
:10476000620202EB4202A0EB82007330DFF8B8B2C3
:10477000C0B205F0A9F8BBF80030022B7EF65AAEA5
:1047800099F80000BAF80030A34AC31A82FB03214B
:10479000DA17C2EB610202EB4202A3EB820303EBE6
:1047A000430304EB83035B6818447F2840F32584AC
:1047B0007F380C2290FBF2F302FB13007330C0B27F
:1047C00005F082F8BBF80030032B7EF633AE99F883
:1047D0000000BAF80030904AC31A82FB0321DA17AE
:1047E000C2EB610202EB4202A3EB820303EB430341
:1047F00004EB8304A36818447F287FF784AD7F38D7
:104800000C2290FBF2F302FB1300733035E4DFF867
:1048100014A23868BAF800307F4A804CC31A82FB71
:10482000031ED917C1EB6E0101EB4101A3EB81031C
:1048300003EB430354F8233018447F2840F370817E
:104840007F3882FB0032C317C3EB620202EB4202E5
:10485000A0EB82007330DFF8D481DFF8CCB198F898
:104860000010C0B205F008F8BBF80030022B7EF64D
:104870003AAF3868BAF80030674AC31A82FB03219E
:10488000DA17C2EB610202EB4202A3EB820303EBF5
:10489000430304EB83035B6818447F2840F3B4832D
:1048A0007F380C2290FBF2F302FB13007330C0B28E
:1048B00098F8001004F0E0FFBBF80030032B7EF600
:1048C00012AF3868BAF80030534AC31A82FB03218A
:1048D000DA17C2EB610202EB4202A3EB820303EBA5
:1048E000430304EB8304A36818447F287FF733ADA8
:1048F0007F380C2290FBF2F302FB1300733041E48B
:10490000FBF7C0FEFFF761BBDFF818A14249BAF818
:104910000020424C9A1A81FB020ED017C0EB6E00A9
:1049200000EB4000A2EB800202EB420254F82200AE
:1049300018447F2840F3FA80A0F17F0381FB032114
:10494000DA17C2EB610101EB4101A3EB8100733087
:10495000DFF8D4B098F80010C0B204F08DFFBBF8B7
:104960000030022B7FF698AC3868BAF800302A4A3B
:10497000C31A82FB0321DA17C2EB610202EB420287
:10498000A3EB820303EB430304EB83035B6818444C
:104990007F2840F33C837F380C2290FBF2F302FB2C
:1049A00013007330C0B298F8001004F065FFBBF834
:1049B0000030032B7FF670AC3868BAF80030164A26
:1049C000C31A82FB0321DA17C2EB610202EB420237
:1049D000A3EB820303EB430304EB8304A3681844B3
:1049E0007F287FF7B1AC7F380C2290FBF2F302FBFB
:1049F000130073304BE4FBF745FEFFF767BBFBF793
:104A000041FEFFF7EDBB00BF669FFF1F0A9FFF1F20
:104A1000909EFF1F6E9DFF1FABAAAA2A2C2A0100A1
:104A20004C9FFF1FC09EFF1FC29CFF1F419DFF1F89
:104A3000DFF838A399F80000BAF80030C34AC44C34
:104A4000C31A82FB0317D917C1EB670101EB4101C0
:104A5000A3EB810303EB430354F8233018447F286E
:104A60006ADD7F3882FB0032C317C3EB620202EBC0
:104A70004202A0EB82007330DFF8F4B2C0B204F05F
:104A800023FFBBF80030022B7FF61DA999F8000028
:104A9000BAF80030AD4AC31A82FB0321DA17C2EB21
:104AA000610202EB4202A3EB820303EB430304EB3C
:104AB00083035B6818447F2840F3AC827F380C2264
:104AC00090FBF2F302FB13007330C0B204F0FCFE63
:104AD000BBF80030032B7FF6F6A899F80000BAF86F
:104AE00000309A4AC31A82FB0321DA17C2EB610233
:104AF00002EB4202A3EB820303EB430304EB8304C8
:104B0000A36818447F2814DD7F380C2290FBF2F351
:104B100002FB13007330C0B204F0D6FEFFF7D3B827
:104B2000FBF7B0FD97E6FBF7ADFD1FE6FBF7AAFD2F
:104B30000EE7FBF7A7FDEEE7FBF7A4FD9CE7DFF828
:104B40002CA299F80000BAF80030804A814CC31AB0
:104B500082FB031ED917C1EB6E0101EB4101A3EBF0
:104B6000810303EB430354F8233018447F28DADD34
:104B70007F3882FB0032C317C3EB620303EB4303AE
:104B8000A0EB83007330F1E5DFF8E0A13868BAF8F4
:104B900000306E4A6F4CC31A82FB031ED917C1EB5B
:104BA0006E0101EB4101A3EB810303EB430354F8D6
:104BB000233018447F28B3DD7F3882FB0032C317CF
:104BC000C3EB620303EB4303A0EB8300733042E6C5
:104BD000FBF758FD88E4DFF894A15C49BAF800209F
:104BE0005C4C9A1A81FB020ED017C0EB6E0000EBF2
:104BF0004000A2EB800202EB420254F8220018446B
:104C00007F2893DDA0F17F0381FB0321DA17C2EB3C
:104C1000610000EB4000A3EB8000733098E6FBF7E7
:104C200031FDFFF7DFBBFBF72DFDDAE4DFF83CA138
:104C300099F80000BAF80030444A474CC31A82FB86
:104C40000317D917C1EB670101EB4101A3EB810306
:104C500003EB430354F8233018447F287FF76CAFED
:104C60007F3882FB0032C317C3EB620303EB4303BD
:104C7000A0EB83007330FFE638480090384839498C
:104C80000390FEF758B8DFF8E4A099F80000BAF8EE
:104C900000302E4A344CC31A82FB0321DA17C2EBD0
:104CA000610202EB4202A3EB820303EB430354F8DD
:104CB000233018447F2840F3A4817F380C2290FBD6
:104CC000F2F302FB13007330DFF8A4B0C0B204F0BB
:104CD000FBFDBBF80030022B19D999F80000BAF897
:104CE00000300C22C11A91FBF2F302FB131302FBFA
:104CF00003435B6818447F2840F384847F3890FB2B
:104D0000F2F302FB13007330C0B204F0DDFDBBF818
:104D10000030032B7EF68EABBAF8003099F8000015
:104D20000C22C11A91FBF2F302FB131302FB0344A2
:104D3000A36818447F287FF7E6AA7F3890FBF2F338
:104D400002FB13007330FFF798B900BFABAAAA2A81
:104D5000C8260100342301009C290100189FFF1F71
:104D60008D9CFF1FC49EFF1F64280100C09EFF1F73
:104D7000C29CFF1FDFF864A33868BAF80030CE4A3F
:104D8000CE4CC31A82FB0321DA17C2EB610202EB9D
:104D90004202A3EB820303EB430354F8233018448D
:104DA0007F2840F324817F380C2290FBF2F302FB32
:104DB00013007330DFF82883DFF828B398F8001069
:104DC000C0B204F059FDBBF80030022B1AD9386884
:104DD000BAF800300C22C11A91FBF2F302FB131354
:104DE00002FB03435B6818447F2840F3D4837F3879
:104DF00090FBF2F302FB13007330C0B298F800107E
:104E000004F03AFDBBF80030032B7EF66CACBAF828
:104E1000003038680C22C11A91FBF2F302FB131325
:104E200002FB0344A36818447F287FF794AA7F38C5
:104E300090FBF2F302FB13007330FFF7A3B9FBF70B
:104E400021FCFFF7EFB8FBF71DFCFFF76FB9DFF8A8
:104E50008CA29949BAF80020984C9A1A81FB02104A
:104E6000D117C1EB600101EB4101A2EB810202EB22
:104E7000420254F8220018447F2840F3BB80A0F17E
:104E80007F030C2093FBF0F200FB12307330DFF84D
:104E900054B298F80010C0B204F0EEFCBBF8003039
:104EA000022B1AD93868BAF800300C22C11A91FBCB
:104EB000F2F302FB131302FB03435B6818447F28E1
:104EC00040F39D837F3890FBF2F302FB13007330B5
:104ED000C0B298F8001004F0CFFCBBF80030032BF0
:104EE0007FF6DAA9BAF8003038680C22C11A91FBB3
:104EF000F2F302FB131302FB0344A36818447F2858
:104F00007FF722AA7F3890FBF2F302FB1300733085
:104F1000FFF7BDB9012B3DF4C0AE0124FFF7DAB9AC
:104F2000DFF8B8A199F80000BAF80030624A644C82
:104F3000C31A82FB0321DA17C2EB610202EB4202C1
:104F4000A3EB820303EB430354F8233018447F2878
:104F500046DD7F380C2290FBF2F302FB1300733026
:104F6000DFF880B1C0B204F0AFFCBBF80030022B18
:104F700019D999F80000BAF800300C22C11A91FB37
:104F8000F2F302FB131302FB03435B6818447F2810
:104F900040F38F807F3890FBF2F302FB13007330F5
:104FA000C0B204F091FCBBF80030032B7EF68BAE50
:104FB000BAF8003099F800000C22C11A91FBF2F304
:104FC00002FB131302FB0344A36818447F287FF7F6
:104FD000B0AD7F3890FBF2F302FB130073309AE51B
:104FE000FBF750FBBCE7FBF74DFBFFF726B9FBF7E0
:104FF00049FBDFE6FBF746FB49E7FBF743FBFFF71F
:10500000DEBBFBF73FFB5FE6FBF73CFB4FE4FBF748
:1050100039FBC7E4FBF736FB57E5DFF8C0A099F88A
:105020000000BAF80030244A264C34E6DFF8ACA081
:105030003868BAF80030204A224CA2E6DFF89CA07B
:1050400099F80000BAF800301B4A1F4C70E7029B29
:105050001B78002B7EF4CEA9FEF7F1B9DFF87CA017
:105060001549BAF80020174CF7E6FBF70BFBFFF7E2
:1050700068BAFBF707FBFFF7E2BAFBF703FBFFF7A2
:10508000E1B9124B1B78002B00F0D682104B1B7835
:10509000002B7DF402AE0F4B1B78002B3DF4FDADD1
:1050A000B8F800300C490A33A8F800300A70FDF750
:1050B000F4BDFBF7E7FA73E7ABAAAA2A642801005C
:1050C0002C2A0100202B010034230100639FFF1FC5
:1050D000649FFF1F659FFF1FAD9CFF1FC09EFF1FAA
:1050E000419DFF1FC29CFF1FA44C2288002A00F094
:1050F0002383A349DFF89CB20988BBF80000033181
:10510000884227DD9F48A0490088B1F800E0DFF819
:105110007CC2181A0C2190FBF1F901FB19004FF029
:10512000900909FB0EFE01FB00E06FF00B0E5CF82E
:10513000000003440EFB02307F2840F3CE847F380A
:1051400090FBF1F301FB13007330C0B298F800102C
:1051500004F092FBBBF8002023881344022B23DDCC
:10516000884B894A38681B88B2F800C0DFF81CE217
:10517000C31A0C2193FBF1F201FB1232902303FBC3
:105180000CF301FB023373445B6818447F2840F33F
:10519000A7857F3890FBF1F301FB13007330C0B299
:1051A00098F8001004F068FBBBF800202388134433
:1051B000032B23DD734B744A38681B88B2F800C098
:1051C000DFF8C8E1C31A0C2193FBF1F201FB1232A4
:1051D000902303FB0CF301FB023373449B681844D8
:1051E0007F2840F30B857F3890FBF1F301FB130020
:1051F0007330C0B298F8001004F03EFBBBF80020FA
:1052000023881344042B7FF747A85D4B1B88012B91
:105210007FF442A83A68A2F10C007F287FF794A897
:105220008B3A0C2092FBF0F300FB13207330FFF756
:105230002EB8524C2388002B40F00D83DFF854B178
:105240005049514A0988D7F80080B2F800E04F4829
:10525000C1EB080C0C229CFBF2F102FB11C14FF0D8
:10526000900C0CFB0EFE02FB01E16FF00B0E4058A0
:1052700080440EFB03807F2840F36A84A0F17F0303
:1052800093FBF2F002FB10307330414BC0B219783F
:1052900004F0F2FABBF8002023881344022B23DD2C
:1052A000384A394B11883868B3F800C0DFF8DCE0C1
:1052B000411A0C2291FBF2F302FB1311902303FB22
:1052C0000CF302FB013373445B6818447F2840F3FE
:1052D000F1847F3890FBF2F302FB130073302C4B08
:1052E000C0B2197804F0C8FABBF800202388134430
:1052F000032B23DD234A244B11883868B3F800C000
:10530000DFF888E0411A0C2291FBF2F302FB131143
:10531000902303FB0CF302FB013373449B68184496
:105320007F2840F3CF847F3890FBF2F302FB130019
:105330007330174BC0B2197804F09EFABBF8002006
:1053400023881344042B7EF7CEA90D4B1B88012B19
:105350007EF4C9A93A68A2F10C007F2840F3568177
:105360008B3A0C2092FBF0F300FB13207330084BB8
:10537000C0B2197804F080FAFEF7B5B9489DFF1F56
:10538000DE9CFF1FC09EFF1F6E9EFF1FC4230100F7
:10539000419DFF1FC29CFF1FCF4C2388002B40F074
:1053A0006582DFF868B3CD49CD4A098899F80000D5
:1053B000B2F800E0DFF85883C1EB000C0C229CFB34
:1053C000F2F102FB11C14FF0900C0CFB0EFE02FB40
:1053D00001E16FF00B0E58F8011008440EFB0300BA
:1053E0007F2840F37E83A0F17F0393FBF2F002FB62
:1053F00010307330C0B204F067FABBF80020238885
:105400001344022B22DDB54AB54B118899F80000F0
:10541000B3F800C0DFF8F8E2411A0C2291FBF2F376
:1054200002FB1311902303FB0CF302FB01337344C3
:105430005B6818447F2840F341847F3890FBF2F387
:1054400002FB13007330C0B204F03EFABBF8002038
:1054500023881344032B22DDA04AA14B118899F81D
:105460000000B3F800C0DFF8A8E2411A0C2291FB5B
:10547000F2F302FB1311902303FB0CF302FB013345
:1054800073449B6818447F2840F320847F3890FB46
:10549000F2F302FB13007330C0B204F015FABBF84C
:1054A000002023881344042B7DF7C4AF8D4B1B8849
:1054B000012B7DF4BFAF99F80020A2F10C007F28EA
:1054C0007EF721AF8B3A0C2092FBF0F300FB132008
:1054D0007330FEF7D2BDDFF804A299F80000BAF8E5
:1054E0000030814CC11A0C2291FBF2F302FB131322
:1054F00002FB03F3E35818447F287FF771AD7F3830
:1055000090FBF2F302FB1300733029E5774B1A8806
:10551000182A13D03B681344A3F118007F2840F3E6
:10552000C6830C20973B93FBF0F200FB123303F190
:1055300073006F4BC0B2197804F09EF96D4B6E4941
:105540001A78022A94BF013200221A701A7831F8B0
:105550001200182810D10424022A02F10100C2B25C
:1055600088BF002231F81200182804D1013CF3D181
:105570001A70FEF7B8B81A703B680344A3F118001C
:105580007F2843DD0C20973B93FBF0F200FB1233A6
:1055900003F17300EBE6FBF775F82EE4534B1B8821
:1055A000182B12D099F800201344A3F118007F287B
:1055B00040F393830C20973B93FBF0F200FB1233F4
:1055C00003F17300C0B204F07FF94A4A4A4B1278E3
:1055D00033F81230182B3DF42DAF99F80020134406
:1055E000A3F118007F287EF78EAE0C20973B93FB2B
:1055F000F0F200FB123303F17300FEF73EBDFBF740
:1056000041F865E4FBF73EF8FFF77EBBFBF73AF89D
:10561000ADE63A4B1B78002B7DF43FAB384B1B7843
:10562000002B3DF43AABB8F800303649013BA8F8FE
:1056300000300A70FDF731BB304B1B78002B7DF436
:1056400076AF2F4B1B78002B3DF427ABB8F800301A
:105650002C490133A8F800300A70FDF71EBBDFF8B3
:105660007CA099F80000BAF80030274C3AE71F4AAE
:105670001288182A12D01344A3F118007F2840F38F
:10568000C1820C20973B93FBF0F200FB123303F135
:105690007300C0B298F8001004F0EEF8154B1649EC
:1056A0001A78022A94BF013200221A701A7831F84F
:1056B000120018282FD10424022A02F10100C2B2DC
:1056C00088BF002231F81200182823D1013CF3D101
:1056D0001A703B68FEF7FEB8489DFF1FC09EFF1F73
:1056E0006E9EFF1FDE9CFF1F64280100169FFF1F98
:1056F000419DFF1FBC89FF1FDC9EFF1F649FFF1F92
:10570000659FFF1FAD9CFF1F202B0100C29CFF1F48
:10571000C42301001A703B680344A3F118007F28DA
:105720007EF712AE0C20973B93FBF0F200FB123396
:1057300003F17300FEF7ABBDDFF82CB3E2E4BE4B20
:105740001A88182A13D03B681344A3F118007F2845
:1057500040F37A820C20973B93FBF0F200FB12336C
:1057600003F17300B54BC0B2197804F085F8B44B5F
:10577000B4491A78022A94BF013200221A701A78AA
:1057800031F8120018287FF4F7AE0424022A02F13F
:10579000010294BFD2B2002231F8120018287FF41F
:1057A000EAAE013CF2D11A70FDF79DBFA24B1B88F7
:1057B000182B12D099F800201344A3F118007F2869
:1057C00040F372820C20973B93FBF0F200FB123304
:1057D00003F17300C0B204F077F8994A994B12783C
:1057E00033F81230182B7FF4F8AEFDF723BE924A3F
:1057F0001288182A12D01344A3F118007F2840F30E
:1058000069820C20973B93FBF0F200FB123303F10B
:105810007300C0B298F8001004F02EF8884B894944
:105820001A78022A94BF013200221A701A7831F8CD
:10583000120018287FF46FAF0424022A02F101023B
:1058400094BFD2B2002231F8120018287FF462AF60
:10585000013CF2D13CE77C4ADFF80CB21288BBF87D
:105860000010033291427FF715ADE9E4764ADFF884
:10587000F8B11288BBF80010033291427FF7BDAD3A
:1058800091E5724C2388002B40F0E481DFF8D8B119
:105890006F4999F800006F4A09881788DFF8B8E166
:1058A000411A0C2291FBF2FC02FB1C114FF0900CF0
:1058B0000CFB07F702FB01716FF00B075EF801109C
:1058C000014407FB03107F2840F3C1817F3890FB20
:1058D000F2F302FB13007330C0B203F0F5FFBBF824
:1058E000002023881344022B21DD594B594A99F893
:1058F00000001B88B2F800E0574FC31A0C2193FB3D
:10590000F1F201FB1232902303FB0EF301FB023391
:105910003B445B6818447F2840F3F8817F3890FB54
:10592000F1F301FB13007330C0B203F0CDFFBBF8FD
:10593000002023881344032B21DD454B454A99F869
:1059400000001B88B2F800E0434FC31A0C2193FB00
:10595000F1F201FB1232902303FB0EF301FB023341
:105960003B449B6818447F2840F3C1817F3890FBFB
:10597000F1F301FB13007330C0B203F0A5FFBBF8D5
:10598000002023881344042B7EF79DA92E4B1B88EF
:10599000012B7EF498A999F80020A2F10C007F2831
:1059A0007FF7C7A88B3A0C2092FBF0F300FB132083
:1059B0007330FFF7B0B8294B00227F2107201A80EF
:1059C00003F032FF7F210B2003F02EFFFDF7E2BD35
:1059D000234B01227F2107201A8003F025FF7F211E
:1059E0000B2003F021FFFDF7CDBD1E4B04227F21CC
:1059F00007201A8003F018FF00210B2003F014FF8A
:105A0000FDF7B9BD174B02227F2107201A8003F052
:105A10000BFF7F210B2003F007FFFDF7A7BD114B04
:105A2000002107201C8003F0FFFE7F210B2003F0E4
:105A3000FBFEFDF796BD00BFD69CFF1F419DFF1FDB
:105A4000BC89FF1F509EFF1FDE9CFF1F489DFF1F4C
:105A5000C09EFF1F6E9EFF1FC4230100AA9CFF1F54
:105A60005A9DFF1FB89EFF1FC29CFF1FAF4B1A8895
:105A7000182A13D03B681344A3F118007F2840F381
:105A80003F810C20973B93FBF0F200FB123303F1B4
:105A90007300A74BC0B2197803F0EEFEA54BA649E0
:105AA0001A78022A94BF013200221A701A7831F84B
:105AB000120018287FF460AD0424022A02F10102CA
:105AC00094BFD2B2002231F8120018287FF453ADEF
:105AD000013CF2D11A70FDF706BEFAF7D3FDFFF7CD
:105AE00034BBFAF7CFFD85E4904A1288182A12D009
:105AF0001344A3F118007F2840F3F6800C20973B55
:105B000093FBF0F200FB123303F17300C0B298F87C
:105B1000001003F0B1FE874B87491A78022A94BF20
:105B2000013200221A701A7831F8120018287FF416
:105B3000F2AD0424022A02F1010294BFD2B2002283
:105B400031F8120018287FF4E5AD013CF2D1BFE531
:105B5000FAF798FDFFF799BB744B1B88182B12D0EE
:105B600099F800201344A3F118007F2840F3C58062
:105B70000C20973B93FBF0F200FB123303F1730010
:105B8000C0B203F0A1FE6B4A6B4B127833F81230AF
:105B9000182B7FF422ADFDF74DBC684B1B88182BEA
:105BA00012D099F800201344A3F118007F2840F385
:105BB000B0800C20973B93FBF0F200FB123303F113
:105BC0007300C0B203F080FE5A4A5D4B127833F87E
:105BD0001230182B3EF477A899F800201344A3F153
:105BE00018007F287EF7A5AF0C20973B93FBF0F2BF
:105BF00000FB123303F17300FEF78DBFFAF742FD8D
:105C0000FFF7F7BAFAF73EFD43E5484B1B88182B20
:105C100011D099F800201344A3F118007F2872DDF9
:105C20000C20973B93FBF0F200FB123303F173005F
:105C3000C0B203F049FE3F4A3F4B127833F81230AE
:105C4000182BC9D1FEF73FB8FAF71CFD8AE5FAF721
:105C500019FD41E63B4ADFF800B11288BBF800109D
:105C6000033291427FF73BAE12E6374B1B88182B6D
:105C700011D099F800201344A3F118007F2839DDD2
:105C80000C20973B93FBF0F200FB123303F17300FF
:105C9000C0B203F019FE274A2C4B127833F81230A9
:105CA000182B99D1FEF70FB8FAF7ECFC92E5FAF74A
:105CB000E9FC3EE4FAF7E6FCFFF711BBFAF7E2FC79
:105CC000FFF7C1BBFAF7DEFCFFF733BBFAF7DAFCEC
:105CD000FFF7E2BBFAF7D6FC9BE5FAF7D3FC71E4D9
:105CE000FAF7D0FCFFF75BBAFAF7CCFC0EE7FAF74D
:105CF000C9FC41E6FAF7C6FCCAE7FAF7C3FC3FE77E
:105D0000FAF7C0FCC5E6FAF7BDFC91E7FAF7BAFC72
:105D10000AE6FAF7B7FC54E70D4B03930D4B0293D9
:105D2000FDF7A4BE23601946FDF7D8BBD89CFF1F22
:105D3000419DFF1FBC89FF1F589EFF1F169FFF1F1D
:105D4000DC9EFF1FDE9CFF1FD69CFF1F509EFF1F87
:105D50008D9CFF1F6A9DFF1FC29CFF1F38B507F077
:105D60004FFD0E4805F086FC0D4805F083FC0D48FC
:105D700005F080FC00234FF07E5201210A48FAF71B
:105D800075FB0A4B0A4A0B49802400251C711846F2
:105D90001D60BDE838400BF0F5B900BFC09CFF1F87
:105DA000F49CFF1F609DFF1F949EFF1F249FFF1FF9
:105DB0001C89FF1F2906000010B50446A420636853
:105DC000198803F0B5FEE368A6201988BDE81040E5
:105DD00003F0AEBE43682A20198803F0A9BE00BFB5
:105DE00010B5044622206368198803F0A1FEE36819
:105DF00024201988BDE8104003F09ABE10B504466F
:105E00000A206368198803F093FEE3680C20198860
:105E1000BDE8104003F08CBE10B504460620636850
:105E2000198803F085FEE36808201988BDE8104052
:105E300003F07EBE10B5044602206368198803F0A3
:105E400077FEE36804201988BDE8104003F070BEB7
:105E500070B50E4C84B0122504220123064603902F
:105E6000029320468DE824001423102106F006FE3C
:105E700006220923029303960195204600921423DB
:105E8000102106F0FBFD04B070BD00BF949FFF1F02
:105E9000F8B5B04CB4F90030032B00F01281002BA0
:105EA0006AD0022B00F08A80052B00F0B580012B10
:105EB00000F0DD80042B00D0F8BDA74FA74E0025D1
:105EC0004FF4AF74E9B2A64805F03CFC57F8043B28
:105ED000C3F5967300FB03F086FB0023C017C0EBED
:105EE0006310844205F10105A8BF0446062DE9D1DF
:105EF0009C4F9A4E0025E9B29B4805F023FC57F8C9
:105F0000043BC3F5967300FB03F086FB0023C01728
:105F1000C0EB6310844205F10105A8BF04460C2DB7
:105F2000E9D1924F8D4E0025E9B2914805F00AFC67
:105F300057F8043B894AC3F5967300FB03F086FBD0
:105F40000013C017C0EB6310844205F10105A8BF20
:105F500004460C2DE8D1A4F11401312900F3A380EB
:105F600040F26C7232218348834B01801A602A20F0
:105F7000BDE8F84003F0DCBD0E2007F0A5FB40F6BD
:105F8000FF71C8308842A8BF084620EAE07000F5DB
:105F9000FA6283B28A42794D794EA8BF0A4602203E
:105FA000194633802A8003F0C3FD2988042003F0BA
:105FB000BFFDB4F90030022B7FF476AF012008F06A
:105FC000C7FA0546002008F0C3FAA842B8BF284621
:105FD00000F1C801B1F5FA7FC0F2B480B1F57A6F73
:105FE000A8BF4FF47A6101F54873B3F57A6FA8BF83
:105FF0004FF47A639BB289B2624A634D11800A20E2
:106000002B8003F095FD29880C2003F091FDB4F955
:106010000030052B7FF44BAF0F2008F099FAC0F544
:106020003F630433B3F5AF6FC0F28980B3F5FA6F05
:10603000A8BF4FF4FA6399B2544BC0F54360B0F572
:10604000AF6F198061DBB0F5FA6FA8BF4FF4FA604B
:1060500083B24F4DA4202B8003F06AFD2988A6202F
:1060600003F066FDB4F90030012B7FF423AF152057
:1060700007F02AFB00F59671B1F52F7F4DDB41F259
:106080005C23994263DC434A00F5617089B2B0F544
:106090002F7F1180B8BF4FF42F7344DB8342A8BF1A
:1060A00003469BB23FE040F23A73A4F5B97403FB98
:1060B00004F482FB0432E417A4EB621289B2323298
:1060C00051E7102008F044FAC830B0F5FA7F1FDB22
:1060D000B0F57A6F0146A8BF4FF47A6101F51673E7
:1060E000B3F57A6FA8BF4FF47A639BB289B22A4A9C
:1060F0002A4D118022202B8003F01AFD29882420AC
:1061000003F016FDB4F90030C9E64FF4AF63A0E721
:1061100040F24C434FF4FA71E9E740F214534FF464
:106120002F711C4A11801E4D06202B8003F000FDAC
:106130002988082003F0FCFCB4F90030BAE64FF4DB
:10614000AF6179E740F214534FF4FA7154E71946FE
:10615000E7E700BF729FFF1F4C8AFF1FB5814E1BF0
:10616000C09CFF1F1C8AFF1FF49CFF1F2C89FF1F70
:10617000609DFF1F2E9FFF1F088AFF1F349FFF1F78
:10618000689DFF1FCC9EFF1FD49CFF1F6C9DFF1FAF
:10619000EC9EFF1F0E9DFF1F7C9EFF1F789EFF1F22
:1061A000009FFF1F2DE9F041224D82B0012602B26F
:1061B00084B20092284601967823192106F0A4FBA8
:1061C00004F10C0212B28DE844002846A719782386
:1061D000192104F1020806F097FB3FB20FFA88F884
:1061E00019233A46284619460196CDF8008006F054
:1061F0008BFB78233A4628461946CDF80080019655
:1062000004F10A070B3406F07FFB3FB224B2782377
:106210003A46284619468DE8500006F075FB1923CA
:1062200000943A4601962846194606F06DFB02B0E6
:10623000BDE8F081949FFF1F30B583B000230C466A
:1062400005B2009326225B231C210C4806F0ACF813
:10625000294601232622094805F0B6FB002C24B26A
:1062600005DB214601232622044805F0ADFB044A44
:10627000044B15801C8003B030BD00BF949FFF1FEE
:10628000668AFF1F688AFF1F2DE9F041BB4C237807
:1062900082B01BB1BA4B4FF6FF721A80B94BB3F9FB
:1062A0000030CBB9B84AB64B1068B3F9002080F380
:1062B0000C005B2303FB00F000131C3082424BD028
:1062C0004FF0FF31FFF7B8FFB04806F0D1F80023D8
:1062D000237002B0BDE8F081012B1BD0022B5AD0F5
:1062E000032B3FD0042B00F09980052BEFD10F201A
:1062F00008F02EF9C0F53B600830B0F5AF6F48DB11
:10630000B0F5FA6FA8BF4FF4FA60A0F5AF625B2357
:106310009F4835E09F4B1B78002B75D0152007F068
:10632000D3F99D4B1860B0F52F7F32DB41F25C232F
:106330009842A8BF1846A0F52F735B22974802FB2E
:1063400003F380FB0320DB17C3EBA0201C308C4B36
:10635000B3F900308342B3D1914BB3F9003001332C
:10636000AED1B4E78F4B1B68B3F5FA7F11DBB3F501
:106370007A6FA8BF4FF47A638B48A3F5FA725B2358
:1063800003FB02F380FB0320DB17C3EB20201C3050
:10639000DDE71C20DBE7854B1B68B3F5FA7F3BDBB1
:1063A000B3F57A6FA8BF4FF47A63A3F5FA727E480B
:1063B0005B2303FB02F380FB0320DB17C3EB2020EE
:1063C0001C307B4B1B68B3F5FA7F23DBB3F57A6F88
:1063D000A8BF4FF47A63A3F5FA7273495B2303FBFA
:1063E00002F381FB0321DB17C3EB21211C31644B3A
:1063F000B3F9003083427FF465AF694BB3F90030E5
:106400008B427FF45FAF62E7112008F0A1F8624B86
:10641000186088E71C21EAE71C20D2E72522002526
:106420008DE8240076231C215848624E624FDFF825
:10643000A08106F069FA16E0B0F5AF7FA8BF4FF46F
:10644000AF70323802FB00F088FB0031C017C0EBA0
:1064500061111C3109B201231D4425224B4805F06E
:10646000B3FA0C2D14D0E9B2544805F06BF956F884
:10647000043BC3F5967300FB03F087FB0013C017C2
:10648000C0EB631031284FF05B02D5DC1C21E2E742
:10649000262200258DE8240076231C213B48484E07
:1064A000454FDFF82C8106F02FFA16E0B0F5AF7FEC
:1064B000A8BF4FF4AF70323802FB00F088FB003108
:1064C000C017C0EB61111C3109B201231D44262203
:1064D0002E4805F079FA0C2D14D0E9B2394805F0B0
:1064E00031F956F8043BC3F5967300FB03F087FBC4
:1064F0000013C017C0EB631031284FF05B02D5DCEE
:106500001C21E2E7272200258DE8240076231C21A8
:106510001E482D4E284FDFF8B88006F0F5F917E039
:10652000B0F5AF7FA8BF4FF4AF70323802FB00F078
:1065300088FB0031C017C0EB61111C3109B2012387
:106540001D442722114805F03FFA062D3FF4BCAE4A
:10655000E9B21E4805F0F6F856F8043BC3F5967309
:1065600000FB03F087FB0013C017C0EB631031285A
:106570004FF05B02D4DC1C21E1E700BF6C9FFF1FE2
:10658000668AFF1F729FFF1FD09EFF1F949FFF1FF1
:1065900037800B6D889EFF1F989CFF1FD305854198
:1065A000688AFF1FE49CFF1F011FB812F09CFF1FA9
:1065B000B49CFF1F1C8AFF1FB5814E1BF49CFF1F5C
:1065C0002C89FF1F609DFF1F4C8AFF1FC09CFF1F6F
:1065D0004B48371B2DE9F041044682B071482768CB
:1065E000E56805F039FE1120FFF7DCFD01261923CF
:1065F0004FF02808194624226A480196CDF80080F9
:1066000006F082F978231946242266480196CDF8CF
:10661000008006F079F93146624806F00BFD02224F
:106620001921604806F002FD38460BF089FB394617
:1066300002465C4806F094FE5A4806F0A7FE142273
:106640000021584806F0F2FC03225749554806F04D
:1066500087FE544806F09AFE23220021514806F096
:10666000E5FC032251494F4806F07AFE4D4806F0FA
:106670008DFE7DB12F20FFF795FD32220021494884
:1066800006F0D4FC03224A49464806F069FE454814
:1066900006F07CFE0123474A18461370FFF7D8FB2B
:1066A0002189638962685B1A5C2B128854DD521A57
:1066B00002EB4202C2EB4212013392FBF3F31B33B3
:1066C0003D4A3848138001261A221BB28DE8440047
:1066D0001946142206F018F9002D4FD0218A638A3A
:1066E000E2685B1A5C2B12883EDC511A5C2202FBCA
:1066F00001F292FBF3F31B33304A2A481380012541
:106700001BB2382219468DE82400322206F0FCF82C
:106710004023002209218DE806002248194606F090
:10672000C1F829461F4806F085FC022244211D4875
:1067300006F07CFC63681B48198806F077FE2A4641
:106740001F49184806F00CFEE3681648198802B085
:10675000BDE8F04106F06ABE511A5C2202FB01F26C
:1067600092FBF3F31B33ABE7521A02EB4202C2EB8C
:106770004212334492FBF3F31B33BDE7402309215C
:106780002A46009107480195194606F08BF83146D4
:10679000044806F04FFC02226821024806F046FC3D
:1067A0006368D2E7949FFF1F882C01008C2C0100A6
:1067B000902C010011A0FF1F6E9FFF1F709FFF1FF5
:1067C000942C01002DE9F0471F4682B01446002AA0
:1067D0004ED0052A0646D0F80C8000F0AB800B9B0B
:1067E000894A00EBC305012CB5F80AE029896868DD
:1067F000C1EB0E0382FB03C21A444FEAE373C3EBFF
:10680000A213028851D0042C00F08D800022402376
:1068100009218DE806007D48194606F043F801215C
:106820007A4806F007FC0222B8F1000F00F0E18080
:106830004421764806F0FAFB73687448198806F01C
:10684000F5FD73497148012206F08AFDF3686F482F
:10685000198806F0EBFD6F4B022CB3F9001000F025
:10686000A680082C00F0C280012002B0BDE8F087AD
:10687000694E6A4A33681268CB1A93420D4655D95D
:10688000674A3B8811786148012918BF01241470B8
:106890000A9A06321BB212B28DE814001946BDF9ED
:1068A000282006F031F83560DEE79BB2D31A994212
:1068B00003DC9E457146A8BF19460A9A0180B7F9C4
:1068C0000030BDF928A0514802F106094FF0000E32
:1068D0000FFA89F919465246CDF80090CDF804E038
:1068E00006F012F829896A896868521A03885C2AB6
:1068F000A3EB010373DD03EB43030132C3EB43134B
:1069000093FBF2F303F11B0213B201203A80194604
:1069100052460190CDF800903C4805F0F5FF404B01
:1069200000221A7072E712FA83F3C0E7204602B021
:10693000BDE8F08707254FF000095A2323228DE890
:1069400020021A21314805F0ADFF01212F4806F041
:1069500071FB01212D4806F073FB232235212B48C2
:1069600006F064FB2A462F49284806F0F9FC274820
:1069700006F00CFD254805F07BFD4FF4FA6007F0AA
:10698000F5FBFFF785FA5A2323221A218DE820020E
:106990001E4805F087FF1D4805F06AFD3046FFF7E9
:1069A00019FE214B01221A70FFF76EFC2EE74A1CDC
:1069B00012B21A8091423FF457AF0A9AB7F90030E9
:1069C00012480632012412B2009219460194BDF910
:1069D000282005F099FF204602B0BDE8F0875C2131
:1069E00001FB03F393FBF2F21B328DE700221A80C6
:1069F000E0E76821054806F019FB73680348198829
:106A000006F014FD27E700BFC94216B2949FFF1F8E
:106A1000942C0100769FFF1FFC9FFF1F403C01004C
:106A200011A0FF1F982C01006C9FFF1F2DE9F04F54
:106A30005A4E5B4DB6F900704C7855F8277085B00A
:106A40008146984604B10C78DFF874A11AB99AF817
:106A50000030002B39D0534D002338462B808AF864
:106A60000030FFF7B7FD504A504BB5F90000012147
:106A700011704FF6FF721A8060B301285ED00120BA
:106A800032232246019000934946494B3846FFF78E
:106A900099FE00240346B5F90020022A39DD0022C0
:106AA0002A80B6F900203D49002A3BDB052AC4BFF5
:106AB00000220A80B8F1000F39D1002C0CBF184613
:106AC0004FF0FF3005B0BDE8F08F364DB5F900004E
:106AD0000028D2D1DFF8ECB0364ADBF8003012687B
:106AE000C3EB0903934227D9334B1A78012A18BF05
:106AF00001201870FFF7ACF90123CBF80090012CAE
:106B00002AD0042C35D0022C3AD0082C3ED00024B8
:106B1000C1E7C6D1FA68002AC1D0B6F900201F49E2
:106B2000002AC3DA05220A80B8F1000FC5D003930A
:106B3000FFF7AAFB039BC0E70346E0E74FF0000E18
:106B4000142322468DE8084049461C4B38467446BB
:106B5000FFF738FE03469EE732888AF8004001328C
:106B600032807A6982B10024384603939047039BB0
:106B700091E732880121013A32808AF80010F0E76B
:106B800001222A8000248CE7144684E77A690021D8
:106B900029804FF0FF34002AE6D182E7729FFF1F61
:106BA0006C8AFF1F769FFF1F6C9FFF1F668AFF1F67
:106BB000709FFF1F403C010011A0FF1F6E9FFF1F31
:106BC000749FFF1FFC9FFF1F01210D2007F092BA49
:106BD00000210D2007F08EBA01460D2007F08ABA79
:106BE00008B50D2007F08CFAB0FA80F149090D20A4
:106BF000BDE8084007F07EBA10B5002144080D201A
:106C000007F078FA204607F0B1FA0D20012107F0CD
:106C100071FA2046BDE8104007F0A8BA2D4A2E4B65
:106C200010881B68984210B549DA2C4A1288141A49
:106C30009A42A8BF1A46B4F5157F36DA121A40F206
:106C4000532303FB02F393FBF4F105310A2007F011
:106C5000C1F8234B1978C9B3224B23491B6840F272
:106C6000271283F3070302FB03F381FB032119447B
:106C7000DB17C3EBA1110531092007F0ABF81B4B63
:106C80001968F1B181F3070140F22712164802FB9F
:106C900001F380FB03211944DB17C3EBA11105317C
:106CA0001620BDE8104007F095B8131A4FF415727E
:106CB000611C02FB03F393FBF1F10531C6E70021F0
:106CC000C4E71620BDE8104007F084B8092007F09B
:106CD00081F8D4E7689DFF1F909CFF1F349FFF1F22
:106CE000129DFF1F1C9FFF1F09040281E89EFF1FCA
:106CF0007F2838B5A8BF7F200F4C4FF4167202FBD7
:106D000000F284FB02311144D2170546C2EBA111F7
:106D10000A2007F05FF87F3D4FF4967303FB05F3FD
:106D200084FB03211944DB17A3EBA1110920BDE863
:106D3000384007F04FB800BF09040281C368B3F9B7
:106D4000003030B583EAE374A4EBE374002BA0B207
:106D500018DB012300E0134603EB83025200944248
:106D6000F9DA0A4D90FBF3F285FB03E403FB120012
:106D7000DB173032D3EBA40380B201F8012BF1D141
:106D80000B7030BD2D230B700131E2E7676666663C
:106D900038B5094D8224204602F0E4FE35F8021B86
:106DA00000B28842204601D002F0C2FE0234A4B2F2
:106DB0008A2CF0D138BD00BF589EFF1F024B8020A7
:106DC000198802F0B5BE00BFD89CFF1F38B5094D29
:106DD0007824204602F0C6FE35F8021B00B2884235
:106DE000204601D002F0A4FE0234A4B2802CF0D1DF
:106DF00038BD00BF509EFF1F024B7620198802F05D
:106E000097BE00BFD69CFF1F38B5094D46242046CB
:106E100002F0A8FE35F8021B00B28842204601D0DD
:106E200002F086FE0234A4B24E2CF0D138BD00BF71
:106E3000DC9EFF1F024B4420198802F079BE00BF80
:106E4000169FFF1F024B4E20198802F071BE00BF33
:106E5000EA9CFF1F024B9A20198802F069BE00BF0E
:106E6000489DFF1F024B9820198802F061BE00BFA9
:106E7000DE9CFF1F024B8C20198802F059BE00BF18
:106E80006E9EFF1F024B9C20198802F051BE00BF6E
:106E9000C29CFF1F024BA020198802F049BE00BF10
:106EA000E49EFF1F024B9620198802F041BE00BFEE
:106EB000C09EFF1F024B8A20198802F039BE00BF16
:106EC000869EFF1F08B5034B1020198802F030FE84
:106ED000012008BD849EFF1F024B1020198802F07C
:106EE00027BE00BF849EFF1F024B2C20198802F092
:106EF0001FBE00BFBE9CFF1F024B1E20198802F060
:106F000017BE00BFDC9CFF1FC3680E20198802F06B
:106F10000FBE00BF024B2820198802F009BE00BF37
:106F2000DA9EFF1F024B6420198802F001BE00BFE9
:106F3000D49EFF1F024B5A20198802F0F9BD00BFF2
:106F4000A09CFF1F024B1620198802F0F1BD00BF64
:106F5000AA9CFF1F024B2E20198802F0E9BD00BF3A
:106F6000509DFF1F024B3020198802F0E1BD00BF89
:106F7000409FFF1F024B9E20198802F0D9BD00BF21
:106F8000C489FF1F024BAC20198802F0D1BD00BF9D
:106F9000D69EFF1F024BAE20198802F0C9BD00BF6C
:106FA000E89CFF1F024BB020198802F0C1BD00BF52
:106FB000649EFF1F024BB220198802F0B9BD00BFCA
:106FC000069DFF1F024B1820198802F0B1BD00BFBB
:106FD0006E9DFF1F024BA220198802F0A9BD00BFC1
:106FE0000A9FFF1F024B1A20198802F0A1BD00BFA3
:106FF000F69CFF1F024B1C20198802F099BD00BFB0
:10700000EC9CFF1F024B6620198802F091BD00BF67
:10701000149FFF1F024B7220198802F089BD00BF28
:107020003C9FFF1F024B2020198802F081BD00BF4A
:10703000129FFF1F024B3220198802F079BD00BF5A
:10704000029FFF1F024B6820198802F071BD00BF2C
:10705000309DFF1F024B6C20198802F069BD00BFF4
:10706000949CFF1F024B6E20198802F061BD00BF87
:107070006A9FFF1F024B5220198802F059BD00BFC2
:107080005E89FF1F024B5020198802F051BD00BFDE
:107090002089FF1F024B5420198802F049BD00BF10
:1070A000188AFF1F024B5C20198802F041BD00BF07
:1070B000648AFF1F024B5E20198802F039BD00BFB1
:1070C0005C89FF1F024B5620198802F031BD00BFBA
:1070D0003E9DFF1F244B1B880B2B43D8DFE803F09A
:1070E0000B10151A1F24292E33383D06084604229A
:1070F0001E490AF0E3BE084604221D490AF0DEBE1E
:10710000084604221B490AF0D9BE084604221A493F
:107110000AF0D4BE0846042218490AF0CFBE084639
:10712000042217490AF0CABE0846042215490AF08B
:10713000C5BE0846042214490AF0C0BE084604220F
:1071400012490AF0BBBE0846042211490AF0B6BE35
:10715000084604220F490AF0B1BE084604220E492F
:107160000AF0ACBE704700BFC09EFF1FF43801009C
:1071700048360100B4340100E4350100B8340100A0
:10718000003A0100BC340100C03401008C3701001A
:10719000C434010000390100C8340100064B074A1D
:1071A00010B41C88064B0846002C14BF1146194623
:1071B000042210BC0AF082BE0C9DFF1FCC340100DB
:1071C000D0340100064B074A10B41C88064B084611
:1071D000002C14BF11461946042210BC0AF06EBEE2
:1071E000529DFF1FCC340100D0340100064B074AEA
:1071F00010B41C88064B0846002C14BF11461946D3
:10720000042210BC0AF05ABE769EFF1FCC34010047
:10721000D0340100064B074A10B41C88064B0846C0
:10722000002C14BF11461946042210BC0AF046BEB9
:10723000C29EFF1FCC340100D0340100064B074A28
:1072400010B41C88064B0846002C14BF1146194682
:10725000042210BC0AF032BE5A9DFF1FCC3401003C
:10726000D03401001B4B1B880A2B0AD8DFE803F03F
:107270000A0E12161A1E22262A2E0600164B18680F
:1072800008607047154B186808607047144B186801
:1072900008607047134B186808607047124B1868F5
:1072A00008607047114B186808607047104B1868E9
:1072B000086070470F4B1868086070470E4B1868DD
:1072C000086070470D4B1868086070470C4B1868D1
:1072D00008607047869EFF1FF8340100D03401001B
:1072E000D4340100D8340100DC340100E034010062
:1072F000E4340100E8340100EC340100F034010012
:10730000F4340100F0B52B4E2B4FDFF8C4E00546F6
:107310000FCE87B06C460FC496E803003B68274A3F
:10732000274F44F8040B40F6CC308342C8BF3A469E
:10733000BEF800602180012E11889278ADF80D1002
:107340008DF80F202AD032D340F6CA02022E18BF81
:1073500000229A4226DAA3F698031A491A4AC3EB86
:10736000031381FB03011944DB17C3EB61232433AF
:1073700082FB0321DA17C2EBA10202EB8201A3EB2D
:107380004103303330328DF813308DF811206946C7
:10739000284616220AF092FD07B0F0BD40F698028A
:1073A0009A42D8DB094B1868CDF81100EFE740F698
:1073B000FC02CEE70C350100C89EFF1F003501001E
:1073C000FC3401003B773B98676666660435010034
:1073D000609EFF1FF8B5174C174E2278174D337873
:1073E0002F888E46003218BF012201467046FFF7F3
:1073F0001DFB002398423370237015DB14BF01205E
:1074000000202B889F420ED040F23A72A3F5AF7352
:107410000B490C4C02FB03F381FB0312DB17A3EBBC
:10742000621332332360F8BD0749012218460A70FF
:107430002270E6E7148BFF1F859FFF1F2E9FFF1F03
:10744000B5814E1B088AFF1F10A0FF1F014B187843
:1074500002F006BBF89FFF1F014B187802F01ABB21
:107460002891FF1F134BB3F9003030B583EAE37462
:10747000A4EBE374002BA0B218DB012300E0134659
:1074800003EB830252009442F9DA0B4D90FBF3F2C6
:1074900085FB03E403FB1200DB173032D3EBA403BC
:1074A00080B201F8012BF1D10B7030BD2D230B7090
:1074B0000131E2E72891FF1F67666666144BB3F956
:1074C000003070B583EAE375A5EBE375002BACB231
:1074D0001ADB012300E0034603EB830040008542F2
:1074E000F9DA0C4E94FBF3F086FB03E503FB104442
:1074F000DB173030D3EBA503A4B201F8010BF1D1B7
:1075000005480B70106070BD2D230B700131E0E752
:10751000A09CFF1F6766666624350100134BB3F914
:10752000003030B583EAE374A4EBE374002BA0B21F
:1075300018DB012300E0134603EB83025200944260
:10754000F9DA0B4D90FBF3F285FB03E403FB120029
:10755000DB173032D3EBA40380B201F8012BF1D159
:107560000B7030BD2D230B700131E2E7C489FF1F82
:1075700067666666134BB3F9003030B583EAE3748F
:10758000A4EBE374002BA0B218DB012300E0134648
:1075900003EB830252009442F9DA0B4D90FBF3F2B5
:1075A00085FB03E403FB1200DB173032D3EBA403AB
:1075B00080B201F8012BF1D10B7030BD2D230B707F
:1075C0000131E2E7E89CFF1F67666666134BB3F97B
:1075D000003030B583EAE374A4EBE374002BA0B26F
:1075E00018DB012300E0134603EB830252009442B0
:1075F000F9DA0B4D90FBF3F285FB03E403FB120079
:10760000DB173032D3EBA40380B201F8012BF1D1A8
:107610000B7030BD2D230B700131E2E7069DFF1F7B
:1076200067666666134BB3F9003030B583EAE374DE
:10763000A4EBE374002BA0B218DB012300E0134697
:1076400003EB830252009442F9DA0B4D90FBF3F204
:1076500085FB03E403FB1200DB173032D3EBA403FA
:1076600080B201F8012BF1D10B7030BD2D230B70CE
:107670000131E2E70A9FFF1F67666666134BB3F9A5
:10768000003030B583EAE374A4EBE374002BA0B2BE
:1076900018DB012300E0134603EB830252009442FF
:1076A000F9DA0B4D90FBF3F285FB03E403FB1200C8
:1076B000DB173032D3EBA40380B201F8012BF1D1F8
:1076C0000B7030BD2D230B700131E2E75E89FF1F87
:1076D00067666666134BB3F9003030B583EAE3742E
:1076E000A4EBE374002BA0B218DB012300E01346E7
:1076F00003EB830252009442F9DA0B4D90FBF3F254
:1077000085FB03E403FB1200DB173032D3EBA40349
:1077100080B201F8012BF1D10B7030BD2D230B701D
:107720000131E2E72089FF1F67666666134BB3F9F4
:10773000003030B583EAE374A4EBE374002BA0B20D
:1077400018DB012300E0134603EB8302520094424E
:10775000F9DA0B4D90FBF3F285FB03E403FB120017
:10776000DB173032D3EBA40380B201F8012BF1D147
:107770000B7030BD2D230B700131E2E7188AFF1F1B
:1077800067666666134BB3F9003030B583EAE3747D
:10779000A4EBE374002BA0B218DB012300E0134636
:1077A00003EB830252009442F9DA0B4D90FBF3F2A3
:1077B00085FB03E403FB1200DB173032D3EBA40399
:1077C00080B201F8012BF1D10B7030BD2D230B706D
:1077D0000131E2E7648AFF1F67666666134BB3F9FF
:1077E000003030B583EAE374A4EBE374002BA0B25D
:1077F00018DB012300E0134603EB8302520094429E
:10780000F9DA0B4D90FBF3F285FB03E403FB120066
:10781000DB173032D3EBA40380B201F8012BF1D196
:107820000B7030BD2D230B700131E2E75C89FF1F27
:107830006766666608B5702002F094F9044B1988F3
:10784000884204D07020BDE8084002F071B908BD3C
:10785000609EFF1F08B5742002F084F9044B19885C
:10786000884204D07420BDE8084002F061B908BD28
:10787000F89EFF1F054B1B880846042213B90449D4
:107880000AF01CBB03490AF019BB00BFEA9CFF1FAA
:107890002C350100283501000E4B1B88032B17D80F
:1078A000DFE803F0110C0702084604220A490AF037
:1078B00005BB0846042209490AF000BB0846042219
:1078C00007490AF0FBBA0846042206490AF0F6BA4C
:1078D000704700BF6E9EFF1F3C3501003835010028
:1078E000343501003035010010B40A4B0A4C0A4609
:1078F00093E8030083B0238802AC04E9030004EB9F
:107900008303104653F8081C052203B010BC0AF08C
:10791000D5BA00BF182D0100D49EFF1F30B40A4B0A
:107920000A4D0C4693E8070084B02B8804AD05E9A6
:10793000070005EB8303204653F80C1C042204B017
:1079400030BC0AF0BBBA00BF202D0100609EFF1FB3
:10795000F0B40C4D0C4F0E460FCD8CB001AC0FC4E3
:107960000FCD0FC495E807003B8884E807000CAAF8
:1079700002EB8303304653F82C1C04220CB0F0BCFD
:107980000AF09CBA2C2D0100B89EFF1F30B50A4B9F
:107990000A4D0C460FCB85B00DF1100E0EE90F000D
:1079A0002B880EEB8303204653F8101C042205B0ED
:1079B000BDE830400AF082BA682D0100D69EFF1F54
:1079C00030B50A4B0A4D0C460FCB85B00DF1100EA9
:1079D0000EE90F002B880EEB8303204653F8101C92
:1079E000042205B0BDE830400AF068BA682D0100F5
:1079F000649EFF1FF0B40B4D0B4F0E460FCD86B0AB
:107A00006C460FC495E803003B8884E8030006AA8F
:107A100002EB8303304653F8181C042206B0F0BC76
:107A20000AF04CBA782D01006E9DFF1FF0B40A4D8C
:107A30000A4F0E460FCD86B001AC0FC42A683B88B2
:107A4000226006AA02EB8303304653F8141C0C2272
:107A500006B0F0BC0AF032BA902D0100EC9CFF1F7A
:107A6000F0B40B4D0B4F0E460FCD86B06C460FC4D5
:107A700095E803003B8884E8030006AA02EB830331
:107A8000304653F8181C042206B0F0BC0AF016BAAF
:107A9000A42D0100F89EFF1F164B1B880BB31BB2D1
:107AA00083EAE370A0EBE370002B30B584B21DDBFA
:107AB000012300E0134603EB830252009042F9DAFF
:107AC0000D4894FBF3F280FB03E503FB1244DB1744
:107AD0003032D3EBA503A4B201F8012BF1D10B7026
:107AE00030BD0846042205490AF0E8B92D230B7081
:107AF0000131DDE7309DFF1F676666664035010096
:107B0000F0B40A4D0A4F0E460FCD86B001AC0FC43B
:107B10002A683B88226006AA02EB8303304653F8AA
:107B2000141C042206B0F0BC0AF0C8B9BC2D010038
:107B3000949CFF1F054B1B881BB9054B18680860F8
:107B400070470846042203490AF0B8B9489DFF1F50
:107B5000D0340100CC340100164B1B880BB31BB290
:107B600030B583EAE374A4EBE374002BA0B21CDB12
:107B7000012300E0134603EB830252009442F9DA3A
:107B80000D4D90FBF3F285FB03E403FB1200DB17C2
:107B90003032D3EBA40380B201F8012BF1D10B708A
:107BA00030BD064B1868086070472D230B700131FB
:107BB000DEE700BFDC9CFF1F67666666D03401000D
:107BC000164B1B880BB31BB230B583EAE374A4EBEE
:107BD000E374002BA0B21CDB012300E0134603EB8F
:107BE000830252009442F9DA0D4D90FBF3F285FBCB
:107BF00003E403FB1200DB173032D3EBA40380B2A3
:107C000001F8012BF1D10B7030BD064B18680860EC
:107C100070472D230B700131DEE700BFC69EFF1FAA
:107C200067666666D0340100164B1B880BB31BB227
:107C300030B583EAE374A4EBE374002BA0B21CDB41
:107C4000012300E0134603EB830252009442F9DA69
:107C50000D4D90FBF3F285FB03E403FB1200DB17F1
:107C60003032D3EBA40380B201F8012BF1D10B70B9
:107C700030BD064B1868086070472D230B7001312A
:107C8000DEE700BFAA9CFF1F6766666644350100F9
:107C9000174B1B881BB31BB270B583EAE375A5EBCA
:107CA000E375002BACB21EDB012300E0034603EBBF
:107CB000830040008542F9DA0E4E94FBF3F086FB18
:107CC00003E503FB1044DB173030D3EBA503A4B26C
:107CD00001F8010BF1D108480B70106070BD074B23
:107CE0001868086070472D230B700131DCE700BF76
:107CF000509DFF1F6766666648350100D03401005D
:107D0000164B1B880BB31BB230B583EAE374A4EBAC
:107D1000E374002BA0B21CDB012300E0134603EB4D
:107D2000830252009442F9DA0D4D90FBF3F285FB89
:107D300003E403FB1200DB173032D3EBA40380B261
:107D400001F8012BF1D10B7030BD064B18680860AB
:107D500070472D230B700131DEE700BF409FFF1FEE
:107D600067666666D0340100164B1B880BB31BB2E6
:107D700030B583EAE374A4EBE374002BA0B21CDB00
:107D8000012300E0134603EB830252009442F9DA28
:107D90000D4D90FBF3F285FB03E403FB1200DB17B0
:107DA0003032D3EBA40380B201F8012BF1D10B7078
:107DB00030BD064B1868086070472D230B700131E9
:107DC000DEE700BF149FFF1F67666666D0340100C0
:107DD000164B1B880BB31BB230B583EAE374A4EBDC
:107DE000E374002BA0B21CDB012300E0134603EB7D
:107DF000830252009442F9DA0D4D90FBF3F285FBB9
:107E000003E403FB1200DB173032D3EBA40380B290
:107E100001F8012BF1D10B7030BD064B18680860DA
:107E200070472D230B700131DEE700BF3C9FFF1F21
:107E300067666666D0340100174B1B881BB31BB204
:107E400070B583EAE375A5EBE375002BACB21EDBDE
:107E5000012300E0034603EB830040008542F9DA8A
:107E60000E4E94FBF3F086FB03E503FB1044DB1797
:107E70003030D3EBA503A4B201F8010BF1D10848CF
:107E80000B70106070BD074B1868086070472D2399
:107E90000B700131DCE700BF129FFF1F676666664B
:107EA00048350100D0340100054B1B881BB1054B40
:107EB000186808607047044B18680860704700BF76
:107EC0003E9DFF1F5C35010058350100184B1A8894
:107ED00052B3184A128830B50A80B3F90030002B2B
:107EE00083EAE374A4EBE374BCBF2D238B70A0B2D0
:107EF000ACBF02310331012300E0134603EB8302E0
:107F000052009442F9DA0C4D90FBF3F285FB03E446
:107F100003FB1200DB173032D3EBA40380B201F86D
:107F2000012BF1D10B7030BD044B1868086070470D
:107F3000F69CFF1F6035010067666666D03401005D
:107F400070B53C4D2B780646002B35D11C46737816
:107F50000BB9204670BDFAF773F8374A374B3848EB
:107F6000127831781B78007802EB43034A1E03EB4A
:107F700080030E2AEDD801A050F822F0E57F000022
:107F800007800000537F0000E57F0000537F000062
:107F9000537F0000537F0000D37F0000537F000019
:107FA000537F0000537F0000537F0000537F000089
:107FB000537F0000CF7F0000AE21224803F0FCFE7B
:107FC000204804F049F900232B700124BFE706F094
:107FD000DFFBAF211B4803F0EFFE1B4A01231370A8
:107FE0002B70B6E783B91948038804294FF6FF714F
:107FF00003F1FF320CBF01230B46134403F07F0350
:10800000013303800FE073B1013B114A32F81330A2
:108010004BB10E4E0F481049104A33800123002601
:1080200006700B701370084A0221012311702B7027
:10803000204670BD148BFF1F199FFF1F1A9FFF1F43
:108040001B9FFF1F949FFF1F10A0FF1F049FFF1F78
:10805000409EFF1F289DFF1FAD9CFF1F13A0FF1F09
:1080600010B5064B064C1A882046012101F04EFD42
:1080700021884220BDE8104001F05ABD0C9DFF1F31
:10808000369FFF1F10B5064B064C1A88204602216A
:1080900001F03CFD21884220BDE8104001F048BDC0
:1080A000529DFF1F369FFF1F10B5064B064C1A88C6
:1080B0002046042101F02AFD21884220BDE810401D
:1080C00001F036BD769EFF1F369FFF1F10B5064B91
:1080D000064C1A882046002101F018FD2188422014
:1080E000BDE8104001F024BDC29EFF1F369FFF1F58
:1080F00008B5122001F036FD054B1988884206D0DC
:10810000122001F015FDBDE8084001F029BC08BDB2
:10811000B89EFF1F08B5582001F024FD054B1988B3
:10812000884206D0582001F003FDBDE8084001F068
:1081300017BC08BDC69EFF1F08B5142001F012FD34
:10814000054B1988884206D0142001F0F1FCBDE8E7
:10815000084001F005BC08BD5A9DFF1FF0B480EA3D
:10816000E075A5EBE0750028ACB21FDB1DBF2B232B
:108170000B704E1C0E46012300E0134603EB8302F6
:1081800052009542F9DA0B4F94FBF3F287FB03059B
:1081900003FB1244DB173032D3EBA503A4B206F87D
:1081A000012BF1D133700846F0BC70472D230B70C2
:1081B0004E1CE0E767666666084B188828B10D28F4
:1081C00007D00D3800B2FFF7C9BF054A1068086034
:1081D0007047044A10680860704700BF6A9FFF1F1D
:1081E000D034010064350100174B18880C2813D0D7
:1081F000192815D01A2817D01B2819D01C281BD0D5
:108200001D281DD01E2803D00C3800B2FFF7A6BFD2
:108210000E4A1068086070470D4A10680860704781
:108220000C4A1068086070470B4A10680860704775
:108230000A4A106808607047094A10680860704769
:10824000084A106808607047029FFF1F80350100D0
:10825000683501006C35010070350100743501008E
:10826000783501007C350100034B1888A0EB8000B5
:10827000400000B2FFF772BFF89FFF1F024B188843
:10828000033800B2FFF76ABFDA9EFF1F024B18885F
:108290000C3800B2FFF762BFA69CFF1F024B188884
:1082A000183800B2FFF75ABFD89CFF1F024B18883E
:1082B000183800B2FFF752BFD69CFF1F024B188838
:1082C000183800B2FFF74ABF169FFF1FC36818880F
:1082D000183800B2FFF742BF054B1B881BB9054B8E
:1082E00018680860704708460422034909F0E6BD93
:1082F000E49EFF1FD0340100CC340100054B1B88E5
:108300001BB9054B186808607047084604220349EA
:1083100009F0D4BDDE9CFF1FD0340100CC34010035
:1083200030B5134C85B001252B463C220221204656
:10833000009503F0B7FD204603F08EFF0022402198
:10834000802320460191009311460A4B029504F0C8
:1083500031FC204604F08CF807480849084A0023FD
:10836000036083800B608B801360938005B030BD09
:10837000949FFF1F38300100789FFF1F8C9FFF1FC5
:1083800000A0FF1F10B500EBC00000F10F02D2B239
:1083900093B284B09C1E981C3D2303918DE8190074
:1083A0003921024804F06AFB04B010BD949FFF1FFE
:1083B000014B01221A707047859FFF1FF0B5704B6B
:1083C000704C714F714E724D85B004228DE80C00D7
:1083D000029320466F4B4022802103F06BFB204626
:1083E0006D4C6E4A6E4908F0CDFEA7616D486E4F28
:1083F000E7616E4F87616E496E4FC7616E4F8F6147
:108400006E4A6F4FCF616F4F97616F4B6F4FD76160
:108410006F4F9F616F4FDF616F4FB7616F4FF761B4
:108420006F4FAF616F4C704FEF61704FA761704835
:10843000704FE761704F87617049714FC761714F2D
:10844000714A8F61714FCF61714F724B9761724F5B
:10845000D761724F724E9F61724FDF61724F734DE1
:10846000B761734FF761734F734CAF61734FEF6137
:10847000734F7448A761744FE761744F7449876103
:10848000744FC761744F8F61744A754FCF61754FD8
:108490009761754B754FD761754F9F61754E764FDC
:1084A000DF61764FB761764D764FF761764FAF61FA
:1084B000764C774FEF61774FA7617748774FE76149
:1084C000774F87617749784FC761784F8F61784AD6
:1084D000784FCF61784F9761784B794FD761794F5B
:1084E0009F61794E794FDF61794F7A4DB7617A4F4D
:1084F000F7617A4F7A4CAF617A4FEF617A4F7B48E0
:10850000A7617B4FE7617B4F7B4987617B4FC761E9
:108510007B4F7C4A8F617C4FCF617C4F7C4B976156
:108520007C4FD7617C4F7D4E9F617D4FDF617D4FDA
:108530007D4DB7617D4FF7617D4F7E4CAF617E4FC2
:108540007E487F49EF617F4F7F4DA761E5617F4F97
:108550007F4D804CDFF820E27F4A804B8761C56108
:108560008C617F4E7F4F804D804CC1F81CE080486D
:1085700080499761D5619C61D861B16005B0F0BD5B
:1085800040420F00949FFF1F8D820000BC8DFF1F93
:108590002C8DFF1F7491FF1FE08DFF1F1C89FF1F93
:1085A0000DBB00007C8FFF1F096F00007D82000063
:1085B000C88EFF1F156F00009D710000C08CFF1F4B
:1085C00061800000C5710000A08FFF1F8580000042
:1085D000ED710000A9800000E9780000256F00001F
:1085E00015720000988DFF1FCD8000006982000089
:1085F000748DFF1F4D74000065740000588FFF1FBD
:10860000597400001D790000548CFF1F357800005C
:10861000517900000C90FF1FF1800000C17B000029
:10862000088DFF1F15810000BD740000148CFF1F12
:10863000356F00003D7200009C90FF1F39810000E3
:10864000297C0000E48CFF1F456F0000917C000036
:10865000048EFF1F556F0000017D00009C8CFF1FE2
:10866000656F00001D750000CC8BFF1F756F00004B
:108670008D7900005490FF1F856F00007575000014
:10868000108FFF1F956F0000C1790000848BFF1FC2
:10869000A56F0000CD7500003C8BFF1FB56F00007B
:1086A000F5790000CC8AFF1FC56F00002576000019
:1086B000508DFF1FD56F0000CD7E0000348FFF1F4F
:1086C000E56F00002D7A00003891FF1FF56F000064
:1086D000697D0000A48EFF1F05700000D17D0000A1
:1086E000608BFF1F15700000617A00003090FF1F43
:1086F00055780000397E0000EC8EFF1F25700000C9
:10870000E9810000A88BFF1F35700000997A0000F6
:10871000188BFF1F45700000017B0000848AFF1F3B
:1087200055700000B98100000491FF1F65700000C2
:108730007D760000788CFF1F75700000F08AFF1FA7
:10874000F08BFF1FD5760000857000002D770000AC
:108750009570000085770000C48FFF1FA88AFF1F57
:108760002C91FF1FDD770000B5700000A97E00008E
:10877000C5700000018D0000A5700000F0B5461C1A
:1087800083B00D460127032336B22AB20446314690
:108790008DE888002348ADB204F006F90C23AA1C2A
:1087A00012B200930197052321B21E4804F0FCF891
:1087B0001D4A1E4B12881B68BA422AD023D3022AB4
:1087C00010D11B4CA3F6CA0384FB03241C44DB1703
:1087D000C3EB24140A2CA8BF0A2424EAE474A2B22E
:1087E00023B202E000231A461C460D35AA1A0120C6
:1087F0000093019012B2314603230A4804F052F864
:10880000204603B0F0BD0B4CA3F6FC0384FB03240D
:10881000DDE7094CA3F6980384FB0324DB17C3EBC5
:10882000A404D7E7949FFF1F609EFF1FC89EFF1FF1
:10883000898888881F85EB51398EE3382DE9F0430C
:108840008FB283B0DFF84C80BD1D461D2DB204B23F
:1088500036B24FF001090AB2234631464046009530
:10886000CDF8049004F050F82A463346214640469D
:108870008DE8200204F048F807F10C020095334619
:1088800012B22146CDF80490404604F03DF803B002
:10889000BDE8F083949FFF1F2DE9F043804685B02B
:1088A000002956D10121304804F0C4FB2F4998F823
:1088B000062098F8083011F80290994522DA4FEA1C
:1088C00089064D460C24D8F80C3027489B595F6820
:1088D00022B2002104F0AAFB384609F031FA3946E9
:1088E0000246214804F03CFD1F4804F04FFD98F873
:1088F000083001350934AB42A4B206F1040601DDAB
:10890000422CE0D1B9F1000F13D109F106099945C4
:108910000CDA3C2301213B22039102930093019244
:1089200039233F223A21104804F0A8F805B0BDE8E9
:10893000F0830F2301213B220391029300930192C4
:1089400039230C223A21084804F098F898F80830A6
:10895000DBE700213423009301913F230C220248DE
:1089600003F0A0FF9EE700BF949FFF1F8C9FFF1F97
:1089700010B5104C0121204604F062FB2046012175
:1089800004F058FB20463422552104F04FFB2046CA
:108990000222094904F0E4FC20460522074904F0BC
:1089A000DFFC204604F0F2FC2046BDE8104003F056
:1089B0005FBD00BF949FFF1FCC350100D035010083
:1089C00070B50D46064609F0BBF900EB4000840087
:1089D000002D36D0284609F0B3F900EB40004000E6
:1089E00023185B1003F16001091A282209B2174805
:1089F000C3F1600404F01AFB0121144804F01AFBCF
:108A0000284609F09DF929460246104804F0A8FCC2
:108A10000E4804F0BBFC02210C4804F00BFB21B211
:108A200021220A4804F002FB304609F089F9314658
:108A30000246064804F094FC0448BDE8704004F087
:108A4000A5BC6410C4F16004E5E700BF949FFF1F5C
:108A5000184B70B5B3F9003083EAE374A4EBE37408
:108A6000002B82B0A1B21EDB68466D46012300E0F8
:108A7000134603EB830252009442F9DA0E4E91FB47
:108A8000F3F286FB03E403FB1211DB173032D3EB66
:108A9000A40389B205F8012BF1D119462B70FFF719
:108AA0008FFF02B070BD2D238DF800300DF1010550
:108AB0006846DBE7849EFF1F6766666610B50D4B50
:108AC0001B5C51F82340237884B013B1012004B01B
:108AD00010BD04AA01A942F8103D2046A369984799
:108AE000A38A9B07F2D401A80099FFF769FF012030
:108AF00004B010BD789FFF1F2DE9F04F2F4DDFF818
:108B0000CCB0DFF8C4A0DFF8C8900FCD91B003ACB3
:108B10000FC40FCD0FC40FCD0FC42B6823600025E9
:108B2000A8462F462E4600E09846BAF80030244961
:108B30005BF8232028461123F7F754FE00EBC0040E
:108B400000EB840089FB00340444C017C0EB64349C
:108B5000C4F13C00C6F13C0207F14101012600B21C
:108B600008F1410300901BB2019612B209B21548F8
:108B700003F0CAFE08EB060305F211153C2B26464E
:108B8000ADB24746D0D134226B210E4804F04EFAE4
:108B900000210C4804F04EFA0B4B1B8810AA02EB84
:108BA000830353F8344C204609F0CAF802460548BE
:108BB000214611B0BDE8F04F04F0D2BBD02D01002A
:108BC000A0270100949FFF1FBE9CFF1F04260100E9
:108BD0000900028010B5424C424882B003F03CFBD1
:108BE0002378C3B906213F4804F024FA2378012BE7
:108BF00037D90A22022B11463A486BD004F016FAF4
:108C000039490322374804F0ABFB364802B0BDE8CF
:108C1000104004F0BBBB354B1A7801210523002A14
:108C200035D10191009311462E4803F0BDFE304B23
:108C30001A78002A36D005230122019200930022DF
:108C40000A21284803F02EFE2A4B1A78002A35D133
:108C500001210523019100931421224803F0A4FE71
:108C6000C0E7254C2388092B32D9632B8CBF0A21FE
:108C70001F210A221B4804F0D9F92188194804F061
:108C8000D5FB184802B0BDE8104004F07FBB0022BD
:108C9000019100931146134803F004FE144B1A7817
:108CA000002AC8D105230121019100930A210D4812
:108CB00003F07AFE0F4B1A78002AC9D0012205234F
:108CC0000192009300221421064803F0EBFD89E78E
:108CD0003021CEE704F0AAF90322084992E700BF49
:108CE00013A0FF1F949FFF1FDC350100199FFF1F7A
:108CF0001A9FFF1F1B9FFF1F049FFF1FD8350100F6
:108D0000F8B56D4D287840B96C4B1B6899425CD31F
:108D10006B4A012313702B70F8BD0C46002669487E
:108D2000664F03F099FA04F6AC53324665483B604F
:108D300031212E7004F07AF901216248624D04F06D
:108D40007FF931465F4804F075F905225F495D48B7
:108D500004F006FB5B4804F019FB0C221021594873
:108D600004F064F90B225A49564804F0F9FA052236
:108D70005849544804F0F4FA524804F007FB564BA3
:108D800050481C68A4F69803C3EB031385FB032526
:108D90001D441021DB172022C3EB652504F046F9A2
:108DA00040F6CC339C4205F124054FF022014FF0F0
:108DB00004000BDCFFF7E2FC484B1C88064674B34A
:108DC000012C46D0022C41D00120F8BDFFF736FD22
:108DD000092243493B4804F0C3FA2A2210213948AA
:108DE00004F024F93F4C374884FB0534EB17C3EB00
:108DF000A404214604F01AFB01223B49314804F047
:108E0000AFFA04EB8401A5EB41012E4804F00EFB00
:108E1000012236492B4804F0A3FA0120F8BD344959
:108E20001022284804F09CFA264804F0AFFA2A22BF
:108E30001021244804F0FAF83146224804F0F6FAEA
:108E400007222C491F4804F08BFACBE70C222A4951
:108E5000E7E70C2229491B4804F082FA194804F07C
:108E600095FA2A221021174804F0E0F831461548F7
:108E70001C4E04F0DBFA07221E49124804F070FA77
:108E800086FB0536EB17C3EBA60631460D4804F00A
:108E9000CDFA224614490B4804F062FA06EB86012B
:108EA000A5EB4101074804F0C1FA22460F490548E5
:108EB00004F056FA2046F8BD148BFF1FF49FFF1FE5
:108EC00010A0FF1F949FFF1F3B773B98E0350100E8
:108ED000E8350100D0350100C89EFF1F609EFF1FCE
:108EE000F435010067666666DC3D01004C3D01001B
:108EF00000360100143601002C3601001C3601003A
:108F00002DE9F041754C2278002A05460F4614BF22
:108F10004FF001084FF000084ED1714E3368CB1A64
:108F2000B3F5FA6F04D86B78A3B94046BDE8F08179
:108F30006C4B6D486D49DFF8D0E11A700123037066
:108F40000988237026208EF8002000F0F1FD6B7850
:108F5000002BEAD03760F9F773F8654A654B66492C
:108F6000127828781B78097802EB4303421E03EB42
:108F700081030E2AD9D801A151F822F06D9000008A
:108F8000399000002B8F00006D9000002B8F0000A7
:108F90002B8F00002B8F0000219000002B8F0000F2
:108FA000D38F00002B8F00002B8F00002B8F000031
:108FB0002B8F0000CF8F0000AF215048484E02F0A9
:108FC000FBFEFFF707FE002337602370ABE705F0D9
:108FD000DFFB4A4803F040F90221484804F02AF830
:108FE0000F222321454804F021F805224449434833
:108FF00004F0B6F9414804F0C9F91E2223213F4884
:1090000004F014F805223F493C4804F0A9F93B4814
:1090100004F0BCF9394803F02BFA00F0ADFC84E70A
:10902000394D2B78012B50D9304B2620198800F070
:109030007FFD00232B7078E7002B3FF476AF013BD8
:10904000324A32F81330002B3FF46FAF274C3048D0
:1090500025492D4A23804FF001080023037081F831
:10906000008082F80080FFF7B5FD5EE793B1013B19
:10907000264A32F8131019B31C4B254D1A4C224ABC
:1090800019800026012326202E702370137000F013
:109090004FFD15E0154C1E4922880B7004284FF631
:1090A000FF7002F1FF310CBF012202460A440E4E4E
:1090B000154D02F07F0201320121228031702B70A8
:1090C000FFF788FD4FF001082FE70649064A012304
:1090D0000020087013702370A6E700BF148BFF1FD9
:1090E0000CA0FF1F10A0FF1FAD9CFF1F049FFF1FC0
:1090F000199FFF1F1A9FFF1F1B9FFF1F949FFF1F9A
:109100003C3601004436010013A0FF1F409EFF1FA4
:10911000289DFF1F2DE9F04F05468BB00F46AD4847
:109120000121164603F08CFFAA8812F0010440F0DA
:10913000B080DFF8CC8298F80030002B7DD1AB797D
:10914000A54AD15CA1B9DFF8BCA279781AF80390DE
:1091500041B339780139072900F2B780DFE811F00F
:10916000F1005401B5006C01B500B500B500E9008F
:109170007C78002C00F0CA800139EC68387854F80B
:109180002170FC68411EB4F80080072900F2A78016
:10919000DFE811F074015901A5006C01A500A500DC
:1091A000A5009F00DFF854A2DAF80020B21AB2F549
:1091B000967F75D9894A107801281ABF012010704E
:1091C0001170874A18BF0146D05CC0EB0900C0B2DD
:1091D000FFF7D8F80124CAF80060AB889B0770D568
:1091E0007B78002B6DD0F8F72BFF7E4B7E4A7F48B3
:1091F0001B78127839780078022515FB02330A298A
:1092000003EB800300F04E810C295AD1002B58D07B
:1092100003F11900764E774A013B0021400080B2ED
:1092200026F813100123157088F8003000F080FC38
:10923000714B032220461A702FE0664803F00CF8A9
:109240000121644803F0F6FE62482246214603F0FD
:10925000EDFEAB88580725D42C68204608F070FD39
:10926000214602465B4804F07BF85A4804F08EF829
:10927000092201238DE80C0000217F23554803F0CB
:1092800043FB00212846FFF707FB002388F8003046
:1092900055E7AB683146384698470BB0BDE8F08FCC
:1092A0000846FAE72B6804A8984704A808F048FD88
:1092B00004A90246474804F053F8464804F066F80B
:1092C000D6E720460BB0BDE8F08F00240AF80390E3
:1092D00083E70021D1543846FB699847FC68A4F81D
:1092E0000080002725223C238DE88400412118229C
:1092F000384803F0D7FAE968A879FFF7DFFB374A67
:109300003E4B17701E600BB0BDE8F08F3B490A68FA
:10931000B21AB2F5967FD4D9304F0E603E78012E46
:1093200000F0B480E968184601233B70FFF7C6FBE4
:10933000B3E7304AE9791170012288F8002000244F
:10934000C4E72A7A013A4A45BFDD09F10104E4B2D3
:10935000A145BAD0224E16F803B0CBEB0900C0B23B
:109360000021FFF70FF82B7A052BD9461BD9CBEB41
:109370000402042A40F3AE80A4F1040BBBF1000FF9
:10938000C0F2B080063B5B45A8BF5B465FFA83F93D
:10939000AA791348B15C994205D000F802900121E6
:1093A0002846FFF779FAC9EB0400C0B201210B4E41
:1093B000FEF7E8FF00213423019100930548317046
:1093C00040230B223F21A14603F06CFA0124AB7924
:1093D0007CE700BF949FFF1F00A0FF1F11A0FF1F8D
:1093E0008C9FFF1F199FFF1F1A9FFF1F1B9FFF1FAF
:1093F000409EFF1F10A0FF1F13A0FF1FFC9FFF1F19
:10940000148BFF1F789FFF1F0FFA89F1E868604CEB
:1094100050F821602168049134785E49049808600E
:10942000002C71D0012C7FF450AF5B4A317A88F860
:1094300000401170002449E7B9F1000F50D009F144
:10944000FF34E4B284E7B98A01F0040189B200294B
:109450003FF440AF3B6A03929847039A00283FF4D9
:109460003DAFAB79FC680021D15438E77B8A434596
:109470003CD908F101081FFA88F830E73B8A4345D8
:109480003BD208F1FF381FFA88F828E725238DE83A
:10949000180042483C703C231822412103F002FA94
:1094A0003046FAE6002B3FF40CAF3D4A3D4E1188A2
:1094B000394A03F11900013B400080B226F813102D
:1094C000012388F80030157000F032FB364B20463F
:1094D0001D70E2E6002A3FF755AF04F1FF3B4DE770
:1094E0004C46F3E64FF000094B4651E7BB8ADA07DA
:1094F0007FF5F5AEB7F81080F1E6BB8AD9077FF5A6
:10950000EEAEB7F81280EAE62849C85CC0EB090065
:1095100009F1010EC0B201214FF0340B02F803E053
:10952000FEF730FFB6681D48019440230B223F210F
:109530000124CDF800B003F0B5F940230B223F2100
:109540001648CDF800B0019403F02EFA21461348D6
:1095500003F070FD304608F0F3FBA0EB800000F153
:109560005F0109B20F220D4803F060FD304608F09C
:10957000E7FB31460246094803F0F2FE074803F0D4
:1095800005FFE968A879FFF799FAAB799EE600BF75
:1095900050A0FF1FFC9FFF1F10A0FF1F949FFF1FE5
:1095A000049FFF1F409EFF1F13A0FF1F8C9FFF1FE4
:1095B0002DE9F047DFF808926D4B99F800601B68C1
:1095C000DFF800A282B0003601934FF0030018BF0D
:1095D0000126019F9AF8008004F092FD05460420C0
:1095E00004F08EFD0446052004F08AFD800040EA68
:1095F0004404062004F084FD2C4364B25D4944EA2F
:10960000C0000A7880F00F03DBB29A425A4A3CD07D
:109610001760002259480B7003788DF800808DF890
:10962000012053B3564A12684EF66021BA1A8A4294
:1096300019D8022B59D0012B5FD0062B48D0032B11
:1096400063D0042B69D0052B77D0072B7DD0082B56
:1096500000F08380092B68D016B14A4802F008FF59
:1096600002B0BDE8F087484A484C0023012123702E
:1096700003701360938089F800103A4669464448A5
:10968000FFF748FD3043C6B2E6E71268BA1A1E2A51
:109690006BD99AF80020934222D0394C3D488AF881
:1096A0000030012B276082EA030207609846B1D0A0
:1096B000042BAFD137480068381AB0F5C87FA9D954
:1096C000354C2068381A3228A4D927601A46A1E7F9
:1096D0003A4669463148FFF71DFD3043C6B2BBE745
:1096E000012B4FF00002E3D1E4E73A4669462C48EB
:1096F000FFF710FD3043C6B2AEE73A466946294847
:10970000FFF708FD3043C6B2A6E73A466946264849
:10971000FFF700FD3043C6B29EE73A46694623484C
:10972000FFF7F8FC3043C6B296E73A466946204850
:10973000FFF7F0FC3043C6B28EE73A4669461D4853
:10974000FFF7E8FC3043C6B286E73A4669461A4856
:10975000FFF7E0FC3043C6B27EE73A466946174859
:10976000FFF7D8FC3043C6B276E7002252E700BFCD
:1097700050A0FF1F14A0FF1F809FFF1F10A0FF1FFE
:1097800008A0FF1F949FFF1F00A0FF1F12A0FF1F34
:109790000830010018A0FF1F889FFF1F3834010008
:1097A000842F0100982E0100342E01008C3C010012
:1097B000882E0100F02E0100CC3C01002C91FF1FEF
:1097C000148BFF1F849FFF1F28B11028044BA8BFD4
:1097D000102018607047024B01201860704700BFCE
:1097E0001CA0FF1F38B50F4D2B78013B01381B0221
:1097F000C4B203F47063200443F4404343F00C0309
:1098000000F4FE00184305F0E3FD2868013860F01D
:109810003F00C0B204F00AFE2046BDE8384004F024
:1098200005BE00BF1CA0FF1F70B5124D2B78013B79
:109830001B0203F47063064643F430430806320407
:1098400000F0FE4043F00B03034302F4FE00184314
:109850000C4605F0BDFD2868013860F04F00C0B22D
:1098600004F0E4FD304604F0E1FD2046BDE8704020
:1098700004F0DCBD1CA0FF1F70B5124D2B78013B1E
:109880001B0203F47063064643F4104308063204D7
:1098900000F0FE4043F00903034302F4FE001843C6
:1098A0000C4605F095FD2868013860F06F00C0B2E5
:1098B00004F0BCFD304604F0B9FD2046BDE8704020
:1098C00004F0B4BD1CA0FF1F38B5104D2B78013B30
:1098D0001B0203F47063044643F41043000443F096
:1098E000090300F4FE00184305F072FD28680138F2
:1098F00060F06F00C0B204F099FD204604F096FDC0
:109900000020BDE8384004F091BD00BF1CA0FF1F3F
:1099100038B50E4D2B78013B1B0203F470630446EF
:1099200043F45043000443F00D0300F4FE001843D9
:1099300005F04EFD2868013860F02F00C0B204F039
:1099400075FD2046BDE8384004F070BD1CA0FF1F27
:1099500008B5002005F006FE0028FAD108BD00BFBA
:1099600008B564210720FFF75FFF7F210B20BDE8CA
:109970000840FFF759BF00BF10B500217B20FFF75B
:1099800053FF0024E0B2FFF79FFF0134022004F0F0
:10999000EDFB802CF6D110BD10B504464FF44060AD
:1099A00004F0F4FC04F04CFD2CB1102C044BA8BFC7
:1099B00010241C6010BD024B01241C6010BD00BFB0
:1099C0001CA0FF1F10B5044641F0E00004F02EFD7E
:1099D00004F07F0004F02AFDC4F3C610BDE8104077
:1099E00004F024BD38B5134D2B78044641F6FF72C0
:1099F000A0F50050824203F1FF33A8BF02461B02CC
:109A000002F5005203F47063100443F4604343F022
:109A10000E0300F4FE005204184302F0FE4210430D
:109A200005F0D6FC296801392046C9B2BDE83840A6
:109A3000FFF7C8BF1CA0FF1F38B504460D46F02035
:109A400004F0F4FC35B1254414F8010B04F0EEFCED
:109A5000AC42F9D1F720BDE8384004F0E7BC00BFC4
:109A600000B50B4B83B00246998818680090032A12
:109A7000ADF8041002D903B05DF804FB6846062176
:109A80008DF80520FFF7D8FF03B05DF804FB00BF99
:109A90000C3D010000B50B4B024683B01868998855
:109AA0000090131F4C2BADF8041002D903B05DF8E1
:109AB00004FB684606218DF80520FFF7BDFF03B0C3
:109AC0005DF804FB143D0100030203F4FE43C0F300
:109AD000C6101843704700BF03784078DB0103F4D9
:109AE0007E5300F07F001843704700BF82B002AA87
:109AF000114642F8040D002012F8013B03F07F03E9
:109B0000914243EA0020F7D102B07047003210B40E
:109B100003884FF0010404FA01F418BF012202FA8D
:109B200001F123EA04020A43028010BC704700BF1F
:109B300070B5CEB20C46054603F0AAFE864203D0AD
:109B40003146284603F0BEFE0135284603F0A0FE4C
:109B5000240A844205D021462846BDE8704003F01F
:109B6000B1BE70BD38B5054603F092FE4FF000045B
:109B700060F30704681C03F08BFE60F30F24A0B2AF
:109B800038BD00BFF8B504460020FFF7EBFF002CFE
:109B900000F09C854FF4AF610220FFF7C9FF4FF43E
:109BA0007A610420FFF7C4FF4FF496610620FFF7A7
:109BB000BFFF4FF4FA610820FFF7BAFF4FF4FA61D4
:109BC0000A20FFF7B5FF40F6B8310C20FFF7B0FFD1
:109BD0004FF42F612220FFF7ABFF40F6AC51242059
:109BE000FFF7A6FF7D212A20FFF7A2FF0C210E2000
:109BF000FFF79EFF01211020FFF79AFF022112209C
:109C0000FFF796FF00211420FFF792FF0021162096
:109C1000FFF78EFF02211820FFF78AFF01211A208B
:109C2000FFF786FF01211C20FFF782FF04211E2081
:109C3000FFF77EFF14212020FFF77AFF0121262065
:109C4000FFF776FF03212820FFF772FF04212C2065
:109C5000FFF76EFF14212E20FFF76AFF002130204E
:109C6000FFF766FF0C213220FFF762FF002134204E
:109C7000FFF75EFF00213620FFF75AFF0021382052
:109C8000FFF756FF00213A20FFF752FF00213C204A
:109C9000FFF74EFF00213E20FFF74AFF0021402042
:109CA000FFF746FF00214220FFF742FF1F2144201B
:109CB000FFF73EFF13214620FFF73AFF0E21482011
:109CC000FFF736FF11214A20FFF732FF0A214C200F
:109CD000FFF72EFF00214E20FFF72AFF062150201C
:109CE000FFF726FF02215220FFF722FF0C2154200C
:109CF000FFF71EFF00215620FFF71AFF0021582012
:109D0000FFF716FF01215A20FFF712FF08215C2000
:109D1000FFF70EFF0A215E20FFF70AFF00216020F7
:109D2000FFF706FF04216220FFF702FF01216420F4
:109D3000FFF7FEFE00216620FFF7FAFE0B216820E8
:109D4000FFF7F6FE7F216A20FFF7F2FE00216C206C
:109D5000FFF7EEFE00216E20FFF7EAFE00217020E3
:109D6000FFF7E6FE00217220FFF7E2FE00217420DB
:109D7000FFF7DEFE1F217620FFF7DAFE13217820A1
:109D8000FFF7D6FE0E217A20FFF7D2FE11217C20AC
:109D9000FFF7CEFE0A217E20FFF7CAFE1F2180209A
:109DA000FFF7C6FE13218220FFF7C2FE0E2184209A
:109DB000FFF7BEFE11218620FFF7BAFE0A21882098
:109DC000FFF7B6FE00218A20FFF7B2FE00218C20AB
:109DD000FFF7AEFE00219620FFF7AAFE0021982093
:109DE000FFF7A6FE00219A20FFF7A2FE05219C2086
:109DF000FFF79EFE06219E20FFF79AFE0021A0207D
:109E0000FFF796FE7F21A220FFF792FE40F2A461A9
:109E1000A420FFF78DFE4FF4E161A620FFF788FE36
:109E20000021A820FFF784FE0021AA20FFF780FE72
:109E30000221AC20FFF77CFE0121AE20FFF778FE67
:109E40000121B020FFF774FE0B21B220FFF770FE56
:109E50002A210020FFF76CFE0220FFF783FEB0F5F9
:109E6000805F034680F0F585D24A04201380FFF717
:109E700079FEB0F5805F034680F0E285CE4A062089
:109E80001380FFF76FFEA0F52F739BB2B3F57A6FC7
:109E9000024606D940F628210620FFF749FE40F683
:109EA0002822C64B08201A80FFF75CFEA0F52F730E
:109EB0009BB2B3F57A6F024606D940F6E44108201A
:109EC000FFF736FE40F6E442BD4B0A201A80FFF74A
:109ED00049FEA0F5FA739BB240F6AC518B420246A4
:109EE00006D94FF4FA610A20FFF722FE4FF4FA6216
:109EF000B44B0C201A80FFF735FEA0F5FA739BB225
:109F000040F6AC518B42024606D940F6B8310C20DF
:109F1000FFF70EFE40F6B832AB4B0E201A80FFF76B
:109F200021FE1828034600F28485A84A10201380D9
:109F3000FFF718FE431E9BB20F2B024604D90121E6
:109F40001020FFF7F5FD0122A14B12201A80FFF728
:109F500009FE0A28034600F265859E4A14201380F4
:109F6000FFF700FE0128034604D900211420FFF763
:109F7000DFFD0023984A16201380FFF7F3FD7F28AA
:109F8000034600F24885954A18201380FFF7EAFD42
:109F90000528034600F23885914A1A201380FFF7FE
:109FA000E1FD0C28034600F228858E4A1C20138010
:109FB000FFF7D8FD0428034600F218858A4A1E20C0
:109FC0001380FFF7CFFD0928034600F20885874A72
:109FD00020201380FFF7C6FD4628034600F2F884D0
:109FE000834A22201380FFF7BDFDA0F5FA739BB2D0
:109FF00040F6AC518B42024606D94FF42F61222025
:10A00000FFF796FD4FF42F627A4B24201A80FFF75A
:10A01000A9FDA0F5FA739BB240F6AC54A3420246E8
:10A0200004D921462420FFF783FD2246724B2620C7
:10A030001A80FFF797FD7F28034600F2C2846F4A1B
:10A0400028201380FFF78EFD0628034600F2B28415
:10A050006B4A2A201380FFF785FDA0F132039BB2E3
:10A06000B3F5967F024604D97D212A20FFF760FDD3
:10A070007D22644B2C201A80FFF774FD0C280346C8
:10A0800000F29184604A2E201380FFF76BFD1E289A
:10A09000034600F281845D4A30201380FFF762FDA1
:10A0A0000928034600F25384594A32201380FFF7EF
:10A0B00059FD1E28034600F24384564A342013807B
:10A0C000FFF750FD7F28034600F23384524C3620C0
:10A0D0002380FFF747FD7F28034600F223843820C2
:10A0E0006380FFF73FFD7F28034600F214843A2087
:10A0F000A380FFF737FD7F28034600F205843C204C
:10A10000E380FFF72FFD7F28034600F2F7833E2010
:10A110002381FFF727FD7F28034600F2E9834020D3
:10A120006381FFF71FFD7F28034600F2DB83422097
:10A13000A381FFF717FD394D28804420FFF712FD5A
:10A140003028034600F2C883354A46201380FFF7C3
:10A1500009FD3028034600F2B983324C48202380A1
:10A16000FFF700FD3028034600F2AA834A206380EF
:10A17000FFF7F8FC3028034600F29C834C20A380B4
:10A18000FFF7F0FC3028034600F28E834E20E38078
:10A19000FFF7E8FC0128034604D900214E20FFF711
:10A1A000C7FC0023204A50201380FFF7DBFC431E2E
:10A1B0003CE000BF689DFF1F349FFF1F0E9DFF1FE7
:10A1C000009FFF1FCC9EFF1FD49CFF1FA69CFF1F5C
:10A1D000849EFF1FB89EFF1F5A9DFF1FAA9CFF1F52
:10A1E0006E9DFF1FF69CFF1FEC9CFF1FDC9CFF1F5A
:10A1F000129FFF1F7C9EFF1F789EFF1F049FFF1F63
:10A20000DA9EFF1F2E9FFF1FBE9CFF1F509DFF1F4A
:10A21000409FFF1F029FFF1F409EFF1F369FFF1F93
:10A22000169FFF1FDC9EFF1FEA9CFF1F9BB20B2B9C
:10A23000024604D906215020FFF77AFC0622CF4BB4
:10A2400052201A80FFF78EFC0428034600F2268372
:10A25000CB4A54201380FFF785FC431E9BB21D2B75
:10A26000024604D90C215420FFF762FC0C22C54B96
:10A2700056201A80FFF776FC0128034604D90021F6
:10A280005620FFF755FC0023BF4A58201380FFF7E4
:10A2900069FC7F28034600F2FB82BC4A5A201380E7
:10A2A000FFF760FC431E9BB2092B024604D9012133
:10A2B0005A20FFF73DFC0122B54B5C201A80FFF7C6
:10A2C00051FC431E9BB2102B024604D908215C208E
:10A2D000FFF72EFC0822AF4B5E201A80FFF742FCEE
:10A2E000431E9BB21D2B024604D90A215E20FFF7B4
:10A2F0001FFC0A22A84B60201A80FFF733FC0228BB
:10A30000034600F2BF82A54A64201380FFF72AFCAF
:10A310000128034604D901216420FFF709FC012329
:10A320009F4A62201380FFF71DFCC31E9BB2012BC6
:10A33000024604D904216220FFF7FAFB0422994B5C
:10A3400066201A80FFF70EFC7F28034600F29482F5
:10A35000954A68201380FFF705FC7F28034600F22A
:10A360008582924A6A201380FFF7FCFB7F28034610
:10A3700000F276828E4A6C201380FFF7F3FB0428EC
:10A38000034600F267828B4A6E201380FFF7EAFBD8
:10A390001928034600F25882874A70201380FFF77D
:10A3A000E1FB0228034600F24982844A72201380AE
:10A3B000FFF7D8FB0628034600F23A82804A742051
:10A3C0001380FFF7CFFB0528034600F22B827D4A5E
:10A3D0008A201380FFF7C6FB0A28034600F21C827E
:10A3E000794A8C201380FFF7BDFB0428034600F256
:10A3F0000D82764A98201380FFF7B4FB01280346AC
:10A4000004D900219820FFF793FB0023704A9A207B
:10A410001380FFF7A7FB0128034604D900219A20E7
:10A42000FFF786FB00236B4A96201380FFF79AFB09
:10A430000B28034600F2E481674A9C201380FFF753
:10A4400091FB831E9BB2032B024604D905219C205D
:10A45000FFF76EFB0522614B76201A80FFF782FB27
:10A460003028034600F2C6815D4A78201380FFF74A
:10A4700079FB3028034600F2B7815A4C7A202380BA
:10A48000FFF770FB3028034600F2A8817C20638030
:10A49000FFF768FB3028034600F29A817E20A380F4
:10A4A000FFF760FB3028034600F28C818020E380B8
:10A4B000FFF758FB3028034600F27E814A4A82208B
:10A4C0001380FFF74FFB3028034600F26F81474CA3
:10A4D00084202380FFF746FB3028034600F260818A
:10A4E00086206380FFF73EFB3028034600F252814E
:10A4F0008820A380FFF736FB3028034600F2448112
:10A50000A020E380FFF72EFB0128034604D9002199
:10A51000A020FFF70DFB0023354A9E201380FFF794
:10A5200021FBC31E9BB20C2B024604D906219E20A0
:10A53000FFF7FEFA06222F4BA2201A80FFF712FB2C
:10A54000431E9BB27E2B024604D97F21A220FFF737
:10A55000EFFA7F22284BA4201A80FFF703FBA0F517
:10A56000AF639BB2B3F5167F024647D940F2A461B0
:10A57000A420FFF7DDFA40F2A4623FE02089FF1F2C
:10A580005E89FF1F188AFF1F3E9DFF1FC69EFF1F8B
:10A59000A09CFF1F648AFF1F5C89FF1F749EFF1F22
:10A5A000D49EFF1FFC9CFF1F149FFF1F309DFF1FA9
:10A5B000E09CFF1F949CFF1F6A9FFF1F609EFF1F70
:10A5C0003C9FFF1FF89EFF1F869EFF1F6E9EFF1F72
:10A5D000DE9CFF1F489DFF1FC09EFF1FC29CFF1FE8
:10A5E000D69CFF1F509EFF1FD89CFF1F589EFF1F29
:10A5F000E49EFF1FC489FF1F0A9FFF1FD74BA620A1
:10A600001A80FFF7AFFAA0F5AF639BB2B3F5167FE0
:10A61000024606D94FF4E161A620FFF789FA4FF40C
:10A62000E162CF4BA8201A80FFF79CFA0628034668
:10A6300000F2A480CB4AAA201380FFF793FA0328E4
:10A64000034600F29580C84AAC201380FFF78AFACF
:10A650000328034600F28680C44AB0201380FFF727
:10A6600081FA0328034677D8C14AAE201380FFF74A
:10A6700079FA7F28034669D8BE4AB2201380FFF7D3
:10A6800071FA7F285CD82B88DFF808E3BA4FBB4A01
:10A69000BB4DBC4EBC4CBD4903F0010CAEF800C034
:10A6A000C3F3400EA7F800E0C3F380071780C3F39D
:10A6B000C007B74A2F70C3F30017C3F34015C3F3A5
:10A6C0008013378025800B801080F8BD4FF6FF7314
:10A6D00098423FF45FAA2A283FF4BEAB17287FF6C2
:10A6E00059AA19287FF6C2AA1B287FF6DFAA1C28C0
:10A6F0003FF4F4AA1E287FF6F9AA1F283FF4FEAA09
:10A7000020283FF417AB21283FF420AB22283FF448
:10A7100025AB23283FF42EAB24283FF45FAB25283C
:10A720003FF464AB26283FF465AB27283FF46AABBF
:10A7300028283FF475AB29287FF48AABFFF778BB54
:10A74000B2200B21FFF7F4F90B209CE70121AE208A
:10A75000FFF7EEF901238FE70121B020FFF7E8F9B9
:10A76000012381E70221AC20FFF7E2F9022373E71E
:10A770000021AA20FFF7DCF9002364E70021A820CC
:10A78000FFF7D6F9002355E70A218820FFF7D0F913
:10A790000A23B5E611218620FFF7CAF91123A7E69F
:10A7A0000E218420FFF7C4F90E2399E6132182209D
:10A7B000FFF7BEF913238AE61F218020FFF7B8F9BF
:10A7C0001F237BE60A217E20FFF7B2F90A236DE6FC
:10A7D00011217C20FFF7ACF911235FE60E217A20CE
:10A7E000FFF7A6F90E2351E613217820FFF7A0F911
:10A7F000132342E61F217620FFF79AF91F2333E641
:10A8000000219620FFF794F9002315E600218C2003
:10A81000FFF78EF90023ECE500218A20FFF788F985
:10A820000023DDE500217420FFF782F90023CEE547
:10A8300000217220FFF77CF90023BFE50021702082
:10A84000FFF776F90023B0E500216E20FFF770F9DD
:10A850000023A1E500216C20FFF76AF9002392E5AF
:10A860007F216A20FFF764F97F2383E50B216820AD
:10A87000FFF75EF90B2374E500216620FFF758F916
:10A88000002365E500216020FFF752F900233AE537
:10A8900000215820FFF74CF90023FEE4022152204A
:10A8A000FFF746F90223D3E40A214C20FFF740F9D1
:10A8B0000A236BE411214A20FFF73AF911235DE4E2
:10A8C0000E214820FFF734F90E234FE413214620D0
:10A8D000FFF72EF9132340E41F214420FFF728F946
:10A8E0001F2331E400214020FFF722F900231EE45A
:10A8F00000213E20FFF71CF9002310E400213C203A
:10A90000FFF716F9002302E400213A20FFF710F9BF
:10A910000023FFF7F4BB00213820FFF709F90023DB
:10A92000FFF7E5BB00213620FFF702F90023FFF710
:10A93000D6BB00213420FFF7FBF80023FFF7C6BB8E
:10A940000C213220FFF7F4F80C23FFF7B6BB0021EF
:10A950003020FFF7EDF80023FFF7A6BB6C9DFF1F2B
:10A96000EC9EFF1FA29CFF1F149DFF1FD69EFF1F82
:10A97000649EFF1FE89CFF1F0C9DFF1F529DFF1F41
:10A98000669EFF1F769EFF1FD89EFF1F8A9EFF1F99
:10A99000069DFF1FC29EFF1F14212E20FFF7C8F83F
:10A9A0001423FFF778BB04212C20FFF7C1F8042300
:10A9B000FFF768BB03212820FFF7BAF80323FFF74E
:10A9C00047BB01212620FFF7B3F80123FFF737BB70
:10A9D00014212020FFF7ACF81423FFF701BB04215A
:10A9E0001E20FFF7A5F80423FFF7F1BA01211C2070
:10A9F000FFF79EF80123FFF7E1BA01211A20FFF7C4
:10AA000097F80123FFF7D1BA02211820FFF790F839
:10AA10000223FFF7C1BA00211620FFF789F80023AF
:10AA2000FFF7B1BA02211220FFF782F80223FFF7E5
:10AA300094BA0C210E20FFF77BF80C23FFF775BAB0
:10AA40004FF47A610420FFF773F84FF47A63FFF74D
:10AA500015BA4FF4AF610220FFF76AF84FF4AF6305
:10AA6000FFF702BAF8B5C52006F0C6FB204B214A15
:10AA7000054603CB1368C5F803001A0CB420C5F8CB
:10AA800007102B80AA70FFF71FF82E46002426F827
:10AA90000B0FA0B2FFF766F8FFF716F80234B42CDC
:10AAA00026F8020FF5D16C1E05F1C0064FF0FF30FD
:10AAB00014F8013F082758400F4B40F300017A1E5D
:10AAC0000B4012F0FF0783EA5000F5D1B442EFD1FA
:10AAD000C043FFF70BF83A46C5F8C100C521284628
:10AAE00004F0C4FC2846BDE8F84006F08DBB00BF6A
:10AAF000203D01001C3D01002083B8EDF0B50E4B58
:10AB00000E4C054693E8070085B024682E88AD7882
:10AB100001AB83E80700270C184600220B21ADF893
:10AB200004408DF80670ADF80C608DF80E5004F0FE
:10AB30009DFC05B0F0BD00BF2C3D01001C3D010097
:10AB4000F0B5124B124D1E68124F0FCD87B06C46F8
:10AB50000FC495E8030044F8040B38683B79CDF83E
:10AB60000D00320C2A2021808DF802208DF8113042
:10AB7000ADF80060FEF7A8FF0022ADF80B0012212F
:10AB8000684604F073FC07B0F0BD00BF1C3D010037
:10AB9000383D0100D0350100002004F0E3BC00BFC7
:10ABA00002F02EBE70B5124C82B00025402306463E
:10ABB00029462046009301958023202201F072FE51
:10ABC00020222946204602F031FA2046012102F0D7
:10ABD00037FA304607F0B4F831460246204602F014
:10ABE000BFFB204602B0BDE8704001F041BC00BF91
:10ABF000949FFF1FF0B5C42983B075D90546441E44
:10AC000000F1C0064FF0FF3014F8012F0827504024
:10AC1000404A40F300017B1E0A4013F0FF0782EA1E
:10AC20005000F5D1B442EFD1C043FEF75FFF0146BB
:10AC3000D5F8C1000190019A914202D0B2F17F2F64
:10AC40000BD105F10B00FEF747FFB4280BD03248BB
:10AC5000FFF7A8FF002003B0F0BD3048FFF7A2FFC8
:10AC6000384603B0F0BD05F10D00FEF735FF2A2888
:10AC700040D1002440F6AC5613E004281AD0062830
:10AC800021D008281FD00A2828D00C2822D1A1F5CD
:10AC9000FA7292B2B24201D8FEF74AFF0234B42CE3
:10ACA0000ED004F10D002844FEF716FF022C0146D9
:10ACB000A0B2E2D1B1F5805FEED30234B42CF0D172
:10ACC000012003B0F0BDA1F52F7292B2B2F57A6FF8
:10ACD000E4D8E1E7222801D0242811D1A1F5FA72A5
:10ACE00092B2B242DAD8D7E70D48FFF75BFF0020F7
:10ACF00003B0F0BD0B48FFF755FF002003B0F0BDD7
:10AD00002A28C9D1A1F1320292B2B2F5967FC5D8F4
:10AD1000C2E700BF2083B8ED7C3D0100683D010023
:10AD2000503D0100903D010003290CD970B5461C2F
:10AD300082B005460C46304603222A4907F06EF8D9
:10AD400010B102B070BD70470B2C05D90522264901
:10AD5000281D07F063F840B12448FFF723FF24487B
:10AD600002B0BDE87040FFF7C9BE05F1090103223A
:10AD700001A807F0A3F801A803221E4907F04EF826
:10AD8000D8B103221C4901A807F048F808B301A86C
:10AD900003221A4907F042F8B0B91948FFF702FF39
:10ADA000A11E89B23046FFF725FF0028C9D01548FB
:10ADB00002B0BDE87040FFF7F5BE1348FFF7F2FEA2
:10ADC000FFF750FE1148F3E71148FFF7EBFE11487B
:10ADD000C6E71148FFF7E6FE02B0BDE87040FFF796
:10ADE000AFBE00BF1C3D0100A83D0100B03D010009
:10ADF000C43D0100C83D0100F03D0100083E0100D6
:10AE00000C3E0100203E0100CC3D0100E03D010070
:10AE1000343E0100483E0100F43D01002DE9F043BD
:10AE2000174D2B6883B081460F469046F3B1154EFF
:10AE300034880A1992B218461146328006F05AFD3B
:10AE400028603A464946204402F06CFDB8F1000FF4
:10AE500009D031882868FFF767FF286806F0D4F921
:10AE600000232B60338003B0BDE8F083054E0193CF
:10AE70000846318006F0C0F9019B28601C46E0E7D7
:10AE800024A0FF1F20A0FF1F10B51F4C4FF4FA7025
:10AE9000FBF7B2FE204601F0DFF900221146204602
:10AEA00002F0C4F82046012102F0CAF82046002131
:10AEB00002F0C0F80B221549204602F051FA204654
:10AEC00002F064FA0F221249204602F049FA2046A5
:10AED00002F05CFA0F490722204602F041FA2046B0
:10AEE00002F054FA204601F0C3FA0B4B0B4A1A60E9
:10AEF0004FF4FA70FBF780FEFFF722FE0848BDE82A
:10AF00001040FFF74FBE00BF949FFF1F4C3E010053
:10AF1000583E0100683E0100DCA1FF1F1DAE00008D
:10AF2000703E01000020704790F8392090F83800FA
:10AF3000101A704790F8383090F839209A4205D9A5
:10AF40005A1C034480F83820187E70474FF0FF30B9
:10AF5000704700BF90F8383090F839209A4286BF89
:10AF60001B18187E4FF0FF30704700BF704700BFBE
:10AF700038B50546B0F85E0090B195F85D301446DE
:10AF8000C3F1210294420CD805F13B00184422463B
:10AF900002F0C8FC95F85D30234485F85D3020460A
:10AFA00038BD012014462871EEE700BFB0F85E30CE
:10AFB0006BB190F85D30202B07D8C218013380F8B0
:10AFC0005D30012082F83B1070470123037100209F
:10AFD000704700BF0023426980F8383080F839306C
:10AFE00080F85C3080F85D3080F85E3080F85F304B
:10AFF00006CA30B40D68046943662A4383660A6052
:10B00000A370426990F861301649146813441D7AA0
:10B010005B7B01EBC5051B026D6803F4E06343F045
:10B0200064032B6090F8623013449D7CDB7D01EB60
:10B03000C5011B02496803F4E06343F064030B603D
:10B0400021685368194205D0036927225A700369A1
:10B0500004229A71036920225A71036980229A702E
:10B0600030BC7047A449010043690CCB12681A42F6
:10B070000CD0094B99420AD9084B9942036994BFF5
:10B080001A220D225A70036904229A7170470369CB
:10B0900027225A70F7E700BF7F1A06003F420F00D1
:10B0A00010B50269D378DBB2D90604463DD510212C
:10B0B0005806D17038D503F0040303F0FF02002BCB
:10B0C00051D03D49626E00230B7084F85D30002A38
:10B0D0005BD0904794F85D30002B56D02369D02286
:10B0E0009A70236994F83B201A712369012284F82D
:10B0F0005C200222DA7010BD304B84F860009C4264
:10B100004AD02F4B9C4252D094F8391013791F2902
:10B11000DBB207D82848007820B16018013184F8E4
:10B12000391003760223D37010BD5906C3D4917829
:10B1300001F0100101F0FF000029DDD013F0010340
:10B140001ED194F85C1094F85D00884281BF4B1CBE
:10B15000091984F85C3091F83B3013712369D022CF
:10B160009A702269DEE7236984F83920C0229A7038
:10B170002369114A1979012111700222DA7010BD78
:10B18000C023937022691379CCE70122002384F84D
:10B190005D2084F83B30A1E7626994F86130094989
:10B1A00013440322187A02F043FD2269ACE7626976
:10B1B00094F861300449F3E728A0FF1F7491FF1F42
:10B1C000E091FF1F29B2000035B200000369DB786F
:10B1D00003F0200373B190F860300133DBB2012B30
:10B1E00080F860301AD9426990F861301344187AB7
:10B1F00002F09ABD70B5426903F0FF0590F8613026
:10B2000013440446187A02F08FFDA36E5BB184F8F4
:10B21000385094F83900BDE87040184790F85F3016
:10B22000002BE0D0704770BD0148FFF7CFBF00BFD3
:10B230007491FF1F0148FFF7C9BF00BFE091FF1FD6
:10B240002DE9F047374FDFF8E0903B68026982B0A4
:10B2500006460093DDF800800021A025D3789B06E8
:10B260005BD53B680193019BC8EB03030F2BF5D91A
:10B2700049B1102BF2D000209070336980229A706F
:10B2800002B0BDE8F087726996F861301344052179
:10B29000187A02F043FF726996F861301344012175
:10B2A00093F812A0504602F039FF092400215046BD
:10B2B00002F020FF2B46013BFDD10121504602F058
:10B2C00019FF2B46013BFDD1013CEFD1706996F887
:10B2D000611001444FF4A0720C7A4B7B09EBC4015E
:10B2E0001B02496803F4E06343F064030B6096F8C3
:10B2F00062300344997CDB7D09EBC1011B02496884
:10B3000003F4E06343F064030B60013AFDD132695A
:10B31000D3789B064FF00101A3D4012002B0BDE811
:10B32000F08700BF50A0FF1FA4490100F0B50369DA
:10B330001222DA700269937803F0200385B0044684
:10B340000D46002B5ED0B42393703C4922690B68F4
:10B350000093009E05E00B680193019B9B1B042B4F
:10B3600042D8D37803F0200303F0FF00002BF2D083
:10B3700094F85D30002B31D04FF0000E4FF0020CEE
:10B3800004EB0E0393F83B3013710B680393039F98
:10B39000206907E09B060DD50B680293029BDB1B1F
:10B3A000052B28D8C378DBB203F0020202F0FF06B7
:10B3B000002AEFD080F803C02669F378DBB2DF06FD
:10B3C00032462DD49F062BD5DB0731D40EF1010E6A
:10B3D00094F85D305FFA8EFE7345D1D800201DBB16
:10B3E000002384F85E3004E09070236980229A7014
:10B3F000042005B0F0BD86702369802204209A7075
:10B4000005B0F0BD03F0FF06FFF71AFF10B90420E6
:10B4100005B0F0BD236984F85F60B0229A7094E7AC
:10B420008023B3700420DAE726698023B370D7E75E
:10B43000BEF1000F0CBF02200320F6E750A0FF1F53
:10B440002DE9F04106690025122780F8385080F870
:10B450003950F770D0F810C09CF802E00EF0200EC2
:10B4600088B00446884615461E46BEF1000F49D0F6
:10B47000B4238CF80230784B21691A680092DDF809
:10B4800000E006E01A6801920198CEEB0000042863
:10B4900030D8C87800F0200000F0FF070028F1D075
:10B4A0004FEA480242F00102D2B20A711A680292CF
:10B4B000DDF808E0206906E01A6803920399CEEBF4
:10B4C000010105292AD8C17801F0020101F0FF0726
:10B4D0000029F1D04FF0020C80F803C02269D17826
:10B4E00011F0110722D12DBB002E0CBFA023802309
:10B4F000937003E08F70236980229A70384608B0F9
:10B50000BDE8F0810EF0FF07FFF79AFE0028F5D0A6
:10B51000236984F85F70B0229A70ACE78770236962
:10B52000802238469A7008B0BDE8F081802393707D
:10B530000027E3E7012D75D0A021917021690A79D8
:10B54000BE4667464FF0A80C1A680492049805E0BE
:10B550001A680592059A121A052A4AD8CA7802F082
:10B56000020202F0FF08002AF2D0CF702169CA78E7
:10B57000D2B212F0100F08465AD1920658D5013DAA
:10B58000EDB2012D49D0BEF11F0F3BD90A79012D33
:10B59000DAD11A680692069D05E01A680792079AA2
:10B5A000521B052A46D8C27802F0020202F0FF01BF
:10B5B000002AF2D00223C3702269D378DBB2D90605
:10B5C0003AD49B0634D5B023BEF11F0F93703FD8F9
:10B5D000226904EB0E0312791A760EF1010E5FFA5E
:10B5E0008EFE16B1236980229A7084F839E077467E
:10B5F00084E781F80280236980229A70774684F874
:10B6000039E07BE704EB0E0291F8048082F81880A1
:10B610000EF1010E5FFA8EFEB9E781F802C02169D2
:10B620000846B0E7A82191702069BE460279B0E7CC
:10B63000774663E78170DEE71021A023D170013BDC
:10B64000FDD12269937803F0F7037746937055E7AD
:10B6500023691B79C5E700BF50A0FF1F0148FFF712
:10B660001FBD00BF7491FF1F0148FFF719BD00BF48
:10B67000E091FF1F704700BF38B5144C03780122DA
:10B680005B000546204684F83B3084F85E2084F851
:10B690005D20FFF78BFC20460021FFF747FE0B4C97
:10B6A0002978012320461A46FFF7CAFE0128F6D161
:10B6B00094F8383094F839209A4205D9E2180133C9
:10B6C00084F83830107E38BDFF2038BD7491FF1FDC
:10B6D00038B51B4C037801225B000546204684F8F0
:10B6E0003B3084F85E2084F85D20FFF75FFC204645
:10B6F0000021FFF71BFE124C29782046012302226D
:10B70000FFF79EFE0228F6D194F8382094F83910FD
:10B710008A420FD2531CDBB2A018994284F8383009
:10B72000007E0AD9234402321B7E84F8382040EA86
:10B73000032038BD4FF6FF7038BD40F47F4038BD60
:10B740007491FF1F0C2901D9002070470231490074
:10B7500001F0FE01FFF7BCBF70B50C4C0378164634
:10B7600001255B00204684F83B3084F85E5084F865
:10B770005D50FFF71BFC31462046FFF717FC2946BA
:10B780002046BDE87040FFF7D1BD00BF7491FF1F98
:10B79000F8B505460F461646412421463A46284646
:10B7A000FFF7DAFF611C0234C9B232462846E4B220
:10B7B000FFF7D2FF592CF0D1F8BD00BF38B50446D1
:10B7C0000D463548FFF706FC632280212046257090
:10B7D000FFF7C2FF012002F0C9FC204600225E21D3
:10B7E000FFF7BAFF20465D21FFF746FF242801D06E
:10B7F000002038BD204606220C21FFF7C9FF204655
:10B8000001222B21FFF7A8FF204601222C21FFF760
:10B81000A3FF20460E222D21FFF79EFF2046002287
:10B820002E21FFF799FF204601222F21FFF794FFD9
:10B83000204605223021FFF78FFF204601223121CB
:10B84000FFF78AFF204600223221FFF785FF2046BE
:10B8500000223321FFF780FF204600223421FFF72A
:10B860007BFF204600223521FFF776FF204600228D
:10B870005B21FFF771FF204610225C21FFF76CFF70
:10B88000204620225D21FFF767FF20468F225E21A0
:10B89000FFF762FF012038BD7491FF1F10B4047FD1
:10B8A0004160022CC26002D010BC01F0D7BB83689B
:10B8B00010BC184790E80C00F0B41C685968256863
:10B8C000164F174E29432160164D17491760D66051
:10B8D00015611160417A154A5C180A3194F82440C8
:10B8E00053F8215002EBC40149680D60017A5C18DD
:10B8F00003EB8101247ECD6902EBC40149680D6030
:10B90000817A581803EB810390F83000596B02EBF1
:10B91000C002F0BC53681960704700BF01401F00AF
:10B92000011000380110007800001F80A4490100B8
:10B93000704700BFF0B50C1EBDF8146034DBB0F9E1
:10B9400006701919B942C4BF3B1B1BB2002BA64697
:10B950001CDD002A1146B8BFD11D02F00705CC102E
:10B96000826A012007FB04E1A840012E0A44C0B20C
:10B970001ED00CD3022E09D1013B12FA83F3013AF7
:10B9800012F8011F41409A421170F9D1F0BDC04335
:10B99000013B12FA83F3C0B2013A12F8011F0140D1
:10B9A00093421170F9D1F0BD23441BB20024C6E7C5
:10B9B000013B12FA83F3013A12F8011F01439A4244
:10B9C0001170F9D1F0BD00BFF8B50D1E0EDB1446A5
:10B9D0001F46064601F03AFBA84207DD002C05DBB6
:10B9E000304601F037FBA04201DCF8BDF8BD30461F
:10B9F00001F02AFB022853D003284BD0012806D19E
:10BA00006540F3886C406540013B5D1B2DB2012F02
:10BA100003D02AD3022F14D0F8BD002C2246B6F949
:10BA20000630B06AB8BFE21D42F3CF0202FB0355F5
:10BA300004F00704435D012101FA04F41C4344555A
:10BA4000F8BD002C2246B6F90630B06AB8BFE21D38
:10BA500042F3CF0202FB035504F00704435D0121CA
:10BA600001FA04F45C404455F8BD002C2246B6F9B6
:10BA70000630B06AB8BFE21D42F3CF0202FB0355A5
:10BA800004F00704435D012101FA04F423EA0404ED
:10BA90004455F8BD3389013B591B25460CB2B6E726
:10BAA000F18832890139013A4D1B141B2DB224B2A1
:10BAB000ADE700BF2DE9F041079E9DF91880089D74
:10BAC00004461F4600F0C0FF0D4B0E480E4984F897
:10BAD0003380FF22002F08BF1F4684F82F20002349
:10BAE00084F8302084F8312084F832202060A66564
:10BAF000E565676261652362A3622046BDE8F08167
:10BB00007491FF1FFC3E01000110013810B504467E
:10BB1000806A034B236008B105F076FB204610BD18
:10BB2000FC3E0100F8B5436ADBB190F82C200125FA
:10BB3000AA4083F83B2083F85E5083F85D500446AA
:10BB4000406A03680E461B6800219847606A0368D4
:10BB500031461B6898472946606ABDE8F840FFF700
:10BB6000E5BBC26BC56C1368046A23EA0503136066
:10BB70004CB122684FF00043D3625163D36A002B6B
:10BB8000FCDA936BF8BD836B466B0825802410E0CC
:10BB90003768426C3A4332601F68826C3A431A60DD
:10BBA0001A68876C013D22EA07024FEA54041A60C2
:10BBB00007D02142ECD13268476C22EA070232609A
:10BBC000EAE7F8BD70B50446406A0D4600282BD060
:10BBD000A16DFFF749FA002D20460CBFA621A72131
:10BBE000FFF7A0FF606A20B1E16DBDE87040FFF78C
:10BBF0003BBA216C226D0868236A02430A6093B144
:10BC0000DA7A82B1D00703D5224A99691160DA7ACB
:10BC1000910703D5204AD9691160DA7A520702D513
:10BC20001E4A1B6A136070BD236A002B2BD0D97A81
:10BC3000626DE1B172B6D97ACE0706D51848D968D7
:10BC40000668314099610160D97A880706D51548A0
:10BC5000196906683140D9610160D97A4E0705D566
:10BC600011485969066831401962016062B61B6863
:10BC7000D968914207D00D4818600D49DA6042F04A
:10BC8000804018611960226C216D136823EA01035A
:10BC90001360A0E700E100E004E100E008E100E05B
:10BCA00080E100E084E100E088E100E001403F0045
:10BCB00000003F80436A2DE9F04105460E4690465C
:10BCC000002B3ED090F82C100124A14083F83B10AB
:10BCD00083F85E4083F85D40406A036800211B687A
:10BCE00008F1FF379847FFB2B8F1000F23D037446F
:10BCF000A046013E686A16F8011F03681B68984752
:10BD00000134B742E4B216D0202CF3D10121686A85
:10BD1000FFF70CFB95F82C206B6A520083F83B2050
:10BD200083F85E8083F85D80686A036800211B6881
:10BD300098470124DEE7686A0121BDE8F041FFF77A
:10BD4000F5BAC26BC16C136823EA010306EB080461
:10BD500013604FF00048A6420ED02B6A16F801EB94
:10BD600063B11A68C2F82C80C2F834E0D36A002BA1
:10BD7000FCDAA642936BF0D1BDE8F081AB6BD5F84D
:10BD800034C008208021DCF800206F6C1EEA010F0F
:10BD900014BF3A43BA43CCF800201A68AF6C3A4358
:10BDA0001A601A68AF6C013822EA07024FEA5101A3
:10BDB0001A60E8D1CFE700BF70B50446406A0D466F
:10BDC000002828D0A16DFFF74FF920462946FFF73C
:10BDD000A9FE606A20B1E16DBDE87040FFF744B98B
:10BDE000216C226D0868236A02430A6093B1DA7AF3
:10BDF00082B1D00703D5234A99691160DA7A910795
:10BE000003D5214AD9691160DA7A520702D51F4A4F
:10BE10001B6A136070BD236A002B2BD0D97A626D28
:10BE2000E1B172B6D97ACE0706D51948D968066845
:10BE3000314099610160D97A880706D5154819699A
:10BE400006683140D9610160D97A4E0705D512489C
:10BE50005969066831401962016062B61B68D96889
:10BE6000914207D00D4818600D49DA6042F08040D9
:10BE700018611960226C216D136823EA01031360B5
:10BE8000A3E700BF00E100E004E100E008E100E01A
:10BE900080E100E084E100E088E100E001403F0053
:10BEA00000003F802DE9F041044686B0806A9DF88D
:10BEB00030801E460F461546B4F90830002800F0C1
:10BEC0004281DA1D48BF03F10E02B4F90630D210E8
:10BED00003FB02F2002105F0BBFCB4F90820202A84
:10BEE00000F39280B4F90610A34B0120203A733975
:10BEF00002EBD27201EBD1714FF0200E0290732051
:10BF00008DE8014042F34F0241F34F01204600F01B
:10BF100051FE606A84F82D70002800F04D81002DDC
:10BF200040F08A80B4F90830202B14BF3D253C2511
:10BF300084F82C50B8F1000F40F0858006B394F9D6
:10BF40003300002818DBC0B2012102F0E7F801211C
:10BF500094F8330002F0CEF8012002F007F9002136
:10BF600094F8330002F0C6F80A2002F0FFF801212D
:10BF700094F8330002F0BEF8606A002800F0828076
:10BF8000A16DFFF771F804227C492046FFF792FE6D
:10BF9000217A0139C9B22046FFF7C4FD784904224D
:10BFA0002046FFF787FE94F92D30012B14BF142192
:10BFB00010212046FFF7B6FD042272492046FFF704
:10BFC00079FEB4F90630802B00F09280602B00F0EF
:10BFD000A680D9212046FFF7A5FD94F92D30012B2D
:10BFE00014BFF12122212046FFF79CFD20460622A6
:10BFF0006549FFF75FFE606A50B3E16DFFF734F803
:10C00000012006B0BDE8F081B4F906105F4B0120B5
:10C01000403A52394FF0400E029002EBD272522059
:10C0200001EBD1718DE8014042F34F0241F34F0122
:10C03000204600F0BFFD6CE76DB284F82C50B8F1DB
:10C04000000F3FF47BAFFEF7C5FF002E94D076E7DC
:10C05000216C226D0868236A02430A6073B1DA7AA0
:10C0600062B1D00703D54A4A99691160DA7A91071B
:10C070007CD4520702D5474A1B6A1360012006B0E0
:10C08000BDE8F081236A002B2BD0D97A626DE1B133
:10C0900072B6D97ACF0706D53F48D96805682940D6
:10C0A00099610160D97A8E0706D53C4819690568FF
:10C0B0002940D9610160D97A4D0705D538485969B9
:10C0C000056829401962016062B61B68D96891420F
:10C0D00007D0344818603449DA6042F08040186173
:10C0E0001960226C216D136823EA010313604AE78B
:10C0F000B4F90830202B00F08680402B7FF469AF24
:10C100002A4920460322FFF7D5FD94F92D30012B53
:10C1100014BFCF219F212046FFF704FD59E7B4F952
:10C120000830102B7FF455AF214920460322FFF73A
:10C13000C1FD94F92D30012B14BFAF2110212046F1
:10C14000FFF7F0FC45E7DA1D48BF03F10E02B4F932
:10C150000630D21003FB02F21046059205F04CF8AF
:10C16000A06200283FF44DAF059AB3E6114AD969A1
:10C170001160DA7A7DE700BF543F010034410100CD
:10C18000384101003C4101004041010048410100AB
:10C1900000E100E008E100E080E100E084E100E08F
:10C1A00088E100E001403F0000003F80503F010077
:10C1B0000844010004E100E0012194F83100244F1B
:10C1C00001F0ACFF94F83200012101F0A7FF94F9CF
:10C1D000312094F9323057F83220E26357F8333087
:10C1E000206A23640125E56425651A682A431A60DC
:10C1F00078B1B8F1000F3FF428AFFFF75BFB002EDA
:10C200003FF4BAAE9BE6042212492046FFF752FDE6
:10C21000DFE6294694F82F0001F080FF294694F8C4
:10C22000300001F07BFF94F92F2094F9303057F85B
:10C230003220626357F833306564A5641A68A363DB
:10C2400022F001021A60002E3FF496AE77E600BF9E
:10C25000A44901004C3F0100B0F90820D31D48BF9C
:10C2600002F10E03B0F90620806ADB1002FB03F234
:10C27000002105F0EDBA00BFF0B50029BDF814505B
:10C280002EDBB0F90660B1422ADA002A59DBB0F998
:10C29000087014461C44BC42C4BFBB1A1BB2002B1E
:10C2A0001EDDD2B2D408D0F828E016FB041112F03B
:10C2B0000702DBB20EEB010421D0C2F10807FAB28B
:10C2C000374F9342BF5C0CD2C3EB020CFF2646FAF9
:10C2D0000CF6012D07EA06073FD005D3022D36D014
:10C2E000F0BD012D39D030D21EF8016026EA0707D3
:10C2F0000EF801709342F3D3B0F906100C449A1A69
:10C30000D2B2072A10D9022D36D0002D14BFFF2635
:10C31000002613462670083BB0F90610DBB2072B47
:10C320000C44F7D802F00702002AD9D01D4B012D8A
:10C330009B5C1DD017D3022DD2D12278534023709D
:10C34000F0BD13441BB20022A1E7022D25D11EF837
:10C35000016077400EF80170CCE71EF801603743AA
:10C360000EF80170C6E7227822EA03032370F0BDBD
:10C37000227813432370F0BD11462378DB432370EA
:10C380000839B0F90630C9B207291C44F5D812F0B3
:10C390000702A5D0034B9B5CCFE73444AFE700BF57
:10C3A000EC3E0100DC3E010070B4C47DBDF80C50D1
:10C3B000022C18D0032C1FD0012C0BD0002A03DB39
:10C3C000B0F90840944201DC70BC7047039570BC22
:10C3D000FFF7B0BAC4880395013CA41A0A4621B2FB
:10C3E00070BCFFF749BF0689C488013E641AB21ABF
:10C3F000E41A12B221B2E1E704890395E41A641A3F
:10C40000114622B270BCFFF737BF00BF70B4C57DC4
:10C41000BDF80C60022D1AD0032D12D0012D03D0CF
:10C42000039670BCFFF728BFC488E41AA41A0A4612
:10C4300021B2002A03DBB0F90840944213DC70BC3F
:10C4400070470489013C641A114622B2F1E7C4889E
:10C4500005890396013CAD1AED1A621A11B22AB28F
:10C4600070BCFFF709BF039670BCFFF763BA00BF4B
:10C470002DE9F8430446406A002863D0A16DFEF719
:10C48000F3FD052274492046FFF714FCA179013918
:10C49000C9B22046FFF746FBB4F90820E588A66A32
:10C4A000D31D48BF02F10E03DB10626A15FB03F5D2
:10C4B0001FFA85F8002A7BD094F82C300125AB4078
:10C4C00082F83B3082F85E5082F85D50606A036803
:10C4D00040211B6808F1FF379847BFB2B8F1000F41
:10C4E00023D03744A846013E606A16F8011F03684E
:10C4F0001B6898470135B742EDB216D0202DF3D115
:10C500000121606AFEF712FF94F82C20636A520042
:10C5100083F83B2083F85E8083F85D80606A03685F
:10C5200040211B6898470125DEE70121606AFEF77C
:10C53000FDFE606A002800F08D80E16DBDE8F843E3
:10C54000FEF792BD236A002B2BD0D97A626DE1B140
:10C5500072B6D97ACE0706D54048D9680568294011
:10C5600099610160D97A8D0706D53D48196905683A
:10C570002940D9610160D97A480705D539485969F8
:10C58000056829401962016062B61B68D96891424A
:10C5900007D0354818603549DA6042F080401861AC
:10C5A0001960226C216D136823EA0103136068E7A8
:10C5B000E26BE36C1168276A0B4306EB0809136012
:10C5C0004FF0004E4E450DD016F801CB2FB33A6810
:10C5D000C2F82CE0C2F834C0D36A002BFCDA4E4516
:10C5E000936BF1D1226C236D11680B43136097B1EB
:10C5F000FB7A83B1D90703D51D4BBA691A60FB7A60
:10C600009A0703D51B4BFA691A60FB7A5B0702D5C0
:10C61000194B3A6A1A60BDE8F883A36BD4F83480EA
:10C6200008208021D8F80020656C1CEA010F14BF97
:10C630002A43AA43C8F800201A68A56C2A431A6046
:10C640001A68A56C013822EA05024FEA51011A6006
:10C65000E8D1B7E7276AC5E7E43E010080E100E0E2
:10C6600084E100E088E100E001403F0000003F80FD
:10C6700000E100E004E100E008E100E02DE9F04F16
:10C6800085B09946BDF93870BDF83CA0BB1AC1EB26
:10C69000090B002BB8BF5B42BBF1000FB8BFCBF159
:10C6A000000B5B450D4616460093804648DC4D4521
:10C6B0003A4633464CDC194613460A46C5EB090197
:10C6C0009B1A89B2002B0CB2B8BF5B4204EBD47446
:10C6D000BE42ACBF4FF0FF3201224D4503910292A2
:10C6E0004FEA640429DC9BB201930DE0D8F8007096
:10C6F000BF69B847019BE41AA3B21CB20135002CF4
:10C700002DB211DBA94518DB009B5B452A46534639
:10C7100031464046EADCD8F800205346976929465E
:10C7200032464046B847E5E7029A1644039AA945BF
:10C7300002EB030436B224B2E6DA05B0BDE8F08FAE
:10C740004A462B46B94635464D4517461E46B2DD8C
:10C75000304629463E464D4607468946AEE700BF6D
:10C7600010B404682469A44610BC604730B404685F
:10C77000BDF808500295A46BA44630BC604700BFCA
:10C7800030B40468BDF808500295E46BA44630BC90
:10C79000604700BF70B40468BDF90C60BDF810506C
:10C7A00003960495246CA44670BC6047704700BF94
:10C7B00010B582B0B0F90C200191016800920022FE
:10C7C0000C6CB0F90A301146A04702B010BD00BF92
:10C7D000704700BF01F003010129C17506D003298C
:10C7E00004D0C28803894281838170470289C3884B
:10C7F00042818381704700BF2DE9F0410568134EE7
:10C800006F6986B0B7420446BDF8308010D1013B55
:10C8100013441BB20093CDF804800B46AD6A20464A
:10C82000A8472368DB6AB3420AD106B0BDE8F081AD
:10C83000059304920391B84703A925680EC9E6E75A
:10C84000204606B0BDE8F041184700BFADC7000064
:10C850002DE9F0410568124E6F6986B0B742044673
:10C86000BDF830800FD1013BCDF804800B4400921D
:10C870001BB2AD6A2046A8472368DB6AB3420AD1DF
:10C8800006B0BDE8F081059304920391B84703A96F
:10C8900025680EC9E7E7204606B0BDE8F041184715
:10C8A000ADC700002DE9F04F0568DFF858B06F699B
:10C8B00085B05F450646BDF93890BDF83CA00C46F2
:10C8C000904615D11F19BC420CDACDF800A02146C4
:10C8D00001342D6A4B464246304624B2A847BC423A
:10C8E0003568F2DBEB6A5B4507D105B0BDE8F08F38
:10C8F0000393B8473568039BE4E7304605B0BDE8CD
:10C90000F04F1847ADC700002DE9F04387B09942BA
:10C910000546BDF93840BDF83C6025D0A24212D092
:10C920000768DFF88080D7F81490C14532D18DE8D0
:10C9300050002846BC6AA0472B68DB6A434524D1D7
:10C9400007B0BDE8F083994202DD08461946034668
:10C9500028680E96C46B01335B1A1BB22846A446A6
:10C9600007B0BDE8F0436047A24202DD134622460D
:10C970001C4628680E96631C846B9B1A1BB22846C3
:10C98000A44607B0BDE8F0436047284607B0BDE8BD
:10C99000F0431847059304920391C84703A92F68F1
:10C9A0000EC9C4E7ADC700002DE9F04FD0F800E094
:10C9B000DFF89090DEF814B083B0CB450446BDF9A3
:10C9C0003080BDF834A00D4617461E4631D1CDF853
:10C9D00000A0DEF824B0294633463A462046D84720
:10C9E0002368CDF800A008F1FF323A44D3F824B010
:10C9F000294612B233462046D8472368CDF800A016
:10CA00002946D3F820B03A4643462046D847206806
:10CA1000CDF800A0711E29444346056A09B23A4682
:10CA20002046A8472368DB6A4B4506D103B0BDE822
:10CA3000F08FD847D4F800E0C9E7204603B0BDE83E
:10CA4000F04F1847ADC70000F0B4002401264FF6A0
:10CA5000FF75094F07600471C475C4810482447670
:10CA6000C4618675067685824582C18002814181D6
:10CA70008281F0BC704700BF144401002DE9F04FE3
:10CA800085B00668BDF84450BDF93880CDF8008007
:10CA900004460195D6F848B00392BDF93C60BDF953
:10CAA000407089469A46D8472368019500974246C8
:10CAB0005146D3F8488020463346C0472068039B40
:10CAC0000E930F95856C4B463A4631462046AC4650
:10CAD00005B0BDE8F04F60472DE9F04F87B017462D
:10CAE000BDF9404000912546E91D059344BF2B4602
:10CAF00003F10E010268BDF8486053690294C91041
:10CB000003912B49BDF9444001968B42824645D1A1
:10CB1000002C3CDD029B3C445E1EB6B24FF0000987
:10CB200023B2049301364D46029B002B28DD059B62
:10CB3000002403EB090806E0EDB22B0604F1010422
:10CB400011D4A6421CD0A1B211F0070F23B24FEAB4
:10CB50004505F1D1002BB8BF0733DB10013418F8BD
:10CB600003502B06EDD5009BD2F818B019443A4675
:10CB700009B2019B5046D847A642DAF80020E2D11C
:10CB8000039B01379944049B3FB2BB42CCD1D36A8B
:10CB9000074A934206D107B0BDE8F08F9847DAF80C
:10CBA0000020B5E7504607B0BDE8F04F184700BF7A
:10CBB000ADC7000070B4BDF90C60BDF91050BDF8F0
:10CBC000144003960495059470BCFFF785BF00BF21
:10CBD0002DE9F04F93B090460591C1691090BDF8D2
:10CBE00070000790BDF874909DF878A00493002918
:10CBF00000F0CD800A7A0AC9894604998A1AD2B20D
:10CC000003EBC203BAF1010FDA780B9293F9052016
:10CC10001E8893F802B00F9293F9064079D913B2A7
:10CC2000099323B20C93109B1A68A94B11931946D0
:10CC300053698B4240F0A6800B9B002B55D01FFA06
:10CC400088F300210D93C8462344DDF840900691F7
:10CC50000E930F460C46BBF1000F3FD0BDF81810E5
:10CC60000C9B03971FFA8AF0CB1813FB00F3049078
:10CC70000E9801440D98034409B21BB20A9108931F
:10CC8000002505E00135EBB264009B45E4B222D9F2
:10CC9000039B2B44590703D1731C18F806409EB21E
:10CCA0002306EFD5099BBDF81000E91811FB00F130
:10CCB0000598BAF1010F0FFA8AF301441CD00798C6
:10CCC00001900093D26909B217464846089AB847BE
:10CCD000D9F80020D6E7039F5F44FFB2069B0B996B
:10CCE00001330693DBB29942B5D8D36A119A9342C5
:10CCF00043D113B0BDE8F08F0F9B191893690A9ABE
:10CD000029441F4609B2079B4846B847D9F8002076
:10CD1000B8E700230C93099385E70A9A0D9B01322B
:10CD2000013B52B213F0FF030A920D936FD1DDF86D
:10CD30001890079BDDF83C80DDF820A04B4517D00C
:10CD4000BAF1010F00F0C8800B9A109DCDF8049045
:10CD50000BEB8B014FEACB030A4400931146DEF83C
:10CD60001C405346424609B22846A047D5F800E089
:10CD7000DEF82C30119A9342BBD0109813B0BDE866
:10CD8000F04F1847109D284698472A6854E7109A94
:10CD90000598B2F90A308342ABDDB2F90C30434555
:10CDA000A7DD062313FB0A03002BA2DD08EBCA0351
:10CDB000002B9EDD537E2BB9049BAF2B02D9013390
:10CDC000DBB20493109BD3F800E0414B11931A4659
:10CDD000DEF81430934240F08E801FFA88F30E93F1
:10CDE00008339BB2BDF81420059305230D9300234F
:10CDF0000A93CDF83C800FFA8AF3DDF84080CDF835
:10CE000018900B921FFA8AFBCDF820A099460A9A37
:10CE1000BDF810000B9C0E9D0523194611FB002345
:10CE20002C481146C75C039702FB0B4214FA81F3AE
:10CE300012B21BB209920C932C462E461CE0089BA2
:10CE40000999012B2AB24B4640462DD0079F0197E6
:10CE5000CDF80090DEF81CA0D047D8F800E0039B86
:10CE60005B0801340393059BA4B25D445E44A34276
:10CE7000ADB2B6B23FF451AF039BD807DFD4079BE6
:10CE8000069A9342EBD0089B012B16D0069B019388
:10CE9000CDF80090DEF81CA009994B4632B240460E
:10CEA000D047D8F800E0DAE7DEF818A0079B0C9925
:10CEB00022B2D047D8F800E0D1E7DEF818A00C99EC
:10CEC0001346404622B2D047D8F800E0C7E700BF7B
:10CED000ADC70000644401000B99109DCDF800908F
:10CEE0000531DEF8204009B2424608232846A04713
:10CEF000D5F800E03CE7109C20469847D4F800E0C5
:10CF00006BE700BFF0B5C36985B004462BB30A29AF
:10CF100068D00D294AD01A7A914247D3587A88426C
:10CF200044D35D688A1A05EBC205AA78002A50D05E
:10CF3000E87800284DD0207E00283AD095F905E009
:10CF4000B4F90E00A67DB4F90A70724406FB020221
:10CF5000BA4262DCB4F9102030E00A2956D00D291B
:10CF600024D0027E002A4BD0B0F90E00A57DB4F982
:10CF70000A60062212FB0502B2423EDD228AE381EC
:10CF800002EBC50212B218462282A78A668A02956F
:10CF90000B468DE8C00001462046FFF719FEA37D31
:10CFA000E28903EB430302EB4303E381012005B075
:10CFB000F0BDA67DB4F90E00B4F91020B4F814E069
:10CFC000678A02960B468DE8804001462046FFF7AF
:10CFD000FFFD2979E389A27D012001FB0233E38172
:10CFE00005B0F0BD0022C2819A7A817D038A01FBDF
:10CFF00002330382012005B0F0BDB4F91020C4E76C
:10D00000857DB4F91020B0F90E00BEE7028A817D5B
:10D01000C38102EBC1030382C8E70020E0819B7A51
:10D02000228A03FB062212B22282C7E7C181028252
:10D03000704700BF002908BF01218175704700BFFC
:10D0400081824182704700BFC07D7047B0F90A00FD
:10D05000704700BFB0F90C00704700BF10B4EFF389
:10D06000108272B6437F33B9017F012907D00329AB
:10D070000FD00123437702B962B610BC7047124C3F
:10D080002168A1B1114943610B688361086058614F
:10D09000EFE70F4C216881B10E4943610B68836152
:10D0A000086058610C4B4FF080511960E1E7074B65
:10D0B0004161816120601860DBE7064B416181615D
:10D0C00020601860EEE700BF3CA0FF1F38A0FF1FE4
:10D0D0002CA0FF1F30A0FF1F04ED00E070B5EFF3A0
:10D0E000108272B60C4C206880B10C4E002543694A
:10D0F000236073B19D6102B962B645778368984732
:10D10000EFF3108272B620680028F0D102B962B63F
:10D1100070BD3360EFE700BF2CA0FF1F30A0FF1FE2
:10D12000FFF7DCBF184A30B41468002C27D003681E
:10D1300021688B420ED2CB1A00218460C16023602B
:10D14000E06010600223037530BC704711688B42A9
:10D15000144608D3A2685B1A0360002AF6D18260E5
:10D16000C460A060EEE7D268C2608460E060C56819
:10D17000CB1A0222A8602360027530BC704784601D
:10D18000C4601060DEE700BF34A0FF1FF8B5224E78
:10D1900034682CB32368002B3AD1204F1D4604E09D
:10D1A0003468ECB12368002B32D1A36803B1DD6091
:10D1B00020693360036825751B68BB4221D1037F5A
:10D1C0004560022BC46020D0FFF748FF6368002B46
:10D1D000E6D023602046FFF7A5FF3468002CE1D19C
:10D1E000EFF3108372B60E4A00211068116003B984
:10D1F00062B628B18468FFF795FF20460028F9D170
:10D20000F8BD224600219847E0E783689847DDE7AC
:10D21000013B2360E4E700BF34A0FF1F9DB800007E
:10D2200044A0FF1F024A136801331360FFF7AEBF2B
:10D2300050A0FF1F704700BF0368F0B4FBB100258A
:10D2400001249D60DC601B4C1A601C44241104F115
:10D2500044056A11032692009E60174F0679174B0A
:10D2600047F8241002F1604202F5614205F01F0503
:10D27000012000FA05F5E6541560F0BC7047104C2B
:10D28000236843F40003236000BF0E4B0E4DA4F54A
:10D290008734A4F59E7401261E60234604609C68B2
:10D2A000002CD0D01033AB420360F8D100230360D0
:10D2B0001846E2E7008FFCBF4C92FF1F44E400E0F9
:10D2C0003C80044000700340407103400168A9B1F4
:10D2D0000B4BF0B40B441B110A4E0B4F0B4D46F891
:10D2E000237003F1440202F01F0401235211A340F2
:10D2F000002445F822308C600460F0BC704700BF09
:10D30000008FFCBF4C92FF1F35D2000080E100E08F
:10D31000024A034B012111601B6818470C7103403E
:10D320004C92FF1F024A034B012111605B681847B2
:10D330001C7103404C92FF1F024A034B01211160F4
:10D340009B6818472C7103404C92FF1F024A034B05
:10D3500001211160DB6818473C7103404C92FF1FAC
:10D36000F8B50E4671B17AB10746144600253B6800
:10D3700016F8011B1B6838469847013C0544F6D156
:10D380002846F8BD0846F8BD1046F8BD00B5064A67
:10D39000036812885B6883B001A9ADF804200222FB
:10D3A000984703B05DF804FB64490100F0B50746F7
:10D3B0008BB0002A33D0012A08BF0A2251B321249E
:10D3C00000E0F4B2B1FBF2F502FB1511C8B2092975
:10D3D00000F1300198BFC8B20AA988BF3730214494
:10D3E00088BFC0B201F8240C661E2946002DE8D182
:10D3F00033B1013CE4B20AAB23442D2203F8242CC0
:10D400003B6801AA11195B683846C4F122029847AB
:10D410000BB0F0BD30228DF825202124E8E7036809
:10D42000C9B21B6898470BB0F0BD00BF0029BABF56
:10D4300049422D2300230A22FFF7B8BF374A384953
:10D4400013681B06FCD40B6813F08003F8D172B686
:10D4500034490A78002A5FD0334A3448F0B4344C57
:10D46000176806682568D4680C303E44143200689A
:10D470001268304F35442C4420440244C2F34E021B
:10D480002D4E2E482E4D2F4C42F400423A60376804
:10D4900006682D682C4A24680C303E4400681268E7
:10D4A0002A4F35442C4420440244C2F34E02284EF5
:10D4B0002848294D294C42F400423A6037680668F2
:10D4C0002D68274A24680C303E4400681268254FB6
:10D4D00035442C4420440244C2F34E02224E2348D9
:10D4E000234D244C42F400423A60376806682D68A8
:10D4F000214A24680C303E440068126835442C44AC
:10D5000020440244C2F34E021C4842F4004202602E
:10D510000B7062B6F0BC704762B6704724B003402F
:10D5200024B00B4049A0FF1F38B003403CB003407B
:10D5300040B003402CB0034058B003405CB00340FF
:10D5400060B0034064B003406CB0034030B00340AF
:10D5500038B00B403CB00B4040B00B4044B00B40E7
:10D560004CB00B402CB00B4058B00B405CB00B40A3
:10D5700060B00B4064B00B406CB00B4030B00B405F
:10D5800030B42948294A2A4B2A4D6024E1210470ED
:10D5900011701B78284C082B30D00A2B27482849BB
:10D5A00037D00C2B0CBF35223D2212232A6023607A
:10D5B00002600B60234B24491B78244ABBB1012332
:10D5C0000B601360224B23491B78234A012B26D979
:10D5D000042B0FD9082B1ED9102B94BF8623872329
:10D5E0000B6013601D4B01221A7030BC70470B603A
:10D5F0001360E7E784230B601360F3E700F58E20E8
:10D600000F490830012213232A60236002600B6057
:10D61000D0E73922F7E785230B601360E2E7802328
:10D620000B601360DEE700BF004007400140074089
:10D630005C92FF1F08B003400CB0034008B00B40E1
:10D640000CB00B404CA0FF1F20B0034020B00B409B
:10D650005D92FF1F24B0034024B00B4049A0FF1F80
:10D660000C2830B417D91023984228BF18461C46FE
:10D67000104A114D1178181A8C42287018D00F4991
:10D6800013700B7823B10E490E4A00230B60136010
:10D6900030BCFFF775BF0A2802D90C231C46E7E708
:10D6A000082802D90A231C46E2E708231C46DFE7C4
:10D6B00030BC70475C92FF1F48A0FF1F49A0FF1FAE
:10D6C00024B0034024B00B4028282FD8334B2DE939
:10D6D000F0411E5CFF2E2BD0314B1B78002B2AD142
:10D6E00032062CD472B62F4D2F4C2F4601232660C4
:10D6F0002B7062B672B623681B060CD43B781BB93C
:10D70000F4E72B78002BF1D062B602F09BF972B6E9
:10D7100023681806F5D5254B1B6800222A7062B6CF
:10D72000234A107843FA00F0BDE8F08100207047EA
:10D730000020BDE8F081FFF781FE3206D2D572B637
:10D740001C4DDFF87C801C4C06F04007FFB206F051
:10D750003F06D8F80030DFB123F01003C8F80030DE
:10D7600001232660134A2B7062B672B6236819062D
:10D770000CD413781BB9ECE72B78002BE9D062B6F8
:10D7800002F060F972B623681B06F5D50B4BC3E7B0
:10D7900043F01003C8F80030E2E700BF6849010019
:10D7A00049A0FF1F4BA0FF1F00B0034010B0034073
:10D7B00048A0FF1F4AA0FF1F00B00B4010B00B4055
:10D7C0000CB00B400A4A0B49136843F480531360B2
:10D7D0000B7843B9084BC0221A70084B80F30C0039
:10D7E00000B218807047044B80221A70F5E700BF22
:10D7F0002C8004404CA0FF1F21C00C4000C00C40F6
:10D80000F0B51B4B1B4E596818689A68DB6885B0E9
:10D810006C460FC4337899071DD5174A174C1378F7
:10D82000174913F0700318BF1370164A164B802760
:10D83000177000263320032226706D4608701A7078
:10D8400072B6043C45F001052046A84762B623782D
:10D8500013F0700309D10D4B064901E0013B02D0E2
:10D860000A78D207FAD505B0F0BD237005B0F0BD37
:10D8700094490100010002400000024004000240FF
:10D880000B000240070002400A000240410D030065
:10D89000B0F5006F0AD210B5094B1B78DB070446C0
:10D8A00006D504F1A0500078C0B210BD002070472A
:10D8B000FFF7A6FF04F1A0500078C0B210BD00BF72
:10D8C00001000240B0F5006F17D238B50F4B1B783E
:10D8D000DA070D46044611D504F1A0500378AB4297
:10D8E0000AD00B4A137813F0700318BF1370074A5D
:10D8F00005701378DB07FCD538BD7047FFF780FF54
:10D9000004F1A0500378AB42EBD1F5E701000240EF
:10D910000000024008B5F4F7B7F9F5F783F802F014
:10D9200091F8FAE7844641EA000313F003036DD14E
:10D93000403A41D351F8043B40F8043B51F8043BD2
:10D9400040F8043B51F8043B40F8043B51F8043BD9
:10D9500040F8043B51F8043B40F8043B51F8043BC9
:10D9600040F8043B51F8043B40F8043B51F8043BB9
:10D9700040F8043B51F8043B40F8043B51F8043BA9
:10D9800040F8043B51F8043B40F8043B51F8043B99
:10D9900040F8043B51F8043B40F8043B51F8043B89
:10D9A00040F8043B51F8043B40F8043B51F8043B79
:10D9B00040F8043B403ABDD2303211D351F8043B19
:10D9C00040F8043B51F8043B40F8043B51F8043B59
:10D9D00040F8043B51F8043B40F8043B103AEDD2C8
:10D9E0000C3205D351F8043B40F8043B043AF9D219
:10D9F000043208D0D2071CBF11F8013B00F8013BEC
:10DA000001D30B8803806046704700BF082A13D3F8
:10DA10008B078DD010F003038AD0C3F10403D21A10
:10DA2000DB071CBF11F8013B00F8013B80D331F844
:10DA3000023B20F8023B7BE7043AD9D3013A11F8C4
:10DA4000013B00F8013BF9D20B7803704B7843702F
:10DA50008B7883706046704708B5104C08E02368E7
:10DA600059050DD423681A050FD42368DB0411D49B
:10DA700023685803F3D500F08DFE23685905F1D5CE
:10DA800002F044F823681A05EFD502F0D5F82368B0
:10DA9000DB04EDD500F0F0FCEAE700BF3480044081
:10DAA00008B5FFF7D9FF00BF014B10221A8070475D
:10DAB00000200540704700BF094908B50B6830B128
:10DAC0006A461844A2F58052904202D20860184675
:10DAD00008BD03F063FB0C2303604FF0FF3008BD6B
:10DAE0006092FF1FFEE700BFEFF3138070B9EFF302
:10DAF00010836BB9EFF305825AB94FF48070EFF3DE
:10DB000011832BB1984228BF184670474FF0FF3061
:10DB100070470F2A01D81846F1E7014BD05CEEE7B9
:10DB2000F0E300E0F0B44D1E2E46002400E0013486
:10DB3000B0FBF2F302FB1300092800F130078ABFA3
:10DB40003730F8B2C0B206F8010F1846002BEED1FC
:10DB50000A1953704CB1107815F8016F2870013311
:10DB6000E01A834202F80169F5DB0846F0BC704711
:10DB7000704700BF10B40F4B53F8302092F880422A
:10DB80002CB1012369B182F8803010BC704703EBDF
:10DB9000C0035B681A6841B922F002021A6010BC27
:10DBA000704782F8003110BC704742F003021A60DF
:10DBB00010BC7047A44901001C4A02EBC0030129B4
:10DBC0005B6811D004291BD052F83000002280F885
:10DBD000802229B1022920D0032922D01A6070475F
:10DBE0004FF480721A60704752F830004FF4A272FE
:10DBF00080F880121A601A6822F020021A607047BA
:10DC000052F830104FF4A272012081F880021A609D
:10DC10001A6842F020021A60704740F203121A603C
:10DC200070474FF481721A60704700BFA449010029
:10DC3000212848D8F8B5042A44D8DFE802F0484B38
:10DC40004E0345004FF410262B4B03EBC0030D464B
:10DC50005C68216811F4E06148D0284B284A2949C2
:10DC6000C3F89C2104F140422748C3F8A411A2F54F
:10DC70009221264FC3F8A0017C292548C3F8A8713A
:10DC8000C3F8AC012CD9A2F594237C2B2AD9A2F598
:10DC900096237C2B28D9A2F598237C2B29D9A2F591
:10DCA0009A227C2A27D81B4872B6236823F4702353
:10DCB00043F08072C4F384011643236040F821507E
:10DCC000266062B6F8BD70474FF43026BCE74FF4CB
:10DCD0000026B9E74FF44026B6E74FF42026B3E715
:10DCE0000D48E1E70D48DFE70D48DDE7FFF764FF8A
:10DCF000B3E70C48D8E7F8BDA44901000082FF1F34
:10DD0000F188FF1F9988FF1FC588FF1F6D88FF1FBF
:10DD10004188FF1F3C93FF1F6492FF1F9C92FF1FCF
:10DD2000EC92FF1F1C93FF1F1A4B03EBC00010B4B3
:10DD3000426802F14043A3F592217C2923D9A3F53F
:10DD400094217C290DD9A3F596217C291FD9A3F50F
:10DD500098217C2919D9A3F59A237C2B11D80E4C34
:10DD600000E00E4C72B613680D4823F08773C2F3BF
:10DD7000840123F4803343F08073136044F821005E
:10DD800062B610BC7047074CECE7074CEAE7074C5B
:10DD9000E8E700BFA44901003C93FF1F9C92FF1FCE
:10DDA00071DB00006492FF1F1C93FF1FEC92FF1FAA
:10DDB00030B4054B054D064C002210211A602A6034
:10DDC0002060196030BC704714D0034004D0034079
:10DDD00000D00340282838B52ED0002904464FDD56
:10DDE0005F4B1B78012505FA03F28A4202D82128ED
:10DDF00037D938BD0338C2B2012A3AD9202C4AD0CB
:10DE0000192C48D0574A126802FB011222FA03F378
:10DE10001D2800F29B80DFE800F0928B847D9999A9
:10DE2000766F99999999999999999968615A53999D
:10DE30004C99999999999945494B1B780B2B08D97D
:10DE40000C2B1CBF0C3B19410846BDE83840FFF7BE
:10DE5000B9BCC3F10C0399400846BDE83840FFF750
:10DE6000B1BC2946FFF786FE2946BDE83840FFF7DA
:10DE7000A3BE3D4A126802FB011222FA03F3C7E770
:10DE80002128B6D80021FFF775FE20460121BDE804
:10DE90003840FFF791BE354A126802FB011222FAA0
:10DEA00003F3B5E73249334A0B604FF45173136003
:10DEB00038BD3149314A0B604FF45173136038BD9E
:10DEC0002F49304A0B6040F24443136038BD2E495D
:10DED0002E4A0B6040F24443136038BD2C492D4A52
:10DEE0000B6040F24443136038BD2B492B4A0B6052
:10DEF00040F24443136038BD29492A4A0B6040F27E
:10DF00004443136038BD2849284A0B6040F244431B
:10DF1000136038BD2649274A0B6040F24443136022
:10DF200038BD2549254A0B6040F24443136038BD93
:10DF30002349244A0B604FF45173136038BD2249C2
:10DF4000224A0B604FF45173136038BD212C3FF609
:10DF500050AF7F29D4BF00210121204693E700BFA5
:10DF60004493FF1F088003400890034008800B4043
:10DF700010800B4048A0044018800B404CA0044087
:10DF80001880034008B004401080034004B00440EF
:10DF90004080034018C004403880034014C004404F
:10DFA0002880034010B00440208003400CB004409F
:10DFB0003080034010C00440488003401CC004402F
:10DFC0001890034034900440109003403090044077
:10DFD00038B1102828BF1020044AC3B2107813703B
:10DFE0007047024A01231078137070474493FF1F53
:10DFF0002DE9F8430E4680463249334D304603F052
:10E0000053F847F6122300281ABF1D464FF00209A5
:10E010004FF00109002425FA04F002F04FFE4FF002
:10E020005E51074602F0A2FE0146304603F050F86A
:10E0300030B90134072CEED1E80902F03FFE074663
:10E040003146384602F046FF4FF07C5102F084FD25
:10E0500003F078F84FF6FF729042A8F1030328BF4F
:10E060001046012B29D9B8F1170F17D8174B23FAEF
:10E0700008F303F0010383F0010223B9B8F1190F8B
:10E080000FD0BDE8F883124B124D13491A6044EAD1
:10E09000C9042A6008601C60BDE8F883B8F1200F4D
:10E0A000ECD10E4B0E4D0F49002244EAC9041A6010
:10E0B0002A6008601C60BDE8F8830B4B0B4D0C49CF
:10E0C000F2E700BF001BB740006CDC026006F00006
:10E0D00000800340048003400880034000800B4020
:10E0E00004800B4008800B400090034004900340E4
:10E0F00008900340212801D8FFF73CBD704700BFBE
:10E10000212806D8044B53F8303093F80002C0B2EF
:10E1100070470020704700BFA4490100212801D8A2
:10E12000FFF74ABD704700BF72B60C490C4B0D4A51
:10E130001B680868126862B6520102D5322B88BF8C
:10E1400001300949C3F5BB334FF47A72FF33A1FBA9
:10E15000031302FB00F000EB9310704750A0FF1F69
:10E1600018E000E004ED00E0ABAAAAAA2DE9F8430C
:10E17000054672B6204F214B214A1B683C68126845
:10E1800062B6520102D5322B88BF013495B3C3F574
:10E19000BB331C4EDFF86490DFF86480FF334FF42C
:10E1A0007A72A6FB031302FB04F404EB931472B619
:10E1B000D9F800103A68D8F800E062B6C1F5BB3370
:10E1C000FF33A6FB03031EF0806FC4EB93134FF4E1
:10E1D0007A7002D0322988BF013200FB0233B3F5D6
:10E1E0007A7F04D3013D05D004F57A74DFE701F0AE
:10E1F00029FCDCE7BDE8F88350A0FF1F18E000E031
:10E2000004ED00E0ABAAAAAAF8B52D4B2D49DFF822
:10E21000D0E0DFF8D0C02C4E2C4D2D4C2D4A2E4F87
:10E220004FF4000018604FF0807018604FF00070DD
:10E2300018604FF0806018604FF000601860002098
:10E24000086028234BF6FF71CCF80010CEF80030A0
:10E25000336013602B6023603B60B36293620922DA
:10E2600045F8242CC4F8D80F05F57F65C7F8D41FEE
:10E2700007F5FF2707F5FA67C6F8F83F2B6006F5A4
:10E28000FF26C4F8D42F05F5FD2504F5FF243860DA
:10E2900006F2F4761148316005F5FF6504F5FD647A
:10E2A0002B6023600260FFF76BF91920FFF75EFF18
:10E2B00000F0B6FF40F21310BDE8F840FFF756BF7C
:10E2C00008E100E004800340148003402480034000
:10E2D0002C8003401C8003403480034000800B40AE
:10E2E0000C800340088003402DE9F84F214B1B6848
:10E2F00007460BB101221A70DFF888901E4D99F87D
:10E300000040DFF884801D4E0134272C8ABF4FF077
:10E31000000A5FFA84FA5446AB462B78A34216D122
:10E32000FFF7E2FB40281FDC33791B06F5D59BF88D
:10E3300000300133272B86BF00221346DAB218F8CB
:10E340000330DBB2F3712A702B78A342E8D00C497A
:10E350000A4BFFB208F804700120AC22087089F85B
:10E3600000A0DA70BDE8F88FFF28D6DD01F06AFB67
:10E37000D3E700BFC8A0FF1FC5A0FF1F00C0064015
:10E38000C4A0FF1FCCA0FF1F5CA0FF1F1C4BDFF829
:10E3900094C01A681B49F0B542F480521A4D1A60B5
:10E3A000DFF884E0194F1A4E1A4C00238CF8003025
:10E3B0004FF451722B701F2840F213358EF8003045
:10E3C0003B70337025600A6012D819460124124A46
:10E3D000124D11701248547000212C274026937260
:10E3E0004FF4003491701174D7702E700460F0BD3A
:10E3F000C0F34431C0F3471400F01F03E7E700BF48
:10E40000348004400CC0044059A0FF1FC5A0FF1F6A
:10E41000C4A0FF1F08C0044000C0064031E400E073
:10E4200004E100E058A0FF1FCCA0FF1F034B1B68B6
:10E43000DB0401D5FFF758BF704700BF34800440AC
:10E4400010B5044C237823B101F0FCFA2378002B9B
:10E45000FAD110BDC4A0FF1F054A064B10781B78E7
:10E46000C0B2DBB2984238BF4030C01A704700BF1C
:10E4700058A0FF1F59A0FF1F30B42B4B1A799406E8
:10E480001FD52A48DA790378294901333F2B0978C7
:10E49000C8BF00238B42D2B203D0264CD9B2E2547B
:10E4A0000170254A116861B1244A1278D2B29342B0
:10E4B00036BFC2F140029B1A9B18272BC4BF012311
:10E4C0000B70194AD378DBB2180611D45A060DD551
:10E4D000154B1B795B0609D5194B1A491B6800229D
:10E4E0000A7003B11A70104B2C22DA7030BC7047DE
:10E4F00011790906EAD5144910480C780178C9B297
:10E500008C420DD04A1C272A84BF00210A460F4D99
:10E51000054C98BFD1B2AA5CD2B2E2710170D5E7C6
:10E520006C21D170D2E700BF00C0064058A0FF1F89
:10E5300059A0FF1F84A0FF1F54A0FF1FC5A0FF1FED
:10E54000C8A0FF1FC4A0FF1FCCA0FF1F5CA0FF1F1F
:10E5500021282FD8184B195CFF292BD0174B184AAC
:10E56000DFF870C003EBC000F0B54368DFF868E087
:10E57000144F154D154E00241C60DEF800300120AC
:10E5800043F020038840CEF8003014604FF4A073AD
:10E5900038602E60C2F800C0013BFDD113689B05B6
:10E5A000FCD42023013BFDD1094B09B233F8110003
:10E5B00080B2F0BD00207047B44A0100A4490100B8
:10E5C000005004400850044004500440000002037E
:10E5D0000051044080014A0038800440431E032B50
:10E5E00014D872B60A4951F8230068B170B4094CC6
:10E5F000058834F81320466841F82360521B24F83C
:10E60000132062B670BC704762B670470020704736
:10E6100028A1FF1F6CA3FF1F013803280BD872B677
:10E62000074B53F8203043B100205B680130002BCA
:10E63000FBD162B67047002070471846F9E700BF6B
:10E640007CA1FF1F30B472B62B4A13781D0706D584
:10E650002A4B196A002936D0996A002941D053788B
:10E660001C0706D5254B196C00293ED0996C002952
:10E6700039D09378190705D5204B196E002936D06B
:10E68000996E89B1D3781B0707D51C4BD3F880202E
:10E690007AB3D3F8882011213AB162B6184B002220
:10E6A0001A7030BC00F04ABE0D21154C154D227871
:10E6B00043F8315003EBC1030830013A586022702F
:10E6C00062B630BC704704220D4C0F4D217843F8E0
:10E6D000325003EBC20308304A1E5860227062B603
:10E6E000EFE70521E1E70921DFE70822ECE70C224B
:10E6F000EAE71022E8E700BFD84A01000080FF1FC8
:10E70000A5A1FF1FC800400088004000431E032B46
:10E710001DD81B4A400140F0100030B4104472B6BE
:10E72000184CE25C032A1BD8DFE802F0021215172E
:10E7300003220D88E25410F0080F14BFC823882369
:10E7400043EA054308310360416062B630BC70475C
:10E7500008300222EDE70522EBE708300422E8E763
:10E76000094A52F8230038B1084A52F823004160A0
:10E7700042F8231062B6E9E742F82310034AF7E7AC
:10E780000080FF1FB4A1FF1F7CA1FF1F8CA1FF1FF2
:10E7900000BE70472DE9F04FDFF818B3DFF818A37B
:10E7A00087B044E0AD4F4FEA930807EBC809013E3C
:10E7B000D9F8042003F00803F6B2A2F1080003F030
:10E7C000FF04002B40F0018157F838301B0C99B240
:10E7D00022F8081C002B00F0EF80A14B22F8064C19
:10E7E00042F8044C53F82620002A00F0CF819D4DBA
:10E7F00055F8263058609C4C45F8260034F8163001
:10E80000194424F8161000F079FD002800F0C281A8
:10E81000964A974B19F0080F00F1080018BF1346ED
:10E82000C9F8040047F8383008238BF800309BF80B
:10E830000040E4B265071CD58E4B1B78B3B18E49FE
:10E840000A7802F0FF0322B1013BDBB20B7003B97F
:10E8500000BE8A490A7802F0FF032AB1013BDBB20D
:10E860000B70002B00F0688100F066FE04238BF82B
:10E87000003004F0080303F0FF02002B00F0C98011
:10E880009AF80030DBB21E098CD19A08DFF8CC91DF
:10E8900059F8321009EBC200C1F383010139406815
:10E8A0000C2900F28580DFE801F07A7A8383838384
:10E8B00083834683838307000168714D4068714FED
:10E8C000714E6860296088B240F281610024674B14
:10E8D00049F832304FF0010E88423C60C9F81040D0
:10E8E000C9F8184086F800E05C4A00F2E780B0F50D
:10E8F000D06F80F01B82B0F5817F00F0D98100F2EB
:10E900006981802800F02A82822840F0D781A98876
:10E9100001F07F01042900F2D1815C485C4A890042
:10E9200008441470547001788C0740F1608382F8B9
:10E9300000E0022173E1534F3A682AB3554B524E1F
:10E94000554819883478057840298E4645F00208E4
:10E9500028BF4FF0400E002C84F001043470CEEB41
:10E9600001010CBF8824C82409EBC80689B285F0D0
:10E97000010544EA0E447260198049F83840724437
:10E980000570002965D03A603D4B1A88B2F5A06F3A
:10E990000ED100219A785970404B1A7008E038491E
:10E9A0003F4C0D68A54200F09880304949F832107C
:10E9B0003C4A0123137037E72C4A2D4B19F0080FFE
:10E9C00018BF134647F838302EE700F0B7FC364A38
:10E9D000364952F82630002B00F0E38058688C5DF1
:10E9E00042F8260003F10802C9F80420032C05D8D8
:10E9F000DFE804F02C02292602228A551A8819F031
:10EA0000080F0CBF8823C82343EA024347F8383075
:10EA10000AE7E00700F19380210600F1D180A20708
:10EA200006D5234A234913780220DBB213700870FD
:10EA3000E30602D51F4B10221A7007B0BDE8F08F15
:10EA400004228A55DAE705228A55D7E703228A5538
:10EA5000D4E7BEF1400F18BF002294E70080FF1FEB
:10EA600028A1FF1FD4A0FF1F6CA3FF1FC8004000F8
:10EA700088004000B0A1FF1F39A1FF1F24A2FF1F83
:10EA80009CA1FF1FD0A0FF1F38A1FF1FC02007407F
:10EA9000A8A1FF1FE4A0FF1FA4A1FF1F982007400B
:10EAA00021090003942007407CA1FF1FB4A1FF1F90
:10EAB000882007408020074090200740B0F5106F65
:10EAC00000F07C8140F2A38040F62112904240F099
:10EAD0007B82A54A012313706AE74C68A3498C42E4
:10EAE0007FF463AF0178A9297FF45FAF41784529AE
:10EAF0007FF45BAF8178C2297FF457AFC1786B296F
:10EB00007FF453AF9A489B4E0178347881F0010529
:10EB1000002C41F0020105700CBF8820C82084F051
:10EB2000010449F8310009EBC10193483470002514
:10EB300005244D60047038E700F064FF94E68F4BC5
:10EB400089488B491A614FF0020E80F800E08C4F23
:10EB50000A708C49196099608B4E8C4D8C4C9A616F
:10EB60000D213970FF213170DFF84CE229702270DD
:10EB7000884D894A8EF800109F27012406F8047CEE
:10EB80005D600470DA6007B0BDE8F08F43F82600DE
:10EB9000824D30E6824A47F838001378013313700B
:10EBA00042E68B5D032B00F2BA8001A252F823F0FB
:10EBB00029E8000029E8000009EC000003EC00004F
:10EBC0006F49724B80220D2008701A70A2077FF5E2
:10EBD0002FAF26E740F20232904240F0ED81AA8842
:10EBE00002F07F02042A69D86D88002D66D164493D
:10EBF000CDF804E0920011440A7842F002020A7053
:10EC0000C1E101238B550FE600238B550CE6B0F5CF
:10EC1000086F53D16349644A097811707146ED88D1
:10EC20008D4280F0E88252480478402DAE4644F090
:10EC3000020C28BF4FF0400E02EB0E0309EBCC0193
:10EC4000029301234A604FEA0E48CEEB050101937F
:10EC50000025C82242EA080384F0010249F83C304A
:10EC600035700270DFF814C1424BDFF8048149BBF4
:10EC7000BEF1400F7FF42DAF42F0020C09EBCC0344
:10EC8000029ADFF8F8E05A608DBB0D0445F0880564
:10EC90009DF804304EF83C500A443370047013461B
:10ECA00040297FF416AF0021404A3B60118010E7F5
:10ECB000AA8802F07F02042A40F28B81304A0F2397
:10ECC000137006E74029D7D942F002020CEBC200CC
:10ECD000029E4660BDB19DF8045035481D70334614
:10ECE000403988F8004040334CF83200DCE79DF8AA
:10ECF000043033700D04029B047045F0C8050B44CA
:10ED00004EF83C50CCE79DF804501D70029B1D4806
:10ED100088F80040403940334CF83200C4E719F01D
:10ED2000080F0CBF022303238B557DE521494A6858
:10ED3000002AC3D06C88B5F804E003E00C314A68BF
:10ED4000002ABBD00B88A342F8D14B887345F5D17C
:10ED5000240A032C0CBF1178098960E7124A0221AA
:10ED6000147054705BE700BF94200740010004005A
:10ED7000A4A1FF1F38A1FF1F39A1FF1F0080FF1FA3
:10ED8000C0200740880040008820074080200740BE
:10ED900098200740E8A0FF1F3CA1FF1FD4A0FF1F41
:10EDA000A5A1FF1FB0A1FF1FA8A1FF1FE4A0FF1F87
:10EDB000C8004000DC4A01008C200740B248116ABC
:10EDC000AC7804700C0600F19881D9F82820AF497E
:10EDD000100600F1DB81D9F83020AC49120600F1B1
:10EDE000D081D9F83820A949130600F1C581D9F896
:10EDF0004020A649150600F1BA81D9F84820A34958
:10EE0000140600F1AF81D9F85020A049100600F196
:10EE1000A481D9F858209D49120600F19981D9F8AA
:10EE200060209A49130600F18E81D9F8682097492D
:10EE3000150600F18381D9F870209449140600F179
:10EE40007881D9F878209149100600F16D81D9F8C0
:10EE500080208E49120600F16181D9F888208B4903
:10EE6000130600F15581D9F890208849150600F164
:10EE70004981D9F898208549140600F1FF8084481B
:10EE8000844A854901908548854D864C0497002326
:10EE90000596029580460F4616461D460394306837
:10EEA00028B1446800F04AFA2046002CF9D100232A
:10EEB0003360029B38681A46002342F8253028B197
:10EEC000446800F03BFA2046002CF9D100223A6059
:10EED000019A98F800301146002241F8042B039A59
:10EEE0000191023B4FF0000122F81510032B07D8C7
:10EEF000DFE803F05D025D024FF0010388F80030A7
:10EF00000135042D06F1040607F1040708F1010894
:10EF1000C5D1654C654D2278654B049F059E002147
:10EF2000100729701A7000F19280624962780A70A5
:10EF30000021C9F83010C9F838101107DFF84C81EA
:10EF40006ED4A2785C49DFF844810A700021120770
:10EF5000C9F85010C9F858104BD4E27857494B4CB7
:10EF60000A7013074FF00001C9F87010C9F8781043
:10EF700000F1AE8033780193002283F00105C9F8D7
:10EF80009020C9F898200021029188468E460A46B2
:10EF90004B48047844F0020C09EBCC030393019B2B
:10EFA000002B039B5A600CBF8822C82252E64FF008
:10EFB000000388F80030A3E7B0F5A06F7FF47EAEC1
:10EFC000012300250193DEE740F621229042F7D08D
:10EFD00074E66D88002D7FF471AE3A49CDF804E0F7
:10EFE000920011440A7822F002020A70CBE7022153
:10EFF00015E600F083F9002800F0EB800830324A73
:10F00000C8F86400C8F8602000F078F9002800F023
:10F01000DA8008302D4AC9F86C00C9F868209CE7EE
:10F0200000F06CF9002800F0E0800830264AC8F8AB
:10F030004400C8F8402000F061F9002800F0CF80BB
:10F040000830224AC9F84C00C9F8482079E700F096
:10F0500055F9002800F0A58008301B4AC9F82400A3
:10F06000C9F8202000F04AF9002800F09480083008
:10F07000164AC9F82C00C9F8282056E7D1F89C0098
:10F08000083800F05BF9FAE6B0A1FF1F0080FF1F0F
:10F090008CA1FF1F28A1FF1F7CA1FF1FB4A1FF1F90
:10F0A000D4A0FF1F6CA3FF1FD84A0100A5A1FF1F1A
:10F0B000C4200740C8200740CC200740D02007408C
:10F0C000A4A1FF1FC020074088004000C8004000E6
:10F0D00000F014F9002870D008304F4AC4F88400BA
:10F0E000C4F8802000F00AF9002860D008304B4AAC
:10F0F000C9F88C00C9F888203CE7506A083800F04D
:10F100001DF962E6D1F89400083800F017F9B0E66E
:10F11000D1F88C00083800F011F9A4E6D1F8840089
:10F12000083800F00BF998E6C86F083800F006F9C7
:10F130008DE6486F083800F001F982E6C86E08389D
:10F1400000F0FCF877E6486E083800F0F7F86CE657
:10F15000C86D083800F0F2F861E6486D083800F034
:10F16000EDF856E6C86C083800F0E8F84BE6486C55
:10F17000083800F0E3F840E6C86B083800F0DEF825
:10F1800035E6486B083800F0D9F82AE6C86A08382E
:10F1900000F0D4F81FE62A78C9F8280001322A7056
:10F1A000C3E62A78C9F8200001322A705AE72A7883
:10F1B000C9F8880001322A70DCE62A78C4F8800099
:10F1C00001322A708EE72A78C9F8680001322A7065
:10F1D000C3E62A78C8F8600001322A7014E72A785A
:10F1E000C9F8480001322A70ABE62A78C8F8400016
:10F1F00001322A701FE740298E4628BF4FF0400E8B
:10F2000002EB0E0302930123CEEB01014FEA0E48FD
:10F2100000250193BCE600BF88004000C800400004
:10F22000F8B500F08FFD294B29482A4C2A4F2B4D69
:10F23000DFF8BCC0DFF8BCE0294E00221A605A603B
:10F240009A60DA601A615A619A61DA611A625A62E6
:10F250009A62DA621A635A639A63DA631A645A64C6
:10F260009A64DA641A655A659A65DA651A665A66A6
:10F270009A66DA661A675A679A67DA67C3F880206F
:10F280000168C3F8842041F480210160C3F30721A1
:10F290002170C3F30740134938701B0E2B70FF23F6
:10F2A0008CF80030104D8EF8003010480B700123A0
:10F2B000337084F8642070264FF40074102207F82D
:10F2C0002C3C2E70046081F8F820F8BD0080FF1FF0
:10F2D000348004409C200740B0200740B420074001
:10F2E000942007401020074049E400E008E100E0D6
:10F2F0008020074088200740704700BF72B60D4845
:10F300000268B2FA82F30F2B10DC4FF00041D940B3
:10F3100022EA0102026062B6074803EBC303DB0086
:10F32000C2180021C15010465160704762B60020DB
:10F33000704700BF4893FF1FBC83FF1F0D4B0E4A51
:10F34000C31AA2FB03231B090F2B0CD80B4A1278FC
:10F3500052B972B60A484FF00041026821FA03F32D
:10F360001A43026062B67047064A1278002AF0D04B
:10F37000FFF768B9BC83FF1F398EE338A5A1FF1FD3
:10F380004893FF1FB0A1FF1F38B50E4B0E4C1B68F2
:10F39000218805468BB1B1F5917F05D20B4A4B1CF4
:10F3A00055549BB2238038BD00220848984700215D
:10F3B000064A55540123238038BDB1F5917FEDD322
:10F3C00038BD00BFDCA1FF1F76A3FF1F7CA3FF1F7A
:10F3D0002DE9F843214E224F3168012380463B70CE
:10F3E000B1B1204D4B8801EB8302013300240F2B78
:10F3F000C2F808802C7004D84B8000233B70BDE815
:10F40000F88340230B800320FFF780F93460F4E792
:10F41000DFF8549099F80030002BF0D0114D45F6EC
:10F42000215408E0013C12D02B7883B900F00AFB8C
:10F4300099F800307BB10320FFF7EEF80528F1D8EA
:10F44000FFF75CFF014630600028EBD0CAE70123DC
:10F450002B70BDE8F883BDE8F88300BFF8A1FF1F5B
:10F46000CCA1FF1FFCA1FF1FB0A1FF1F1201F8B527
:10F47000D5B2A1B3012943D04378044600781B06D6
:10F4800043EA004040F4704045F004068F1E3043CC
:10F49000FFF79EFF022F04F1020314D9053414F87C
:10F4A000023C14F8032C14F8010C1B0443EA022359
:10F4B000334343EA0060033FFFF78AFF022F2346EE
:10F4C00004F10304EBD8022F23D0012F0DD045F413
:10F4D000774040F00500BDE8F840FFF779BF1448D9
:10F4E0002843BDE8F840FFF773BF187845F4770567
:10F4F00045F0060545EA0020BDE8F840FFF768BF83
:10F5000003780C4845EA03452843BDE8F840FFF777
:10F510005FBF1A78587845F0774545F0070545EA0A
:10F52000022545EA0040BDE8F840FFF751BF00BFA3
:10F5300006F0F70007F000F738B5084B1C7824B93F
:10F54000074D296809B14B8803B938BD9B000B8072
:10F550000320FFF7DBF82C6038BD00BFCCA1FF1FF4
:10F56000F8A1FF1F2DE9F041AD4E33680746002B8F
:10F5700000F092801D885A88910803EB81010432C3
:10F58000AA428C6842D25A8004F00F064FEA14282F
:10F59000A449A6F1080208F00F00C4F30313062AD9
:10F5A00000F101050B701AD9B31E012B5FFA88F028
:10F5B0004ED9052E48D0042E00F0A481731F022BD3
:10F5C0007FD90F2E0ED1F72842D8F02802D0964BC3
:10F5D0001B883BB1FFF7D8FE0020BDE8F08127B1C2
:10F5E000BD4202D00020BDE8F081082EC4F30333F1
:10F5F00000F08780092E11D00A2E40F094800A2B4B
:10F60000F0D18A4B8A4A1B68A02181E01846FFF797
:10F6100095FE0420FEF7E2FF3060B5E7092BE1D14B
:10F62000270E00F07B81834B814A1B689021C4F335
:10F6300007461170EDB2FCB2002B00F09D8022460F
:10F6400031462846984797E0F02843D9F72841D01B
:10F65000F1380E28C6D801A353F820F013F80000A3
:10F66000F7F70000E5F70000E5F50000E5F500001C
:10F67000D7F70000E5F50000B7F80000E5F5000059
:10F6800081F800009BF80000BFF70000E5F50000DE
:10F69000A7F700008BF70000674B1B78002BA1D069
:10F6A0000420FEF79BFF0346306000289AD00588AF
:10F6B000002D7FF460AFFFF741FE35602846BDE8BE
:10F6C000F081FFF761FEC4F30740FFF75DFE072EF0
:10F6D00002D1200EFFF758FE534B584A198858485C
:10F6E0001468584D524A017000270E0AF0201F80FE
:10F6F0002E7010700CB301225348A0470120BDE8C2
:10F70000F081082B7FF46EAF504B494A1B68802173
:10F71000C4F307461170EDB2240E6BB3284622469F
:10F720003146984728E00B2E11D10B2B7FF45AAFAE
:10F73000474B3F4A1B68B021EAE7464B1B68002B4A
:10F7400000F0FB80404898470120BDE8F0810C2E76
:10F7500040F000810C2B7FF445AF3F4B344A1B68CF
:10F76000C0211170EDB2C4F30746002B00F0C88031
:10F7700028463146240E98473849314A314B0D709E
:10F7800016701C700120BDE8F081354B1B68002B02
:10F7900000F0D6809847C4F30746254BEDB2240EFF
:10F7A00083F80080E8E72F4B1B68002BF2D12E4B2B
:10F7B0001B68A3B1FE209847C4F30746EDE72B4B27
:10F7C0001B68002BE6D1284B1B6843B1FC209847EF
:10F7D000C4F30746E1E7264B1B68002BDAD1C4F3DC
:10F7E0000746DAE7234B1B68C4F30746002BD4D047
:10F7F00030469847D1E7204B1A68002AEFD0260CF4
:10F80000630C06F07F0003F47E531843F6B2904772
:10F81000C3E71A4B1B68C4F30746002BE8D1BCE7CB
:10F8200004A2FF1F7AA3FF1F76A3FF1FE0A1FF1F03
:10F8300074A3FF1F14A2FF1FB0A1FF1FDCA1FF1FB5
:10F8400078A3FF1F79A3FF1F7CA3FF1F0CA2FF1F3C
:10F8500010A2FF1FF4A1FF1FD0A1FF1F7BA3FF1F5A
:10F86000BCA1FF1FC0A1FF1FC4A1FF1F00A2FF1F5B
:10F87000F0A1FF1F08A2FF1FD8A1FF1FECA1FF1FCF
:10F880003F4B1B68002B85D13E4B1B68002BA6D03D
:10F89000FA209847C4F307467FE73B4B1B68002BD1
:10F8A0007FF478AF374B1B68002B98D0FB2098472C
:10F8B000C4F3074671E7354B1B68002B7FF46AAF32
:10F8C000304B1B68002B8AD0F8209847C4F30746BA
:10F8D00063E70E2B7FF486AE2D4A2E4B1268E02193
:10F8E0001970002A47D0260C610C06F07F0301F442
:10F8F0007E511943EDB2A1F5005128469047F6B26A
:10F90000240E39E7FFF740FDC4F30740FFF73CFD45
:10F91000200EFFF739FD0020BDE8F0811E4B1D4A87
:10F920001B6880211170EDB2C4F3074683B13146E4
:10F9300028463A4698473C461EE70120BDE8F0813C
:10F94000104B1B68002B3FF44AAFFF20984746E757
:10F950001C4611E70D2EBCD10D2B7FF443AE0F4B8F
:10F960000C4A1B68D0211170EDB2C4F30746002B7E
:10F970007FF4FEAEC4E7C4F30746EDB2240EFBE607
:10F98000E8A1FF1FC4A1FF1FC8A1FF1FB8A1FF1F4F
:10F99000D4A1FF1F74A3FF1F0CA2FF1FE4A1FF1F30
:10F9A00038B5164D2868E0B101884488A14213DDBE
:10F9B00003191B7A83B104F10803C2180C1B00233E
:10F9C00002E012F8011F21B10133A342F9D1204610
:10F9D00038BD1C46204638BDFFF7B0FC002028602B
:10F9E00038BD074B1B780BB9002038BD0220FEF74D
:10F9F000F5FD28600028D7D1F6E700BF20A2FF1F41
:10FA0000B0A1FF1F0D4B1B78BBB910B50C4C216882
:10FA100003F0FF024B883F2B07DC07330B4401F157
:10FA2000470003F8012F8342FBD140230B800120C4
:10FA3000FEF76CFE0023236010BD704718A2FF1F65
:10FA40001CA2FF1F38B5224C237803B138BD012317
:10FA50002370FFF7A5FF70BB00F048F840BB00F033
:10FA6000DBF810BBFEF7F8FCE0B900232370EFF3DE
:10FA70000583002BEAD1EFF3108172B6154B18689D
:10FA8000E0B1154C2278CAB945691D600123237085
:10FA9000C5B1AA6101B962B6002545778368984768
:10FAA0002570D3E700F020F8DFE700F01BF8D9E776
:10FAB00000F016F8D3E7FFF71FFCCDE70029C5D10A
:10FAC00062B638BD054B1D600029E5D1E3E700BFF4
:10FAD00025A2FF1F3CA0FF1F40A0FF1F38A0FF1F53
:10FAE000704700BF704700BF704700BF054A064B14
:10FAF00010781B78C0B2DBB2984238BF4030C01AD1
:10FB0000704700BF2CA2FF1F2DA2FF1FF0B4384B7F
:10FB10001A7912F0300F2CD072B6997D01F0FF02E5
:10FB200000293DD062B6334F334938780D78334ED3
:10FB30001C46C0B2EDB2431C402BE17928BF002324
:10FB4000AB4202F1FF32C9B21CBFF154184612F0A9
:10FB5000FF02F0D12A4B1B68C2B23A704BB1A842E7
:10FB600036BFC5F14005401B40192728C4BF0122FC
:10FB70001A701F49CA78D2B2150616D452060DD58E
:10FB80001B4B1B795B0609D51E4B1F491B680022C6
:10FB90000A7003B11A70164B3C22DA70F0BC704741
:10FBA0004022D9795A7462B6E3E70B791C06E5D591
:10FBB000164B174E1C783378E4B2DBB29C420ED061
:10FBC000144D01E0A3420AD00133402B28BF00238B
:10FBD0000879E85CC0B2C871087D0728F2D9DBB2A9
:10FBE000034933700B79180644BF7C23CB70C5E7FB
:10FBF00000A006402CA2FF1F2DA2FF1F70A2FF1F16
:10FC000028A2FF1FB4A2FF1FB0A2FF1FB8A2FF1FB0
:10FC1000B1A2FF1F30A2FF1F054A064B10781B78C8
:10FC2000C0B2DBB2984238BF4030C01A704700BF44
:10FC30002CA3FF1FC1A2FF1FF0B4384B1A7912F09A
:10FC4000300F2CD072B6997D01F0FF0200293DD013
:10FC500062B6334F334938780D78334E1C46C0B204
:10FC6000EDB2431C402BE17928BF0023AB4202F1E7
:10FC7000FF32C9B21CBFF154184612F0FF02F0D196
:10FC80002A4B1B68C2B23A704BB1A84236BFC5F1CD
:10FC90004005401B40192728C4BF01221A701F4984
:10FCA000CA78D2B2150616D452060DD51B4B1B7955
:10FCB0005B0609D51E4B1F491B6800220A7003B161
:10FCC0001A70164B3C22DA70F0BC70474022D9798A
:10FCD0005A7462B6E3E70B791C06E5D5164B174E4E
:10FCE0001C783378E4B2DBB29C420ED0144D01E0B4
:10FCF000A3420AD00133282B28BF00230879E85CEF
:10FD0000C0B2C871087D0728F2D9DBB2034933704D
:10FD10000B79180644BF7C23CB70C5E700B00640C2
:10FD20002CA3FF1FC1A2FF1FECA2FF1FBCA2FF1F3D
:10FD300030A3FF1FC0A2FF1F34A3FF1F2DA3FF1F6F
:10FD4000C4A2FF1F70B584B072B6194B194D1A4882
:10FD5000702241260F2480211A702E701A460470DA
:10FD6000197013781B06FCD5144B186862B6144B37
:10FD7000144C984298BF00EB800001A998BF400046
:10FD80000A22FDF7CFFE01A92046002311F8012B1E
:10FD900001333AB10A2B20F8022FF7D11623237032
:10FDA00004B070BD5B00DBB2237004B070BD00BF57
:10FDB0000000024007000240060002400800024026
:10FDC0007F9698001494FF1F2DE9F043DFF8EC8034
:10FDD0008BB006460F4600F073F898F900300133F7
:10FDE00004460D4637D03046394600F0DFF900288A
:10FDF00031D02BA3D3E900233046394600F026FE4C
:10FE0000814668BB28A3D3E900233046394600F079
:10FE1000FFFD00B398F90030254ACDF82090042466
:10FE200000200021022BCDE90467CDE90267009490
:10FE30000192CDE906012CD0684600F0BDF940B32F
:10FE4000089B1BB101F0AAF9089B0360DDE90601DC
:10FE50000BB0BDE8F083204629460BB0BDE8F08327
:10FE6000134A98F90030019203210022CDE904677A
:10FE7000CDE90267009108922BB90E4B4FF060421A
:10FE8000CDE90623D8E70C490020022BCDE9060175
:10FE9000D2D101F083F922230360D1E7AFF30080D0
:10FEA000EF39FAFE422E864051302DD5104987C0D9
:10FEB000484B0100FFFFEF470000F07F2A94FF1F2F
:10FEC0002DE9F04FB04F21F00042BA4283B00C460A
:10FED0004FEAD17605460DD9AC4FBA4225D9C1F3C8
:10FEE0001303034340F0EF800EB10020014603B03E
:10FEF000BDE8F08FA64B9A4200F2CC80A54B9A4207
:10FF000000F2DE808AA3D3E9002300F05DF900222D
:10FF1000A14B00F09BFD002800F0058128462146FA
:10FF200000229D4B00F050F9E1E783A3D3E90023C1
:10FF300000F08CFD002840F0CB802846214680A3AD
:10FF4000D3E9002300F064FD0028CED1934B28466E
:10FF500003EBC60821467CA3D3E9002300F0E6FAB0
:10FF6000D8E9002300F030F900F07AFD804600F077
:10FF700077FA77A3D3E9002306460F4600F0D6FAB6
:10FF800002460B462846214600F01CF972A3D3E92D
:10FF90000023CDE900013046394600F0C7FA824619
:10FFA0008B4652465B46DDE9000100F00BF9054641
:10FFB0000C462A4623462846214600F0B7FA68A395
:10FFC000D3E9002306460F4600F0B0FA66A3D3E952
:10FFD000002300F0F7F832463B4600F0A7FA64A38E
:10FFE000D3E9002300F0F0F832463B4600F09EFAD9
:10FFF00061A3D3E9002300F0E5F832463B4600F068
:020000021000EC
:1000000095FA5FA3D3E9002300F0DEF832463B46C1
:1000100000F08CFA02460B462846214600F0D2F842
:1000200006460F462846214632463B46B8F1000FA9
:1000300056D000F07BFA324604460D463B4600207F
:100040004FF0804100F0BEF802460B46204629469C
:1000500000F096FB02460B465046594600F0B2F8B7
:10006000DDE9002300F0AEF80B4602464A490020C5
:1000700000F0A8F86FF47F7398454FDA08F57A78A6
:1000800001EB085100224FF0B87300F04FFA03B0B3
:10009000BDE8F08F424B9A423FF658AF414BF40017
:1000A0002344D3E9002300F08DF83F4BC6F101084B
:1000B0001C44CDE90001D4E900ABC6EB080870E7A9
:1000C0004FF0000875E702460B4600F07DF80EE79A
:1000D00017A3D3E900231046194600F027FA06E7D4
:1000E00000F024FA0022804689464FF080433046D3
:1000F000394600F067F802460B464046494600F094
:100100003FFB2A46234600F05DF802460B460020DE
:10011000214900F057F803B0BDE8F08F01EB08511A
:1001200003B0BDE8F08F804643E700BFAFF3008027
:100130009C7500883CE4377EEF39FAFE422E8640FB
:1001400051302DD5104987C0FE822B654715F73FEA
:100150000000E0FE422EE63F763C7935EF39EA3D7D
:10016000D0A4BE726937663EF16BD2C541BDBB3EBD
:100170002CDE25AF6A56113F93BDBE166CC1663F9B
:100180003E5555555555C53F412E8640FFFFEF7FE3
:10019000422ED63FFFFF2F3E0000F03F504B0100A4
:1001A000B1A2F03F704B0100604B010041F00041F3
:1001B00001F58010C00F70470020704781F00041AA
:1001C00002E000BF83F0004330B54FEA41044FEA3C
:1001D000430594EA050F08BF90EA020F1FBF54EAD7
:1001E000000C55EA020C7FEA645C7FEA655C00F073
:1001F000E2804FEA5454D4EB5555B8BF6D420CDD44
:100200002C4480EA020281EA030382EA000083EAC6
:10021000010180EA020281EA0303362D88BF30BD66
:1002200011F0004F4FEA01314FF4801C4CEA1131BC
:1002300002D0404261EB410113F0004F4FEA03331B
:100240004CEA133302D0524263EB430394EA050FA6
:1002500000F0A780A4F10104D5F1200E0DDB02FA15
:100260000EFC22FA05F2801841F1000103FA0EF2A9
:10027000801843FA05F359410EE0A5F120050EF16F
:10028000200E012A03FA0EFC28BF4CF0020C43FAA0
:1002900005F3C01851EBE37101F0004507D54FF0AD
:1002A000000EDCF1000C7EEB00006EEB0101B1F5FD
:1002B000801F1BD3B1F5001F0CD349085FEA300043
:1002C0004FEA3C0C04F101044FEA445212F5800F4E
:1002D00080F09A80BCF1004F08BF5FEA500C50F1EB
:1002E000000041EB045141EA050130BD5FEA4C0CCE
:1002F000404141EB010111F4801FA4F10104E9D157
:1003000091F0000F04BF01460020B1FA81F308BF4D
:100310002033A3F10B03B3F120020CDA0C3208DD19
:1003200002F1140CC2F10C0201FA0CF021FA02F1F4
:100330000CE002F11402D8BFC2F1200C01FA02F164
:1003400020FA0CFCDCBF41EA0C019040E41AA2BF89
:1003500001EB0451294330BD6FEA04041F3C1CDA51
:100360000C340EDC04F11404C4F1200220FA04F071
:1003700001FA02F340EA030021FA04F345EA03011B
:1003800030BDC4F10C04C4F1200220FA02F001FADD
:1003900004F340EA0300294630BD21FA04F029465F
:1003A00030BD94F0000F83F4801306BF81F48011F8
:1003B0000134013D4EE77FEA645C18BF7FEA655C6B
:1003C00029D094EA050F08BF90EA020F05D054EA3D
:1003D000000C04BF1946104630BD91EA030F1EBF42
:1003E0000021002030BD5FEA545C05D14000494146
:1003F00028BF41F0004130BD14F580043CBF01F539
:10040000801130BD01F0004545F0FE4141F470011E
:100410004FF0000030BD7FEA645C1ABF19461046F9
:100420007FEA655C1CBF0B46024650EA013406BFFA
:1004300052EA033591EA030F41F4002130BD00BFB9
:1004400090F0000F04BF0021704730B54FF4806476
:1004500004F132044FF000054FF0000150E700BFF7
:1004600090F0000F04BF0021704730B54FF4806456
:1004700004F1320410F0004548BF40424FF0000143
:100480003EE700BF42004FEAE2014FEA31014FEA86
:1004900002701FBF12F07F4393F07F4F81F06051D5
:1004A000704792F0000F14BF93F07F4F704730B544
:1004B0004FF4607401F0004521F0004120E700BFD7
:1004C00050EA010208BF704730B54FF000050AE05E
:1004D00050EA010208BF704730B511F0004502D55F
:1004E000404261EB41014FF4806404F132045FEA61
:1004F000915C3FF4DCAE4FF003025FEADC0C18BF06
:1005000003325FEADC0C18BF033202EBDC02C2F1FB
:10051000200300FA03FC20FA02F001FA03FE40EA8D
:100520000E0021FA02F11444C1E600BF70B54FF08D
:10053000FF0C4CF4E06C1CEA11541DBF1CEA13556F
:1005400094EA0C0F95EA0C0F00F0DEF82C4481EAD7
:10055000030621EA4C5123EA4C5350EA013518BFF7
:1005600052EA033541F4801143F4801338D0A0FBE4
:1005700002CE4FF00005E1FB02E506F00042E0FB91
:1005800003E54FF00006E1FB03569CF0000F18BF97
:100590004EF0010EA4F1FF04B6F5007F64F540743F
:1005A00004D25FEA4E0E6D4146EB060642EAC621D2
:1005B00041EA55514FEAC52040EA5E504FEACE2E3F
:1005C000B4F1FD0C88BFBCF5E06F1ED8BEF1004F42
:1005D00008BF5FEA500E50F1000041EB045170BDBE
:1005E00006F0004646EA010140EA020081EA030102
:1005F000B4EB5C04C2BFD4EB0C0541EA045170BDFE
:1006000041F480114FF0000E013C00F3AB8014F177
:10061000360FDEBF002001F0004170BDC4F10004C0
:10062000203C35DA0C341BDC04F11404C4F1200541
:1006300000FA05F320FA04F001FA05F240EA02009C
:1006400001F0004221F0004110EBD37021FA04F6D2
:1006500042EB06015EEA430E08BF20EAD37070BD8C
:10066000C4F10C04C4F1200500FA04F320FA05F0EB
:1006700001FA04F240EA020001F0004110EBD370ED
:1006800041F100015EEA430E08BF20EAD37070BD5D
:10069000C4F1200500FA05F24EEA020E20FA04F336
:1006A00001FA05F243EA020321FA04F001F00041E5
:1006B00021FA04F220EA020000EBD3705EEA430E56
:1006C00008BF20EAD37070BD94F0000F0FD101F085
:1006D0000046400041EB010111F4801F08BF013CBE
:1006E000F7D041EA060195F0000F18BF704703F0FC
:1006F0000046520043EB030313F4801F08BF013D83
:10070000F7D043EA0603704794EA0C0F0CEA13553E
:1007100018BF95EA0C0F0CD050EA410618BF52EAF8
:100720004306D1D181EA030101F000414FF00000FE
:1007300070BD50EA410606BF1046194652EA43060C
:1007400019D094EA0C0F02D150EA013613D195EA80
:100750000C0F05D152EA03361CBF104619460AD1C8
:1007600081EA030101F0004141F0FE4141F47001D2
:100770004FF0000070BD41F0FE4141F4780170BDC2
:1007800070B54FF0FF0C4CF4E06C1CEA11541DBF27
:100790001CEA135594EA0C0F95EA0C0F00F0A7F829
:1007A000A4EB050481EA030E52EA03354FEA013156
:1007B00000F088804FEA03334FF0805545EA131369
:1007C00043EA12634FEA022245EA111545EA106531
:1007D0004FEA00260EF000419D4208BF964244F1C8
:1007E000FD0404F5407402D25B084FEA3202B61AE7
:1007F00065EB03055B084FEA32024FF480104FF4BB
:10080000002CB6EB020E75EB030E22BFB61A75462E
:1008100040EA0C005B084FEA3202B6EB020E75EBC1
:10082000030E22BFB61A754640EA5C005B084FEA29
:100830003202B6EB020E75EB030E22BFB61A7546F6
:1008400040EA9C005B084FEA3202B6EB020E75EB01
:10085000030E22BFB61A754640EADC0055EA060EC2
:1008600018D04FEA051545EA16754FEA06164FEA05
:10087000C30343EA52734FEAC2025FEA1C1CC0D1B1
:1008800011F4801F0BD141EA00014FF000004FF03E
:10089000004CB6E711F4801F04BF01430020B4F1FF
:1008A000FD0C88BFBCF5E06F3FF6AFAEB5EB030CB7
:1008B00004BFB6EB020C5FEA500C50F1000041EBB4
:1008C000045170BD0EF0004E4EEA113114EB5C0481
:1008D000C2BFD4EB0C0541EA045170BD41F4801154
:1008E0004FF0000E013C90E645EA060E8DE60CEA5C
:1008F000135594EA0C0F08BF95EA0C0F3FF43BAF79
:1009000094EA0C0F0AD150EA01347FF434AF95EA2F
:100910000C0F7FF425AF104619462CE795EA0C0F13
:1009200006D152EA03353FF4FDAE1046194622E7E0
:1009300050EA410618BF52EA43067FF4C5AE50EABA
:1009400041047FF40DAF52EA43057FF4EBAE12E7AA
:100950004FF0FF3C06E000BF4FF0010C02E000BF8B
:100960004FF0010C4DF804CD4FEA410C7FEA6C5C6E
:100970004FEA430C18BF7FEA6C5C1BD001B050EA11
:10098000410C0CBF52EA430C91EA030F02BF90EAFC
:10099000020F0020704710F1000F91EA030F58BFBB
:1009A000994208BF90422CBFD8176FEAE37040F01D
:1009B000010070474FEA410C7FEA6C5C02D150EABB
:1009C000013C07D14FEA430C7FEA6C5CD6D152EA76
:1009D000033CD3D05DF8040B704700BF844610463B
:1009E00062468C461946634600E000BF01B5FFF73A
:1009F000B7FF002848BF10F1000F01BD4DF808ED0A
:100A0000FFF7F4FF0CBF012000205DF808FB00BFDA
:100A10004DF808EDFFF7EAFF34BF012000205DF834
:100A200008FB00BF4DF808EDFFF7E0FF94BF012081
:100A300000205DF808FB00BF4DF808EDFFF7CEFF82
:100A400094BF012000205DF808FB00BF4DF808EDC1
:100A5000FFF7C4FF34BF012000205DF808FB00BF92
:100A60004FEA410212F5001215D211D56FF47873D6
:100A7000B3EB625212D94FEAC12343F0004343EA79
:100A8000505311F0004F23FA02F018BF4042704754
:100A90004FF00000704750EA013005D111F00040DE
:100AA00008BF6FF0004070474FF00000704700BF74
:100AB0004FEA4102B2F1E04324BFB3F5001CDCF180
:100AC000FE5C0DD901F0004C4FEAC0024CEA5070B8
:100AD000B2F1004F40EB830008BF20F001007047E7
:100AE00011F0804F21D113F13872BCBF01F00040EA
:100AF000704741F480114FEA5252C2F11802C2F11C
:100B0000200C10FA0CF320FA02F018BF40F001009C
:100B10004FEAC1234FEAD32303FA0CFC40EA0C004E
:100B200023FA02F34FEA4303CCE77FEA625307D18B
:100B300050EA01331EBF4FF0FE4040F440007047C2
:100B400001F0004040F0FE4040F40000704700BF5C
:100B500080F0004002E000BF81F0004142001FBF72
:100B60005FEA410392EA030F7FEA226C7FEA236C7B
:100B70006AD04FEA1262D2EB1363C1BFD218414070
:100B800048404140B8BF5B42192B88BF704710F006
:100B9000004F40F4000020F07F4018BF404211F0A9
:100BA000004F41F4000121F07F4118BF494292EA11
:100BB000030F3FD0A2F1010241FA03FC10EB0C003D
:100BC000C3F1200301FA03F100F0004302D54942CA
:100BD00060EB4000B0F5000F13D3B0F1807F06D377
:100BE00040084FEA310102F10102FE2A51D2B1F16F
:100BF000004F40EBC25008BF20F0010040EA030064
:100C00007047490040EB000010F4000FA2F1010210
:100C1000EDD1B0FA80FCACF1080CB2EB0C0200FA9A
:100C20000CF0AABF00EBC25052421843BCBFD040E8
:100C30001843704792F0000F81F4000106BF80F462
:100C400000000132013BB5E74FEA41037FEA226C25
:100C500018BF7FEA236C21D092EA030F04D092F0F0
:100C6000000F08BF0846704790EA010F1CBF002024
:100C7000704712F07F4F04D1400028BF40F0004081
:100C8000704712F100723CBF00F50000704700F0A1
:100C9000004343F0FE4040F4000070477FEA2262C8
:100CA00016BF08467FEA23630146420206BF5FEA99
:100CB000412390EA010F40F4800070474FF0000399
:100CC00004E000BF10F0004348BF40425FEA000C60
:100CD00008BF704743F0964301464FF000001CE008
:100CE00050EA010208BF70474FF000030AE000BF5E
:100CF00050EA010208BF704711F0004302D540429C
:100D000061EB41015FEA010C02BF8446014600200D
:100D100043F0B64308BFA3F18053A3F50003BCFA28
:100D20008CF2083AA3EBC25310DB01FA02FC6344D5
:100D300000FA02FCC2F12002BCF1004F20FA02F2DC
:100D400043EB020008BF20F00100704702F12002CF
:100D500001FA02FCC2F1200250EA4C0021FA02F230
:100D600043EB020008BF20EADC7070474FF0FF0C35
:100D70001CEAD0521EBF1CEAD15392EA0C0F93EA30
:100D80000C0F6FD01A4480EA010C400218BF5FEAD2
:100D900041211ED04FF0006343EA501043EA511145
:100DA000A0FB01310CF00040B1F5000F3EBF49003F
:100DB00041EAD3715B0040EA010062F17F02FD2A43
:100DC0001DD8B3F1004F40EBC25008BF20F0010026
:100DD000704790F0000F0CF0004C08BF49024CEA3D
:100DE000502040EA51207F3AC2BFD2F1FF0340EACF
:100DF000C250704740F400004FF00003013A5DDC40
:100E000012F1190FDCBF00F000407047C2F1000280
:100E1000410021FA02F1C2F1200200FA02FC5FEA6D
:100E2000310040F1000053EA4C0308BF20EADC70B7
:100E3000704792F0000F00F0004C02BF400010F429
:100E4000000F013AF9D040EA0C0093F0000F01F0D6
:100E5000004C02BF490011F4000F013BF9D041EAF8
:100E60000C018FE70CEAD15392EA0C0F18BF93EAFA
:100E70000C0F0AD030F0004C18BF31F0004CD8D124
:100E800080EA010000F00040704790F0000F17BFAB
:100E900090F0004F084691F0000F91F0004F14D0F1
:100EA00092EA0C0F01D142020FD193EA0C0F03D149
:100EB0004B0218BF084608D180EA010000F000404C
:100EC00040F0FE4040F40000704740F0FE4040F427
:100ED000400070474FF0FF0C1CEAD0521EBF1CEAC6
:100EE000D15392EA0C0F93EA0C0F69D0A2EB0302E4
:100EF00080EA010C49024FEA402037D04FF080537E
:100F000043EA111143EA10130CF000408B4238BF42
:100F10005B0042F17D024FF4000C8B4224BF5B1A50
:100F200040EA0C00B3EB510F24BFA3EB510340EA9E
:100F30005C00B3EB910F24BFA3EB910340EA9C004C
:100F4000B3EBD10F24BFA3EBD10340EADC001B01BC
:100F500018BF5FEA1C1CE0D1FD2A3FF650AF8B4260
:100F600040EBC25008BF20F0010070470CF0004C6D
:100F70004CEA50207F32C2BFD2F1FF0340EAC25098
:100F8000704740F400004FF00003013A37E792F059
:100F9000000F00F0004C02BF400010F4000F013AB7
:100FA000F9D040EA0C0093F0000F01F0004C02BFB2
:100FB000490011F4000F013BF9D041EA0C0195E71B
:100FC0000CEAD15392EA0C0F08D142027FF47DAFB4
:100FD00093EA0C0F7FF470AF084676E793EA0C0FA4
:100FE00004D14B023FF44CAF08466EE730F0004CA2
:100FF00018BF31F0004CCAD130F000427FF45CAF32
:1010000031F000437FF43CAF5FE700BF4FF0FF3C9F
:1010100006E000BF4FF0010C02E000BF4FF0010CF2
:101020004DF804CD4FEA40024FEA41037FEA226CBB
:1010300018BF7FEA236C11D001B052EA530C18BFDD
:1010400090EA010F58BFB2EB030088BFC81738BF42
:101050006FEAE17018BF40F0010070477FEA226C30
:1010600002D15FEA402C05D17FEA236CE4D15FEA2C
:10107000412CE1D05DF8040B704700BF8446084660
:101080006146FFE70FB5FFF7C9FF002848BF10F121
:10109000000F0FBD4DF808EDFFF7F4FF0CBF012066
:1010A00000205DF808FB00BF4DF808EDFFF7EAFFF0
:1010B00034BF012000205DF808FB00BF4DF808EDAB
:1010C000FFF7E0FF94BF012000205DF808FB00BFA0
:1010D0004DF808EDFFF7D2FF94BF012000205DF826
:1010E00008FB00BF4DF808EDFFF7C8FF34BF012033
:1010F00000205DF808FB00BF4FEA4002B2F1FE4F4E
:101100000FD34FF09E03B3EB12620DD94FEA0023C9
:1011100043F0004310F0004F23FA02F018BF4042A2
:1011200070474FF00000704712F1610F01D1420289
:1011300005D110F0004008BF6FF0004070474FF03D
:101140000000704742000ED2B2F1FE4F0BD34FF0B9
:101150009E03B3EB126209D44FEA002343F000432D
:1011600023FA02F070474FF00000704712F1610F50
:1011700001D1420202D14FF0FF3070474FF0000022
:10118000704700BF0B460146184600F001B800BF8B
:1011900013460A460146022000F0C4BE014B1868FF
:1011A000704700BF5898FF1F70B50F4E0F4D761B4C
:1011B000B61018BF002405D0013455F8043B9847F9
:1011C000A642F9D10A4E0B4D761B03F0DBFCB6109C
:1011D00018BF002406D0013455F8043B9847A642B6
:1011E000F9D170BD70BD00BF904B0100904B010064
:1011F000A44B0100904B0100024B0146186800F01F
:101200000BB800BF5898FF1F024B0146186800F04A
:101210004DBF00BF5898FF1F2DE9F04F01F10B059E
:10122000162D83B0064640F29F8035F0070500F189
:10123000BF80A94200F2BC8000F058FBB5F5FC7FEE
:10124000C0F09C826B0A00F0BA80042B00F283810C
:10125000A80900F1390E4FEA4E033830C44F07EBAE
:101260008303A3F108015C68A14207D1ACE0002A26
:1012700080F2AC80E468A14200F0A680636823F0AD
:1012800003035A1B0F2AF2DDB9493C6901F1080E2C
:10129000744500F0B381636823F003035A1B0F2ADF
:1012A00000F39981002AC1F814E0C1F810E080F23F
:1012B0009E80B3F5007F80F06781DB0803F1010CAD
:1012C00001229B1002FA03F34A6851F83C80C4F8EB
:1012D000088001EBCC091A43A9F10803E3604A60D6
:1012E00041F83C40C8F80C40831001249C409442D3
:1012F00000F28A80144206D120F0030064001442F8
:1013000000F10400FAD007EBC009CC468046DCF8B7
:101310000C108C4507D173E1002A80F28181C968E5
:101320008C4500F06D814B6823F003035A1B0F2A94
:10133000F2DD0C46D1F80CC054F8088F4B1945F07B
:1013400001054D6042F00101C8F80CC03046CCF8F0
:1013500008807B613B61C3F80CE0C3F808E059608A
:101360009A5000F0C5FA1FE0102921D800F0BEFA0B
:101370001025062302207E4F07EB8303A3F108020A
:101380005C68944200F045816368E168A56823F0D9
:101390000303234430465A68E96042F001028D603D
:1013A0005A6000F0A5FA0834204603B0BDE8F08F7B
:1013B00000240C232046336003B0BDE8F08F802367
:1013C0004FF0400E3F2049E770465DE72344E16857
:1013D0005A68A56842F00102E96030468D605A60A3
:1013E00000F086FA0834204603B0BDE8F08F2344AD
:1013F00030465A6842F001025A6000F079FA083427
:10140000204603B0BDE8F08FBC68636823F0030892
:10141000A84504D3C5EB08030F2B00F38C80554B74
:10142000DFF860911A68D9F8003001332A4404EBE0
:10143000080A00F0608102F580520F3222F47F62C8
:1014400022F00F0211463046019200F04BFCB0F141
:10145000FF3F8346019A00F05881824500F2FC80EC
:10146000454B1968DA451144196000F05381D9F8E9
:101470000000DFF810E101301BBFCAEB0B0A51443A
:10148000CEF800B019601BF0070100F01781C1F120
:101490000800C1F58051834408315A44C2F30B025D
:1014A000C2EB010949463046019300F01BFC431C86
:1014B000019B00F03F81CBEB00024A4442F0010265
:1014C0001968C7F808B04944BC42CBF80420196039
:1014D000DFF8A49016D0B8F10F0F40F2FD806268DB
:1014E000A8F10C0323F00703E01802F001024FF00B
:1014F000050E1A430F2B6260C0F804E0C0F808E044
:1015000000F21C811D4BBC681A68914288BF1960AB
:101510001B4B1A689142626888BF196022F003026F
:101520009542A2EB050301D80F2B04DC304600F0F6
:10153000DFF9002438E7621943F0010345F00105A3
:1015400065603046BA60536000F0D2F90834204636
:1015500003B0BDE8F08F142B71D9542B00F2A48096
:10156000280B00F16F0E4FEA4E036E3076E600BF97
:101570005C98FF1F40A3FF1F44A3FF1F3CA3FF1F56
:1015800038A3FF1F689CFF1F5A0A042A5ED9142A39
:1015900000F2B38002F15C0149005B3207EB810C81
:1015A00057F82110DFF8DC81ACF1080C8C4500F015
:1015B00088804A6822F00302934202D289688C45EF
:1015C000F7D1D1F80CC07A68C4F80CC0A160CCF88F
:1015D0000840CC6088E6631942F0010745F0010538
:1015E000656030464B610B61C3F80CE0C3F808E05E
:1015F0005F609A50083400F07BF9D5E64A6873E6DC
:1016000008F1010818F0030F0CF1080C7FF47FAE0D
:1016100030E0DC68A34208BF02303FF435AEB3E6E9
:101620000B440C465A68C96854F8085F42F001023E
:101630005A603046E9608D6000F05AF9B4E603F173
:101640005C0E03F15B004FEA4E0307E69A0902F1D4
:10165000390149003832A1E7BC424A4B3FF400AFA0
:101660009C68626822F003025AE759F808399945E4
:1016700040F0828010F0030F00F1FF30F5D17B685D
:1016800023EA04037B6064009C423FF6BDAE002C5D
:101690003FF4BAAE1C4240467FF435AE64001C42B3
:1016A00000F10400FAD02EE6B3F5AA7F18D8E80BB3
:1016B00000F1780E4FEA4E037730CFE54FF48051BA
:1016C000EBE60121D8F80430921001FA02F21A4335
:1016D000C8F80420614677E70123CBF8043025E7FA
:1016E00040F25452934220D8A80C00F17D0E4FEAEC
:1016F0004E037C30B2E51032A4E6542A26D81A0BE9
:1017000002F16F0149006E3248E7BC68626822F05E
:10171000030205E7CAF30B0000287FF4A8AE424499
:10172000BB6842F001025A60ECE6FE234FF07F0EE8
:101730007E2093E501224FF00009C1E604F1080183
:10174000304600F0B3FCD9F80010DBE6B2F5AA7F12
:1017500005D8DA0B02F17801490077321EE740F232
:1017600054518A4205D89A0C02F17D0149007C321D
:1017700014E7FE217E2211E77B6884E7E808431C1A
:101780005B00F8E55C98FF1F8842F0B50DD98B1817
:1017900098420AD28118002A51D09A1A13F8014DA2
:1017A00001F8014D9342F9D1F0BD0F2A48D941EA21
:1017B00000039B0746D100F1100401F11003154608
:1017C00053F8106C44F8106C53F80C6C44F80C6C23
:1017D00053F8086C44F8086C103D53F8046C44F856
:1017E000046C0F2D03F1100304F11004E8D8A2F1EA
:1017F000100323F00F0302F00F0E1033BEF1030F9E
:101800001944034421D91E1F0D467446043C55F863
:10181000047B46F8047F032CF8D8AEF1040424F0CE
:10182000030404342344214402F0030262B1013B67
:101830000A4411F8014B03F8014F8A42F9D1F0BD77
:101840000346F3E70346F2E7F0BD7246EEE700BF5A
:1018500070B4840746D0541E002A41D0CDB203464E
:1018600002E0621EE4B3144603F8015B9A07F8D164
:10187000032C2ED9CDB245EA05250F2C45EA0545A6
:1018800019D903F110022646103E0F2E42F8105CC3
:1018900042F80C5C42F8085C42F8045C02F1100269
:1018A000F2D8A4F1100222F00F0204F00F0410325B
:1018B000032C13440DD91E462246043A032A46F847
:1018C000045BFAD8221F22F003020432134404F00E
:1018D00003042CB1C9B21C4403F8011BA342FBD181
:1018E00070BC704714460346C2E700BF704700BF94
:1018F000704700BF024B0A460146186800F002B864
:101900005898FF1F2DE9F04F174683B0002900F0CB
:10191000C1800E46814607F10B05FFF7E7FF56F839
:1019200004EC162D2EF00304A6F1080840D810226E
:101930001546AF4241D8944275DAC94B996808EB15
:1019400004008842416800F0D98021F0010303447B
:101950005B68DB077DD51EF0010F35D03946484660
:10196000FFF75AFC0746E0B156F8043C23F00103A8
:101970004344A0F108029A4200F04481221F242A25
:1019800000F23181132A00F20481034632461168C5
:1019900019605168596092689A603146484600F073
:1019A00085FB4846FFF7A4FF384603B0BDE8F08F3B
:1019B00025F00705002D2A46BBDA0C230020C9F8C4
:1019C000003003B0BDE8F08F56F8083CC3EB080ABE
:1019D000DAF8043023F0030C04EB0C039342BDDB74
:1019E0005746DAF80C1057F8080F221F242AC16056
:1019F000886000F21781132A40F212813168CAF818
:101A000008107168CAF80C101B2A00F22B810836E6
:101A10000AF110023168116071685160B16891601B
:101A20003E461C46D046631B0F2B1DD8D8F8043009
:101A300003F0010323434444C8F80430636843F0CF
:101A4000010363604846FFF753FF304603B0BDE82B
:101A5000F08F21F003012144914221DBC3688268A9
:101A60000C46D3609A60DEE7D8F8042008EB050145
:101A700002F00102154343F001020B44C8F8045080
:101A80004A605A6842F0010208315A60484600F044
:101A90000DFBD7E7114603B0BDE8F04FFFF7BCBB25
:101AA0001EF0010F7FF45AAF56F8083CC3EB080A4A
:101AB000DAF8043023F0030C01EB0C0E96458BDBB7
:101AC000C36882685746D3609A6057F8081FDAF8EF
:101AD0000C30CB60221F242A996000F29980132ACF
:101AE00062D93368CAF808307368CAF80C301B2A08
:101AF00000F2A08008360AF1100356E021F0030B33
:101B0000A34405F11000834559DA1EF0010F7FF45C
:101B100025AF56F8081CC1EB080ADAF8041021F0CA
:101B2000030CE34458453FF757AF5746DAF80C101B
:101B300057F8080F221F242AC160886000F2B48081
:101B4000132A40F2A5803168CAF808107168CAF8F3
:101B50000C101B2A00F2AF8008360AF1100231681F
:101B6000116071685160B16891600AEB0501C5EBC5
:101B70000B0242F0010299604A60DAF8043003F087
:101B800001031D434846CAF80450FFF7B1FE38462A
:101B90005CE733680360736843601B2A27D800F151
:101BA000080306F10802F2E63B4632681A607268E2
:101BB0005A60B2689A603E467446D04633E708EBF6
:101BC0000501C5EB0B0B4BF0010299604A6056F81A
:101BD000043C03F001031D43484646F8045CFFF74C
:101BE00087FE304632E73146FFF7CEFDD5E6B368D3
:101BF0008360F368C360242A28D000F1100306F143
:101C00001002C4E650F8043C23F003031C440AE726
